:020000040800F2
:1000000000800020B9A5000891A5000893A500086C
:1000100095A5000897A5000899A500080000000014
:100020000000000000000000000000009BA5000888
:100030009DA50008000000009FA50008A1A50008DC
:1000400009A6000809A6000809A6000809A60008D4
:1000500009A6000809A6000809A6000809A60008C4
:1000600009A6000809A6000809A6000809A60008B4
:1000700009A6000809A6000809A6000809A60008A4
:1000800009A600080000000009A6000809A600084B
:1000900009A6000869D6000809A6000809A60008F4
:1000A00009A6000809A6000809A6000809A6000874
:1000B000252B000809A6000809A6000809A60008C3
:1000C00009A6000809A6000809A6000809A6000854
:1000D00009A60008E9240008591E000809A600081E
:1000E0001D84000809A6000809A6000809A6000842
:1000F00009A6000809A6000809A6000800000000DB
:100100000000000009A600080000000009A6000881
:1001100009A600080000000009A6000809A60008BA
:1001200009A6000809A6000809A6000809A60008F3
:1001300009A60008000000000000000009A6000851
:1001400009A6000809A60008000000000000000041
:10015000000000000000000000000000000000009F
:1001600000000000000000000000000009A60008D8
:1001700009A60008000000000000000000000000C8
:100180000000000009A600080000000000000000B8
:10019000000000000000000000000000000000005F
:1001A000000000000000000009A6000809A60008E1
:1001B00009A6000809A6000809A60008000000001A
:1001C0000000000009A60008000000000000000078
:0801D00009A6000809A60008B9
:1001D80010B5054C237833B9044B13B10448AFF379
:1001E80000800123237010BD58000020000000008B
:1001F80084E3000808B5034B1BB103490348AFF378
:10020800008008BD000000005C00002084E30008B6
:1002180010F8012B11F8013B012A28BF9A42F7D0A8
:10022800D01A7047034613F8012B002AFBD1181A7D
:10023800013870470022427082700122C270B1FA00
:1002480081F102224909027103220170427170474B
:1002580043788B421FD0012941700AD0022910D05F
:10026800C1B90123C3708170022303710323437151
:100278007047037843B1012383700223C3700023BE
:10028800F3E70378002BF6D0022383700023C370B2
:100298000123EAE7FEE7704782B00B88ADF800302B
:1002A8004B88ADF802308B88ADF80430CB88ADF8B8
:1002B80006300239431C053013F8012F0DF1080CE4
:1002C8000CEB4202834232F8082C21F8022FF3D1BA
:1002D80002B0704701448878704738B54FF07F33D3
:1002E800C0F8A03004464FF6FF737F220025A0F81F
:1002F800A43080F8A62080F8A950A0F8AA30AC3025
:1003080000F0ABFE84F8B85038BD37B51546044642
:100318001146019300F08FFC294604F1140000F007
:100328008AFC294604F1280000F085FC294604F1DE
:100338003C0000F080FC294604F1500000F07BFCF2
:10034800294604F1640000F076FC294604F178009F
:1003580000F071FC294604F18C0000F06CFC04F1FB
:10036800AC00019A4FF4FA734FF4FA6100F060FEA2
:10037800204603B0BDE83040FFF7AFBF704700F03C
:1003880061BC143000F05EBC283000F05BBC90F813
:10039800A43013B990F9A000704790F9A1007047F4
:1003A80090F8A43013B990F9A200704790F9A3000F
:1003B800704710B5044608F0A5F938B104F11400E7
:1003C80000F044FC012838BF0120C0B210BD10B5B0
:1003D800044608F097F938B104F1500000F036FCF3
:1003E800012838BF0120C0B210BD4FF47A71AC307B
:1003F80000F03ABE0021AC3000F036BE08B5AC3093
:1004080000F041FEB0F57A7FA8BF4FF47A7020EA79
:10041800E07008BD10B5044600F0EEFB04F11400CE
:1004280000F0EAFB04F1280000F0E6FB04F13C00D0
:1004380000F0E2FB04F1500000F0DEFB04F1640080
:1004480000F0E6FB04F17800BDE8104000F0E0BBE6
:100458007F2807D0002807DA10F1800F06D0404225
:10046800C0B2704700207047012070477F20704756
:1004780010B1404240B270477F2070477F280FD0AC
:1004880010F1310F0EDA10F1780F0DDB7830FE2302
:1004980040B2584323304623B0FBF3F0C0B2704754
:1004A800FF207047FE207047002070477F2805D046
:1004B80031B1002806DA4042C0B27047FF207047C9
:1004C800FE207047002070477F2811D010F1310FAF
:1004D80010DA10F1780F10DB783040F2A96340B2DF
:1004E800584323304623B0FBF3F0AC3080B270475A
:1004F8000020704740F255707047AC207047632861
:100508009FBF40F2A9635843323064239DBFB0FBBC
:10051800F3F0AC3080B240F2557070474FF4F0639E
:10052800A0F58060584340F2FF7390FBF3F000F5AC
:10053800787080B27047FFF7F1BF4FF49663A0F56B
:100548008060584340F2FF7390FBF3F000F2DC50F8
:1005580080B27047A0F58060D0EB001048BF033030
:1005680040F38F007047032812DD0C2812DD0F2896
:1005780012DD122812DD162812DD192812DD1C28BA
:1005880012DD1F2812DD2128CCBFFF20062070476E
:1005980000207047012070470220704708207047EC
:1005A80003207047072070470420704705207047D4
:1005B80005289ABF014B185CFF207047FBE3000831
:1005C8007F281ABF4042C0B2002070477F2811D050
:1005D80010F1320F10DA884210DD401A6423C1F19D
:1005E800FF21584301F57F01CE31313090FBF1F006
:1005F800C0B27047FF2070476420704700207047E2
:10060800014B4140585C704704E400085AB110B4EB
:10061800054C0A4411F8013B58408A42205CF9D144
:100628005DF8044B7047704704E40008002809DBB4
:100638001F2809DC054B33F810000523B0FBF3F045
:10064800C0B2704700207047FA2070472EE50008B6
:10065800002805DB212805DC044B33F8100070471F
:10066800002070474FF4FA60704700BF2EE500087D
:10067800392808D822280ED9094B2338C0B2C340DC
:1006880003F0010070475F2807D0613819288CBF34
:10069800002001207047002070470120704700BFEC
:1006A80001EC7F00F8B50246451E461D00245F2771
:1006B80015F8010FFF2804BF0134E4B2FFF7D8FF93
:1006C80000B92F70AE42F3D1062C04D119B10B68D2
:1006D80013608B88938000239371F8BD2DE9F8434C
:1006E800DFF83490471E441D012500264FF02808E6
:1006F80017F8011F08480DF0E8FD034610B1A0EBFC
:100708000903DBB2A3FB05329E19A742A5FB0853D8
:10071800EED13046BDE8F88304E5000810B541790C
:10072800A1F13000C3B2092B07D80523B0FBF3F3BE
:1007380003EB8303C01AC0B210BD044C20460DF071
:10074800C4FD0028F1D0001BC0B2EEE704E50008A4
:1007580070B50446FFF766FD82B20023551E98B2B5
:10076800A84214FA83F104DA265C302E03F101035F
:10077800F5D0121A01322046BDE870400DF074BD64
:100788002DE9F04F0D4699B0164600211A461F462E
:1007980080460DF083FD00212A2201A800910DF06A
:1007A8007DFDDFF8CC90DFF8CCA0DFF8CCB005EB0E
:1007B8004606AE4211D16846FFF734FD30B100F16C
:1007C80060030DEB0300002300F8613C69464046D6
:1007D8000DF0BEFD19B0BDE8F08F35F9020B47F6F4
:1007E800FF739842E7D0002812DC59460CA80DF098
:1007F800AFFD6846FFF716FD04460CA8FFF712FD8B
:1008080020448742D5D30CA968460DF04FFDD0E7A8
:10081800B0F57A7F0BDA0CA980B20DF020F90CA89C
:10082800FFF796FF51460CA80DF040FDE1E7642361
:100838000CA93230B0FBF3F080B20DF010F90CA81F
:10084800FFF786FF0CA8FFF7EDFC00F15F036B4490
:1008580000F160010DEB010013F8302C00F8302C8A
:100868002E2203F8302C002300F82F3C4946DAE703
:10087800B8E30008B3E30008AEE30008F0B589B0B8
:100888006D4600242F468E1CE1B28A4204D83946B0
:10089800FFF776FF09B0F0BD36F8241025F8021BE3
:1008A8000134F1E742F210736421B0FBF3F203FB69
:1008B8001200B0FBF1F301FB130000EB023000EB78
:1008C800831080B2704770B50E4600210546144665
:1008D8000DF0E4FC00239AB2944200D870BDF25C9B
:1008E800002AFBD0EA540133F5E70000052911D8A6
:1008F800DFE801F00306080A0C0E0749FFF7E3BF1B
:100908000649FBE70649F9E70649F7E70649F5E727
:100918000649F3E70649F1E7BCE30008C1E300082C
:10092800C6E30008CBE30008D0E30008D5E30008DD
:10093800DAE30008052911D8DFE801F00306080A00
:100948000C0E0749FFF7BFBF0649FBE70649F9E761
:100958000649F7E70649F5E70649F3E70649F1E7E7
:10096800DCE30008E1E30008E6E30008EBE3000845
:10097800F0E30008F4E30008DAE3000870B50E4677
:1009880014460021013205460DF088FC00239AB276
:10099800944200D870BDF25C002AFBD0EA540133BF
:1009A800F5E77D23438043F2390309B2C36000238E
:1009B80001808180C3800372704700000268044987
:1009C800044B01FB023323F000430360180C70470B
:1009D800FD430300C39E2600F0B5002597B00160D3
:1009E800858004465622294668460DF057FC0126A4
:1009F800E27DAA4209D80023802104F1B800A3753A
:100A080017B0BDE8F0400DF049BC2046FFF7D6FF0F
:100A1800E7797B1B002190FBF3F202FB1300C0B2C5
:100A2800EC460A46CBB29F4223D800230022277BFC
:100A38001146D0B2874227D80029D9D1A279033AE2
:100A4800012A04EB050105D925B191F9172012BB3C
:100A5800012BCDD90B76A26852F82310583305F133
:100A68000E026B44013544F8221003F8586CEDB2BD
:100A7800BEE71CF801EBBEF1000F03D18242D5D0CE
:100A88000132D2B20131CDE72069805C013298424F
:100A980008BF0121CDE7501E8342DBDB01329342C0
:100AA800D8DCA5E72DE9F04F154697B0013D016068
:100AB800027104464371EDB25622002168469946F8
:100AC80000270DF0EBFB022D84BF4FF0010A002533
:100AD8003E4694F807809CBF4FF0030AB8FBFAF82B
:100AE800E27DB24209D80023802104F1B800A37541
:100AF80017B0BDE8F04F0DF0D1BB2046FFF75EFF01
:100B0800A8EB060390FBF3F202FB13030020DBB211
:100B1800EC460246C1B2414506D21CF801EBBEF1D3
:100B2800000F22D19A421ED1414528BF414601FB00
:100B38000A50002294F80CE000F0FF009446D3B26B
:100B48009E4514D8BCF1000FCAD1A3680FFA80FCE7
:100B580009F1FF3E53F82C20BEF1030F15D8DFE84A
:100B68000EF00E2A2D300132D2B20130D2E72369BD
:100B78009B5C0132834208BF4FF0010CDFE7DFF8CE
:100B880068E09644174A9645AAD916B117BB0129B9
:100B9800A6D9A2190F46107653F82C2006F10E0399
:100BA80044F8232001F1580301226B44164403F84A
:100BB800582CF6B294E7DFF834E0E2E7DFF830E0EB
:100BC800DFE7A2F53D02DFF82CE0A2F59D42443AAA
:100BD8007245D9E77A1E9142DBDB7A1C9142D8DC58
:100BE8007EE700BF3BB10100C54E47FF776245FF76
:100BF800287643FF3CB10100D0E901236421D31AD0
:100C0800C36082604B43418AB3FBF1F303747047BE
:100C1800D0E90123D31AC0E90223704743682BB1F6
:100C2800C26864214A43B2FBF3F2D3B203740023CF
:100C3800C360436070470023C0E9023341824360C8
:100C4800037470474368013343607047007C704702
:100C580043681944416070472DE9F0410D46044648
:100C68003522002128460DF019FB234610220021C9
:100C780028460CF078F8A31C0822102128460CF00E
:100C880072F8E31C0422182128460CF06CF8277926
:100C9800202F28BF202706344FF000080C2606FB1B
:100CA80008F1B84501F11C0105D3232316FB0730D1
:100CB800C008BDE8F08123460C2228460CF053F802
:100CC80008F101080234EAE72DE9F3410D4604462C
:100CD80040F27912002128460DF0E0FA234620223E
:100CE800002128460CF03FF8231D02222021284627
:100CF8000CF039F8631D0322222128460CF033F842
:100D0800A31D0322252128460CF02DF804F1080321
:100D18001022282128460CF026F804F11003082296
:100D2800382128460CF01FF804F11103082240214D
:100D380028460CF018F804F1120308224821284626
:100D48000CF011F804F114032022502128460CF06D
:100D58000AF804F118034022702128460CF003F821
:100D680004F120030822B02128460BF0FCFF04F10F
:100D780021030822B82128460BF0F5FF04F12207C9
:100D8800C0263B4631460822284608360BF0EBFFC2
:100D9800B6F5A07F07F10107F3D194F832308DF84A
:100DA800073008220DF10703314628460BF0DBFF18
:100DB800002704F133089DF80730FE009F4206F52E
:100DC800A47613D394F83281B8F1500F28BF4FF0AE
:100DD8005008002704F23314474506EBC7010ED329
:100DE80006EBC800C00802B0BDE8F08108EB0703B5
:100DF8000822314628460BF0B6FF0137DBE7E31936
:100E0800082228460BF0AFFF0137E5E713B5044683
:100E18000846002101602346C0F8031020220190F3
:100E28000BF0A1FF0198231D022220210BF09BFF4C
:100E38000198631D032222210BF095FF0198A31D41
:100E4800032225210BF08FFF019804F108031022DB
:100E580028210BF088FF072002B010BDF7B500234A
:100E68000C4600910722194605460BF043FE631C09
:100E7800009301220023072128460BF03BFEAB8A92
:100E8800013B03F0FF03102BA37018D80023E71CC5
:100E9800A2785E1C93424FEAC60107D3AB8AB3EB34
:100EA800D10F14BF0120002003B0F0BD3B440093D4
:100EB8000822002328460BF01DFE3346E8E70120F0
:100EC800F2E7F8B50D4604467F22002128460DF0CA
:100ED800E5F923460822002128460BF044FF631C4D
:100EE8000722082128460BF03EFFA31C05220F21EC
:100EF80028460BF038FFE31C0422142128460BF087
:100F080032FF1822231D114628460BF02CFF267AA3
:100F1800782E28BF782600270934F900B74201F156
:100F2800300103D3F0003730C008F8BDE3190822B8
:100F380028460BF018FF0137EFE7F7B500230C46FA
:100F480000910822194605460BF0D4FD631C009356
:100F580007220023082128460BF0CCFDA31C009390
:100F6800052201230F2128460BF0C4FDE31C009342
:100F780004220023142128460BF0BCFD231D18224F
:100F880000931146002328460BF0B4FDAB8A063BBC
:100F980003F0FF03782B23721AD8002604F10907FF
:100FA800227AF300964203F1300108D3AA8A373334
:100FB800B2EBD30F14BF0120002003B0F0BDBB1962
:100FC80000930822002328460BF094FD0136E7E73A
:100FD8000120F2E70023C0E90133C36003747047BE
:100FE800F0B5047C0360012C11D944688568C66893
:100FF800141B4FF47A774D1B7C4305FB16442B4496
:1010080094FBF3F33344C360C0E90121F0BD1CB97C
:10101800C46001230374F7E743684FF47A74D31A62
:10102800634384680C1B93FBF4F3C3600223F1E76A
:1010380007EE902A0A44F8EE676A07EE902AF8EE5F
:10104800677A436086EEA77A07EE903AF8EEE77A79
:1010580080ED007AC0ED027A7047D0ED017AF8EEA3
:10106800E77AC0ED027A704707EE901A90ED027A9F
:10107800D0ED006AF8EEE77A77EEC77AA6EEA77A9F
:1010880080ED027A7047D0ED027AB6EE007A77EEFC
:10109800877AFDEEE77A17EE900A70477047704737
:1010A8007047002070477047002070470020704745
:1010B800704700207047002070470000054BDA6C2D
:1010C8000243DA64DB6C82B003400193019B02B0F7
:1010D800704700BF00100240054B9A6D02439A65A5
:1010E8009B6D82B003400193019B02B0704700BF23
:1010F80000100240054B1A6E02431A661B6E82B03E
:1011080003400193019B02B0704700BF00100240EA
:1011180050E8003F23F0800340E80032002AF7D16E
:10112800704770470288044B5140C9B233F81130F8
:1011380083EA1223038070475CFF0008A2B110B451
:10114800B0F800C0094C0A4411F8013B83EA0C03CB
:10115800DBB2914234F8133083EA1C2CA0F800C0AB
:10116800F2D15DF8044B7047704700BF5CFF000880
:1011780037B54FF6FF730446ADF806304518AC4254
:1011880003D1BDF8060003B030BD14F8011B0DF102
:101198000600FFF7C7FFF2E7074A00231380074A54
:1011A8001380074A1380074A1380074AD362A2F8BC
:1011B8003438A2F8323870478A4600208C4600201E
:1011C8008E4A0020904A0020B0130020014B187866
:1011D800704700BF000000200278024B51405B5C62
:1011E8000370704770EB0008FF230370704700BF5F
:1011F800704770B50B7803704B7843700B78FD2BF4
:1012080005460C4638D18B788370CB78C3700B7940
:1012180003714B7943718B7983718B68C3718B68C8
:10122800C3F30F2303728B7A43720A26627804F1A0
:101238000C01A8190DF094F86378B4F80C21334424
:10124800981CEA545A1CB4F80C1192B2090AA95411
:10125800A278D20780B20ED504F58872054404F549
:101268008E7452F8041B45F8041BA242F9D1127877
:101278002A700F3398B270BD00238B700B7983707E
:101288004B79C3708B7903718B6843710626CDE760
:1012980008B52422034800210DF000F8024B002273
:1012A8001A7008BDA0230020280300202DE9F04172
:1012B8001378037092F8018080F80180FD2B0446B2
:1012C8000F46154654D193788370D378C370137939
:1012D800037153794371937983716B7A127A1B0482
:1012E80003EB0223EA79134423F07F430A26A2681A
:1012F80063F31702A260A919424604F10C000DF02D
:101308002FF87A7B904507D208F10C00A2EB08026F
:10131800002120440CF0C2FF63781E44AB195A78B0
:10132800AB5D03EB0223A4F80C31A378DB070ED5E1
:10133800023615FA86F304F5887203F10C0153F8A6
:10134800040B42F8040B8B42F9D11B781370BB7A5B
:1013580084F82131FB7A84F822313B7B84F82331ED
:101368007B7B84F824313B7884F82031BDE8F08118
:101378000023438093780371D37843711379837181
:1013880053790626B3E7000070B50D4C0D4E05469F
:10139800062204F10A0106F58970FFF7EFFA237CAB
:1013A800C3F3031386F81A31637CC3F3030386F887
:1013B8001B31637ADB0744BF02232B7370BD00BF68
:1013C800753C0020D400002070B50446BDF81450C8
:1013D800E2702420237122461B0A20706371582072
:1013E8002B0AA1706070A57102F8073F049B591978
:1013F8008B420CD16A1D92B2E11C0020FFF706F95E
:1014080005F10806A05505F1090080B270BD13F872
:10141800010B02F8010FEBE70A4A0B4B12680B4964
:10142800A3FB02323220920C00FB02F2084B486800
:1014380002F5FA72A3FB023292094B681B1A9A4210
:10144800FBD870472C00002083DE1B43001000E00F
:10145800D34D621008B5FFF7DFFF4FF0904310221D
:101468009A6108BD4FF0904310229A62FFF7D4BFEB
:1014780002780A4B90F801C08178D243D2B29A5CC4
:1014880082EA0C0290F803C09A5C4A40995C02799F
:1014980081EA0C01595C4A40985C704770EB00087F
:1014A800F8B53C29BDF81C50044635D0A1F12106F9
:1014B800714271414900D00748BF41F00801E3700B
:1014C80092074FEA13234FF0240248BF41F010015E
:1014D800227023716F222B0AA61C6270A170A3715F
:1014E80065713046FFF7C4FF2246069B02F8070FD6
:1014F80059198B4212D1A91D89B23046FFF738FE1F
:1015080005F1080705F109039BB2E055000AE0540C
:1015180005F10A0080B2F8BD0121CCE713F8010BF0
:1015280002F8010FE5E70000074B084A5B6A02F57D
:10153800006353E8003F43F0200302F5006040E8F1
:1015480000310029F3D170470038014000300140D4
:101558002DE9F04F0C465188B1F58C7F85B00546D2
:1015680011D300211170D91CC9B2012995BF0121DD
:101578000023518053809CBF2370117000232B706F
:1015880005B0BDE8F08F10780E2800F28B8001A618
:1015980056F820F06F150008D91500080116000844
:1015A8001B160008AD160008AD160008AD16000899
:1015B800AD160008AD160008AD160008AD160008F7
:1015C800AD160008AD160008AD1600082D16000867
:1015D800481C508063542178FD299BB206D10C33F6
:1015E8000A21D380918002231370C7E708330621AC
:1015F800D38091800E23F7E7481C50806354D807A6
:1016080042BFD1880D31D180012B8CBF0023032329
:10161800EAE7002B01F101005080635414BF002356
:101628000E23E1E7481C508063545388D1888B42CD
:1016380032D300235380137002232B7069802378E0
:10164800FD2B35D163792B72A3796B72637A227A79
:101658001B0403EB0223E27913446B60637803F104
:101668000C026A80A278D10701D519336B80002655
:101678006968DFF8F0806E814FF4BC720C20B318F3
:1016880001335B0800FB03F758F80770B94218D21A
:101698005A1EB242F3D816E092889A423FF66EAFCD
:1016A80001236CE70023137053809380D38066E78F
:1016B800E3782B7223796B7263796B6063780833F4
:1016C800D4E71E46E5D80C27774358F807309942E7
:1016D80027D123782046FD2B10F801BF0CBF4FF00F
:1016E8000A094FF0060909EB0B03591E89B2474452
:1016F8000193FFF73DFD97F804A0ADF80E005146A1
:101708000DF10E00FFF70EFD019BE218E35C527825
:1017180003EB0223BDF80E209BB29A4203D00523A7
:101728002DE703232BE7BB79DA0706D5FA7993452A
:1017380082BF04EB09018A5CAA729B0709D50C23B6
:1017480003FB068362781B7A9A4282BF4C44E35CAF
:10175800EB720C2303FB068385F80CA05B796B7393
:101768000EE700BF70EC0008F0B50546FD2305F84C
:101778000C3B85B004468DF8043090F8243103F111
:101788000C020244012B42D80026637066808DF853
:1017980005308B7A23718DF808308B7AADF80660A6
:1017A80001338B7263798DF80930A3798DF80A308B
:1017B800A368C3F317031A128DF80B3009211B1401
:1017C8000DF105008DF80D308DF80C20FFF7D0FCD9
:1017D8006778ADF802003A4629460DF10200FFF796
:1017E800ADFC94F82311FFF79DFC94F82421BDF873
:1017F8000230A4F80C31974210D207F10C00D21B2A
:101808003146204405B0BDE8F0400CF047BD12F861
:10181800010D0028B8D1013BDBB2B3E705B0F0BD3C
:10182800012B38B50D4614460FD1012A02D00024E9
:10183800204638BD1A480BF051F80028F7D012A3FB
:10184800D3E90023C5E90023F2E7022BEFD1012AEF
:1018580010D040F6B9339A42E9D1124B1C78002CCB
:10186800E5D00F480BF03AF80028E0D008A3D3E9F8
:101878000023E7E70A480BF031F80028D7D106A380
:10188800D3E90023DEE700BF9E6AC421818A46EEC1
:10189800E9A2A272EAE738B1401DA12026812A0BED
:1018A80070030020B013002007B503688DF80710F7
:1018B8001B6901220DF10701984703B05DF804FB8D
:1018C80013B5044608460191FEF7ACFC236801995C
:1018D8001B6982B2204602B0BDE8104018470000DC
:1018E800B0F1904F08B5014607D10120FFF7E6FB9C
:1018F800114B99420BD1202014E0104B98420BD089
:1019080003F58063984209D10420FFF7D7FB0C4BFD
:10191800994210D1402005E00220E7E7094B9842A0
:1019280004D10820BDE80840FFF7C8BB064B984221
:10193800DED11020F6E708BD001400480004004876
:1019480000180048000C00480010004808B5224B59
:10195800984201460BD14FF40060FFF7CBFB1F4BB9
:1019680099420DD1BDE808402020FFF7B5BBB0F182
:10197800804F0ED01A4B98420FD10220FFF7ACFBD4
:10198800184B99420FD14FF40050BDE80840FFF7BB
:10199800B1BB0120FFF7A0FBE1E7134B984208D148
:1019A8000420FFF799FB114B99420CD14FF480307A
:1019B800EBE70F4B9842D2D11020FFF78DFB0D4B70
:1019C800994206D008BD0C4B9942F8D14FF400302B
:1019D800DBE74FF48020D8E7002C014000140040DA
:1019E800000400400034014000080040004001406D
:1019F8000010004000480140004401402DE9F04338
:101A080087B00E46054614460021142201A89DF809
:101A180038809DF83C901F460CF040FC00960B2C3B
:101A280007D8DFE804F007070A121414141616166C
:101A38001A1CFEE70323019301E002230493032FFA
:101A480011D8DFE807F0111321110123F6E701236C
:101A5800F1E7012301930393F1E70223EBE7022364
:101A680001930123F7E7FEE702230293B8F1100F71
:101A78000CD8DFE808F02D2D0C11131517191B1DB4
:101A88001F21232527292B000123EEE7FEE7012349
:101A98000593022301931EE00223F9E70323F7E7E6
:101AA8000423F5E70523F3E70623F1E70723EFE728
:101AB8000823EDE70923EBE70A23E9E70B23E7E728
:101AC8000C23E5E70D23E3E70E23E1E70F23DFE728
:101AD800B8F1000FDDD1B9F1000F02D02846FFF7A9
:101AE800FFFE053C042C05D8DFE804F0030B0403D3
:101AF8000B00AE626946284609F0A8FF07B0BDE8AA
:101B0800F083AE61F6E713B54FF0010C0024CDE980
:101B1800004CFFF773FF02B010BD000070B586B02F
:101B28000023164604460D46ADF80630FFF70EFFB3
:101B3800042E04D8DFE806F0303404384100FEE70C
:101B48001F4B204A1B68B3FBF2F39BB20022013BF8
:101B580001A92046ADF80430CDE90225049205928A
:101B68000AF076F9236823F080032360A36823F43E
:101B7800A03323F00703A360636823F0007323F006
:101B880070036360636823F470036360A36823F0E1
:101B98008003A36006B070BD094B0B4A1B68D2E7EF
:101BA800074B0A4A1B68CEE7054B074A1B68B3FB7D
:101BB800F2F303EB83035B00C7E70123C6E700BF2B
:101BC8002C00002080A8120140420F008096980047
:101BD80010B50446FFF7A2FF236843F00103236012
:101BE80010BD00224FF0FF31FFF7F2BF034A034652
:101BF80003CA186059601068986070479075FF1F95
:101C08001A4B10B51A4C5B68236008F0FBFC4FF0C8
:101C1800904009F0BBFE174809F0B8FE164809F0D5
:101C2800B5FE16480AF004FB15480AF001FB0AF055
:101C380007F84FF0E022002313615361936172B6F5
:101C48004FF0FF319A0002F1604202F56142013320
:101C5800082BC2F88010C2F88011F3D162B6034B8A
:101C68001B6883F3088823689847FEE70000FF1F76
:101C78002403002000040048000800480038014000
:101C8800004400400749084A881AEFF30883521AAB
:101C98001A44013A013B984288BF0022AA210CF05D
:101CA800FDBA00BF008000200004000010B5114CF0
:101CB8000323204606224021FFF725FF03230222A3
:101CC8004FF400414FF09040FFF71DFF03231A46E1
:101CD80020462021FFF717FF2046032305228021F5
:101CE800FFF711FF20460323BDE81040052201211C
:101CF800FFF709BF00040048024B1869C0F3401001
:101D0800704700BF0004004808B5FFF7F5FF00B9A9
:101D180008BD00BFF9E70000024B01229A62802249
:101D28009A61704700040048024B80229A6201229F
:101D38009A61704700040048104A53694FF4704193
:101D480023F4704391FAA1F153610D4B5A6822F4C0
:101D580000425A601A6822F400421A60DA6822F4D3
:101D68000042DA609A6842F400429A60054BD02239
:101D780083F828234FF480725A60704700000140AE
:101D88000004014000E100E0044B4FF400425A61B6
:101D98001A6842F400421A60704700BF000401400C
:101DA8000348002303224FF48071FFF7ACBE00BF45
:101DB80000040048024B1869C0F30020704700BFB8
:101DC8000004004808B50522002302214FF0904086
:101DD800FFF799FE0023052201214FF09040FFF7FD
:101DE80092FE4FF0904302229A6201229A6208BD45
:101DF8004FF090414B691A04DB4302F4003203F0C0
:101E0800020313438B6170474FF090414B691A04EA
:101E1800DB4302F4803203F0010313438B61704704
:101E280008B5052200234FF480714FF09040FFF76A
:101E38006AFE4FF090434FF480729A6208BD4FF0EB
:101E480090431A284FF48072CCBF9A619A62704707
:101E58000E48C3691A0617D503681B0614D50C4B20
:101E68000C4A1988138889B29BB299420AD0138800
:101E78000133DBB213801388074A9BB2D35CDBB211
:101E880083627047FFF744B9704700BF00440040C1
:101E9800883E0020863E0020863D00200E490F4ADD
:101EA8000B8812880133DBB292B29A4212D00C4AE4
:101EB800D0540B804FF0402202F5806353E8003F76
:101EC80043F0800302F5806040E800310029F3D137
:101ED8000120704700207047883E0020863E002081
:101EE800863D002038B504464518AC4200D138BDBF
:101EF80014F8010BFFF7D2FFF7E708461146FFF782
:101F0800F1BF000070B588B00C46064615460021A2
:101F1800202268460CF0C2F9231E18BF01231B03B8
:101F2800CDE9023569460C230348019604940593CC
:101F38000AF0C0F908B070BD0044004010B5064C66
:101F4800236823F001032360FFF7DCFF236843F0D5
:101F58000103236010BD00BF0044004013B53E4C90
:101F6800236823F0010323604FF40030FFF7B4F82F
:101F780008210123CDE90013384803230A22FFF77B
:101F88003DFD002211463648FFF7BCFF636823F485
:101F980090436360A36823F02A03A360236823F0B7
:101FA800005323604FF0402202F5816353E8003F5D
:101FB80023F0604302F5816040E800310029F3D145
:101FC8004FF0402202F5816353E8003F23F060633D
:101FD80002F5816040E800310029F3D1214BC0228D
:101FE80083F8262340225A601B48FFF791F84FF0E8
:101FF800402101F5806353E8003F23F0400301F5D9
:10200800806040E80032002AF3D1134B4021196266
:1020180015490A8015490A805A6822F400625A60F4
:102028009A6822F008029A605A6822F480425A603C
:102038009A6822F022029A609A6842F480529A6062
:102048001A6842F001021A60DA699102FCD5DA696D
:102058005202F9D502B010BD004400400004004807
:10206800A086010000E100E0863E0020883E0020B6
:10207800064B1A6822F001021A605A6822F40032EC
:102088005A601A6842F001021A6070470044004022
:1020980008B541B14FF4005204484FF48061FFF78E
:1020A8004DFFFFF7E5FF012008BD00BFA086010036
:1020B80008B531B1002211460348FFF73FFFFFF78B
:1020C800D7FF012008BD00BF9A5B0600064B1A68BF
:1020D80022F001021A605A6842F400325A601A6803
:1020E80042F001021A6070470044004008B541B14F
:1020F8004FF4005204484FF48061FFF71FFFFFF7C9
:10210800E5FF012008BD00BFA08601001D280EDCE8
:102118001A280FDC172810DC132811DC1128B5BF8A
:10212800002001201023112308701370704713201A
:102138001E23F9E70C201B23F6E708201823F3E7F2
:1021480004201423F0E7084611461A46FFF7DEBFBD
:102158000C4BD3F8FC2022F08072C3F8FC20D3F893
:10216800FC2042F08072C3F8FC20A3F55D431A6896
:1021780022F001021A601A6842F001021A60002275
:102188005A60704700ED00E0064A074B51681B682B
:1021980010B5064CB3FBF4F3584353685B1A8342FB
:1021A800FBD310BD001000E02C00002040420F00BF
:1021B8007FB50123CDE90413002201A902A8CDE9C6
:1021C800022308F0E3FD00280CBF0420052007B017
:1021D8005DF804FB014608B5002008F041FD002821
:1021E8000CBF0420052008BD08B5FFF7E1FF031F59
:1021F8005842584108BD08B5FFF7ECFF031F584285
:10220800584108BD2DE9F3472A4B2B4D01281446A8
:102218002A482B4A0E4617BFAA463D213C211D4697
:10222800019106BF9A468046904608F0D3FC019972
:102238002846FFF7D9FF30B9002408F0DDFC204616
:1022480002B0BDE8F087002E08BF4FF4FC640734E5
:1022580024F0070405F11007B1463444AAEB050A37
:10226800A1450BD14FF011324FF0FF332846FFF74D
:10227800C2FF003818BF01208400DEE76EB90AEB00
:102288000703D3E90023B3F1FF3F08BFB2F1FF3FD3
:1022980006D1083709F10809E2E7D9E90023F2E78E
:1022A800B84505D93846FFF7A6FF0028F1D1C3E79E
:1022B8000324C2E700E0010800E80108FFEF010875
:1022C800FFE7010810B508F085FC09483C21FFF735
:1022D8008BFF58B107483D21FFF786FF003818BF2C
:1022E8000120840008F088FC204610BD0446F9E768
:1022F80000E0010800E8010830B5084D002340F26D
:10230800EF749AB2914201D8042030BDA34203D0A1
:102318005A5DC2540133F4E70320F6E710E00108E0
:1023280013B50A46044672B6019101460020FFF72C
:1023380069FF62B60428019A05D172B601202146C8
:10234800FFF760FF62B602B010BD000038B5124B4F
:102358001C68D3F80058B4F1113F09D1B5F1113F09
:1023680017D0002211460120BDE83840FFF74ABFC8
:10237800B5F1113F03D1002211461046F4E7FFF7EB
:10238800A1FF042804D12C4001340CBF02200120F5
:1023980038BD0420FCE700BF00E00108034B1873B8
:1023A8009A68D207FCD5187B704700BF00300140FF
:1023B80038B5441E8D18A94200D138BD14F8010F54
:1023C800FFF7ECFF01F8010BF5E7084611461A463E
:1023D800FFF7EEBF38B5064D04460144A14200D1CF
:1023E80038BD2878FFF7DAFF04F8010BF6E700BFDD
:1023F8002400002008461146FFF7ECBF10B5014441
:1024080004468C4200D110BD14F8010BFFF7C6FF3B
:10241800F7E708461146FFF7F1BF000030B58DB069
:102428002822002102A80BF039FF4FF48050FEF754
:1024380061FE1021032306224FF09040FFF763FB53
:102448004FF0904006240125102383610A22CDE92C
:10245800004503232021FFF7D1FACDE900450323E6
:102468000A2280214FF09040FFF7C8FA03231A464A
:10247800CDE9004540214FF09040FFF7BFFA182200
:10248800154C08924FF48272002303924FF40072A5
:10249800CDE90533CDE909330293079207234FF4B9
:1024A800E06202A920460B93049209F097FC636846
:1024B80023F010036360636823F0080363602368F4
:1024C80043F040032360A3689B07FCD5237B034BA1
:1024D800FF221A700DB030BD0030014024000020EA
:1024E8001C4B10B4DC69A00611D51A6891060ED5EC
:1024F80019481A495A6A038809880133C3F30A0339
:1025080089B299421FBF1649D2B2CA5403801148F2
:102518001F232206036215D503681B0612D5114B2B
:10252800114A1988138889B29BB299420DD0138831
:102538000133C3F30903138013880C4A9BB2D35C9D
:10254800DBB283625DF8044B70475DF8044BFEF71D
:10255800DFBD00BF003801408C4600208A460020BD
:102568008A3E0020904A00208E4A00208E46002095
:102578000E490F4A0B8812880133C3F3090392B23C
:102588009A4211D00B4AD0540B4A0B8002F50063D3
:1025980053E8003F43F0800302F5006040E8003153
:1025A8000029F3D10120704700207047904A00208D
:1025B8008E4A00208E4600200030014038B504467F
:1025C8004518AC4200D138BD14F8010BFFF7D0FF15
:1025D800F7E70000054B064A1B8812889B1A98B239
:1025E8001B0444BF00F5006080B270478C46002091
:1025F8008A4600200848094A0188138889B29BB294
:102608009942F9D013880133C3F30A03138013885E
:10261800034A9BB2D05C70478C4600208A46002053
:102628008A3E002070B588B00C4606461546002143
:10263800202268460BF032FE231E18BF01231B031D
:10264800CDE9023569460C230348019604940593A5
:1026580009F030FE08B070BD0038014010B5064CD6
:10266800236823F001032360FFF7DCFF236843F0AE
:102678000103236010BD00BF00380140044B1B78E4
:1026880008461BB100221146FFF7E8BF704700BF9C
:102698000000002073B54C4C236823F0010323602D
:1026A8004FF4804008250126FEF724FD4FF4007101
:1026B80003230A224FF09040CDE90056FFF79EF918
:1026C80003231A464FF480614FF09040CDE900563D
:1026D800FFF794F9002211464FF46140FFF7A2FF7B
:1026E80063683A4A23F490436360A36823F02A039B
:1026F800A360236823F00053236002F6080353E81D
:10270800003F23F0604302F6080040E8003100294A
:10271800F3D102F6080353E8003F23F0606302F6A2
:10272800080040E800310029F3D1294BB02283F892
:10273800252320225A602448FEF7EAFC234A02F5A2
:10274800006353E8003F23F0400302F5006040E8CF
:1027580000310029F3D11C4B402018621D4B198011
:102768001D4B198002F5006353E8003F23F0200356
:1027780002F5006040E800310029F3D1174B1980B9
:10278800174B1980104B5A6822F400625A609A68F5
:1027980022F008029A605A6822F480425A609A68C5
:1027A80022F022029A609A6842F480529A601A686B
:1027B80042F001021A60DA699102FCD5DA69520224
:1027C800F9D502B070BD00BF0038014000300140AB
:1027D80000E100E08E4A0020904A00208A4600204E
:1027E8008C460020024B01221A70FFF753BF00BF2E
:1027F80000000020024B1A68024B1A60704700BFA5
:10280800944A0020A8130020054A064B196813684B
:1028180099421DBF0133012013600020704700BF9B
:10282800A8130020944A0020034A04491368096841
:102838000B441360704700BF944A0020300000200A
:102848000148FFF7CEB900BF00040040014B586AA9
:1028580080B27047000400400B4B10B50B4C586A0F
:10286800238880B283420A4B07D9D3E9002112F5A5
:10287800803241F10001C3E90021D3E90021208021
:10288800801841F1000110BD000400403803002009
:102898003003002008B5FFF7D3FFBDE80840FFF775
:1028A800A9BF70B504460D46164608F093F9083DD1
:1028B80004EBC606B44204D1042408F09DF920466E
:1028C80070BD55F8082FD4E900016B68994208BF1C
:1028D800904201D10834EDE72046FFF78CFC002830
:1028E800F8D10446E9E700001FB503788BB10A4B1D
:1028F8001B68B3F5FA6F0CD3002300220370002382
:10290800CDE90023CDE90223406802226946FFF79A
:10291800C8FF05B05DF804FB944A002000000000E1
:102928000123F0B50380444B444AD3E900510446DF
:102938004348914208BF854285B04FF0000202D15A
:10294800227005B0F0BD3AA1D1E900013D4F6260A7
:10295800C3E900013C484FF0AA33D0E90021B1F1A6
:10296800FF3F08BFB2F1FF3FD0E9026505D09942A9
:1029780008BF9A4201D00A4309D1B5F1FF3F08BF09
:10298800B6F1FF3F0DD09D4208BF9E4209D01030DE
:10299800B842E2D172B63E212B48FFF725FC62B659
:1029A80029486060D0E90032CDE90032B2F1FF3F3A
:1029B80008BFB3F1FF3FD0E9025109D1B1F1FF3FA0
:1029C80008BFB5F1FF3F22D14FF0AA331A4623E0E2
:1029D8004FF0AA36B24208BFB3420BD1B1F1FF3F64
:1029E80008BFB5F1FF3F0FD0B14208BFB5420ED1C5
:1029F8000023EBE753EA020709D1B14208BFB54209
:102A080005D14FF4807121801D46114604E0002352
:102A180023701A461D461946CDE90032CDE9025108
:102A280002226946FFF73DFF8BE700BFAFF3008046
:102A380012345678FEDCBA9008000020FEDCBA900A
:102A48001234567800F8010800F001080A490B888A
:102A580003B9FEE772B64FF0804309885A6A1144F9
:102A680064325963DA636FF002021A616FF0080288
:102A78001A6162B6704700BF7400002000B50322D7
:102A880089B04FF0FF314FF08040FFF7A1F82022C6
:102A9800002168460BF002FC64236A4601214FF0CE
:102AA8008040039309F030FAC8236A464FF48071D6
:102AB8004FF08040039309F027FA054BA02283F8D2
:102AC8001C234FF080521A6009B05DF804FB00BF68
:102AD80000E100E04FF08043DA6842F00202DA6079
:102AE800DA6842F00802DA607047000010B501EBBE
:102AF8008101084B01EB810189001980064B0446CE
:102B080000221A70FFF7BAFF2046BDE81040FFF711
:102B1800E1BF00BF74000020A51300204FF08043E0
:102B28001A6991070AD56FF002021A615A6B64326A
:102B3800DA63084A596B12880A445A634FF0804393
:102B48001A69120705D56FF008021A61024B0122B3
:102B58001A70704774000020A513002038B51A4C6D
:102B680090220021201D0BF099FB012323800F23C5
:102B780016496380A38005222C23A01DFDF77EFE45
:102B8800134A12494FF48033C4E90D2300252C233E
:102B9800052204F13E00A587FDF770FE0D4BE366A4
:102BA8000D4984F87250032304F17C00A4F87030B6
:102BB800C4E91D550BF0CCFB7F2384F89130052325
:102BC80084F8923038BD00BF9002002030EB000836
:102BD8000200010002000700E6E5000870B5094E92
:102BE80005460C46415C30460BF06FFB034628B1A6
:102BF800831B0133DBB2282B28BF0023F35C2B5542
:102C080070BD00BF44EB000870B50D461146044680
:102C180016460BF09DFB2DB3013D082D08D8DFE8C3
:102C280005F00511131517191B1D1F0035236371B6
:102C3800627973799A4215D120460521BDE8704022
:102C4800FFF7CCBF6123F2E76623F0E76B23EEE7DB
:102C58007023ECE77523EAE77A23E8E73123E6E710
:102C68003223E4E770BD000073B5054605F111068F
:102C7800214C224A014636016846FFF7C5FFB01CC1
:102C88006946204426440BF063FB04EB051202233B
:102C980073720023A2F81A31142202FB05400421A2
:102CA800012280F850104FF4807540F20111A0F80D
:102CB8004A20C264A0F8522080F85520A0F8565047
:102CC800A0F8581040F2032084F83430E284A5625A
:102CD800A08584F82E2084F8303084F83330C4F886
:102CE8003A30C4F83E30C4F84230A4F84610A4F88C
:102CF800481002B070BD00BFD400002098E500085D
:102D0800F7B50546AE4CAF4A05F111060146370145
:102D18006846FFF779FFB81C274469462044FDF749
:102D2800C1FC7B7AA84A052B88BF002304EB061058
:102D380088BF7B721188437A41FA03F313F00103C9
:102D48000DD1437259B111F0010308D141FA03F7CB
:102D5800FF07D8B240F1CF8104EB0613587204EB99
:102D680005112B0191F81A01052802D9002081F8D4
:102D78001A01E718508897F81A1140FA01F111F072
:102D880001010FD187F81A1160B110F0010109D1C2
:102D980040FA01FC1CF0010FCFB200F0B181E1183C
:102DA80081F81A71E11891F81B01032802D9002053
:102DB80081F81B0104EB0616717A012903D904294D
:102DC80001D000219180E618908896F81B1140FAEE
:102DD80001F111F001010ED186F81B1158B110F064
:102DE800010108D140FA01F7FF07CEB240F18D8109
:102DF800234483F81B61142303FB054191F84A001F
:102E0800042802D9012081F84A0003FB054393F8FE
:102E18004B10042902D9002183F84B10142303FB1B
:102E28000543918E93F84B0041FA00F0C00712D485
:102E3800012083F84B0071B18807C1F340030AD41D
:102E480041FA03F6F707D8B240F16481142303FB73
:102E5800054383F84B00142303FB054393F84C10F8
:102E6800032902D9012183F84C10142000FB0540E6
:102E7800D18E90F84C3041FA03F313F0010310D1CE
:102E880080F84C3069B111F001030AD141FA03F618
:102E9800F607D8B240F14381142303FB054383F8B6
:102EA8004C00142303FB054393F84E10012902D963
:102EB800002183F84E10142000FB0540118F90F874
:102EC8004E3041FA03F313F0010310D180F84E306D
:102ED80069B111F001030AD141FA03F6F707D8B234
:102EE80040F12281142303FB054383F84E00142389
:102EF80003FB054393F84F10022902D9002183F8F8
:102F08004F10142000FB0540518F90F84F3041FAC4
:102F180003F313F0010310D180F84F3069B111F0B9
:102F280001030AD141FA03F6F607D8B240F101814C
:102F3800142303FB054383F84F00142303FB0541C7
:102F480091F84D00022802D9002081F84D0003FBBA
:102F5800054393F85010052902D9042183F850102D
:102F6800142303FB054191F85200012802D90120DE
:102F780081F8520003FB054393F85510012902D943
:102F8800012183F85510142303FB054393F85310CC
:102F9800022902D9002183F85310142000FB0540B0
:102FA800918F90F8533041FA03F313F0010318D1CD
:102FB80080F85330A9B111F0010312D106E000BF27
:102FC800D400002098E500089002002041FA03F69A
:102FD800F707D8B240F1B280142303FB054383F806
:102FE8005300142303FB054191F856000C2802D91D
:102FF800002081F8560003FB054393F84C10012983
:1030080006D193F84F10022904BF002183F84F100E
:10301800142303FB0543012140F2011083F85710E4
:10302800A3F8580094F82630042B01D984F8261008
:1030380094F82730042B02D9002384F82730B2F8FB
:103048006C0094F8273040FA03F313F0010F814B1A
:103058000ED1012184F8271050B18607C0F3400132
:1030680006D440FA01F7FF07CEB26CD583F8276083
:1030780094F82810022902D9002184F8281094F81D
:103088002910022902D9012184F82910B2F86E10FA
:1030980094F8292041FA02F212F001020CD184F8C6
:1030A800292049B111F0010206D141FA02F6F607CA
:1030B800D0B24CD583F8290094F82A200C2A02D9DA
:1030C800002284F82A2093F832200C2A02D9002200
:1030D80083F8322093F82B20042A02D9002283F89F
:1030E8002B2000225C49104611F9014F14F1780F8A
:1030F80031DA087031E00133102B7FF427AE2EE669
:10310800013110297FF444AE4CE6013110297FF4D7
:1031180069AE70E60133102B7FF492AE9BE6013363
:10312800102B7FF4B3AEBCE60133102B7FF4D4AE82
:10313800DDE60133102B7FF4F5AEFEE60133102BEC
:103148007FF444AF4DE7013110298AD190E701326D
:10315800102AAAD1B0E7782CCBDC0132D2B20C2AE3
:10316800C2D13E490022012011F8014F0132022C40
:10317800D2B288BF0870042AF6D193F83420012A05
:1031880002D9002283F83420354AB2F8701093F837
:10319800342041FA02F212F001020CD183F83420F3
:1031A80049B111F0010206D141FA02F4E407D0B2A4
:1031B80011D583F8340093F82C20052A02D903226C
:1031C80083F82C2093F82D20032A08D80AD100224E
:1031D80083F8342006E00132102AE5D1EBE7022219
:1031E80083F82D2093F82E20022A02D9012283F891
:1031F8002E2093F83020022A02D9002283F83020AA
:1032080093F833200C2A02D9002283F833201421A2
:1032180001FB0531FF2203EB05154FF6FF7081F81E
:10322800512081F8542083F82F2083F831204FF063
:10323800FF32C5F81C21A5F820011A629A84A1F86A
:103248005A20A1F85C2083F83500DA861A8703B083
:10325800F0BD00BFD40000200D010020190100209E
:103268009002002030B5052804D8DFE800F01E04DD
:1032780023191E23FEE7024620251F240F21104B89
:1032880098700338012894BF002001201A7119771B
:103298001A74A3F84850A3F84A409873987630BD3A
:1032A80009256F2400220721E9E71425322400228A
:1032B8000A21E4E73525132402221921DFE700BF9C
:1032C800780000202DE9F04300F111067C4F7D4C79
:1032D800360106F10209B94485B005464846FDF7AE
:1032E800FDF93E4480460390042103A8FDF740FF02
:1032F800737AE0832E0107EB0515C4F80880C4F83B
:10330800148095F81A0163704FF0010884F8518011
:10331800A4F85280A4F85480FFF7A4FF97F8262059
:10332800694B13F92230237323766378052B09D868
:10333800DFE803F0030656585A5C0023637301E084
:1033480084F80D80614B617B1B88617603F0010274
:10335800980748BF42F00202A2855D0748BFA28DC8
:1033680084F8281044BF42F00402A285180742BF1F
:10337800A28D42F01002A285DA0642BFA28D42F069
:103388002002A2859B0642BFA38D43F00803A385B4
:10339800002384F82A3021B94846FDF7BFF984F89C
:1033A8002A003E4496F81B2184F829206AB1E18B53
:1033B80002EB021303EB03230B44E383A3684FF0F0
:1033C800113101FB0233A360636194F82850E38B49
:1033D8006362052D0CD8DFE805F00C5153154749F9
:1033E8000223ABE70423A9E70523A7E70323A5E7FF
:1033F800FEE7A378032B03D8DFE803F00346440372
:10340800FEE7182507EE905A314E84F82050F8EE62
:10341800E77A16E90F00B7EE087A67EE877A86E84A
:103428000F00FCEEE77A40F2E243CDED017A6D0839
:10343800A4F84C309DF80430B4F84820A4F84E3075
:10344800052D4FF47A73B3FBF2F3A4F8403097F8E4
:103458002C3038BF052584F85050052B24D8DFE8D8
:1034680003F0152C202326290225CBE7A378022B6D
:1034780008D0052B06D0012B06D0FEE71925C1E799
:103488000625BFE70C25BDE71225BBE74FF4165309
:1034980063640023A4F8563084F8583005B0BDE8BA
:1034A800F0834FF41643F3E74FF46143F0E74FF42A
:1034B800E133EDE74FF46133EAE74FF49643E7E78A
:1034C800D40000207800002030EB00089002002093
:1034D800A800002002484FF4DE72FF210AF0DEBE89
:1034E800D400002002484FF4DE71FEF719BF00BF78
:1034F800D400002002484FF4DE71FEF7FDBE00BF85
:10350800D400002008B5FFF7F5FF034B1878BDE895
:103518000840FFF7F5BB00BF7800002038B5FFF77B
:10352800D9FFFEF713FF04280CD0FFF7D3FFFEF7EF
:103538000DFF042803D1FFF7DDFF042806D0FFF7AD
:10354800C9FF03E0FFF7D6FF0428EED12649274834
:10355800264C10220AF0C6FE38B125491022204612
:103568000AF0C0FE08B1FFF7B5FFA38AB3F5215FE3
:1035780028D008D30025E8B20135FFF775FB0A2DDE
:10358800F9D10023E3774FF42153A382012522695F
:103598001549164842F642039A424FF010021CBFE2
:1035A800236101250AF09EFE70B10F490F481022D1
:1035B800FDF789F90F4910480822FDF784F9FFF74C
:1035C80091FF03E00025E2E7002DF8D10023E3771F
:1035D8000A4C2370FFF7C2FA2078FFF791FB207896
:1035E800BDE83840FFF76EBE9FE50008D400002014
:1035F800B0E50008C1E50008860200207800002038
:103608000229F7B5054600D9FEE70B4E06EB011374
:103618001C460F016278F15DC3609B780AF036FCA6
:10362800E3790193A379009322796379E1782846B5
:103638000AF055FC03B0F0BD7001010838B5836885
:1036480004466BB1024652F8143BDD6900F11503DC
:10365800A847217D20462022BDE838400AF09BBCBF
:1036680038BD00007FB58D7A8160044675B30121AD
:103678000AF0E2FB012120460AF006FD012120465E
:103688000AF01CFDA368204693F90810FFF7D6FF3F
:10369800A36820461978FFF7B3FF00221146204699
:1036A8000AF0E7FB0023009344F2030220464FF69A
:1036B800FF710AF030FC20464FF6FF710AF052FC09
:1036C800204604B0BDE870400AF0EABC03210AF0C5
:1036D800B3FB204601210AF0D7FC204601210AF05D
:1036E800EDFCA368204693F90810FFF7A7FFA3682D
:1036F8005E680D4B23612A462046102386210AF076
:1037080001FD46F6E823CDE902535B23CDE90053DA
:1037180020461023042270210AF003FD2A46314670
:1037280020460AF028FDB8E75C01010810B50446F8
:103738000AF0B6FC20464FF6FF71BDE810400AF0CB
:1037480011BC000038B58168036891F90810DD697B
:10375800044600F1150300F11402A847A3689A7AF9
:1037680042B11A78022A00D9FEE7044B03EB021390
:10377800E36038BD024B2361FBE700BF700101081D
:103788005C010108836810B5044683B1C3681BB99E
:1037980003690BB9FFF7D6FFA3689B7A1BB1E368EF
:1037A800B3F90C0010BD2369B3F91000FAE7184605
:1037B800F8E7836810B5044643B1C3681BB90369C9
:1037C8000BB9FFF7BFFF94F9150010BD1846FCE7C9
:1037D80090F8D8305BB190F8D930074A180102EB5D
:1037E80003139B681978135853F821007047837D99
:1037F8000E3350F823007047D0EA000813B5194B70
:103808000288DB8B9A42044627D1837813F0D00FC5
:1038180025D18379812B22D84FF6FF730D220146DB
:103828000DF10600ADF80630FDF788FCB4F80D2060
:10383800BDF806309A420ED14C2204F10D01FDF775
:103848007DFCB4F85900BDF80630C01A18BF012035
:10385800800002B010BD0320FBE70120F9E7022039
:10386800F7E700BF780000200A7ACB7902F0070258
:1038780043EA022303804B7A0A7A03F03F035B0191
:1038880043EAD20343808B7A4A7A9B0043EA921335
:10389800CA7A02F0010243EA822383800B7BCA7A48
:1038A80003F00F03DB0143EA5203C3800B7BC3F32E
:1038B8000112012A11D813F0300F14BF012300237D
:1038C8009B0203830B7B7F2B0AD813F0C00F14BF16
:1038D800012300239B024383704740F2FF73F0E704
:1038E80040F2FF73F7E70A7ACB7902F0070243EA5E
:1038F800022303804B7A0A7A03F03F035B0143EA11
:10390800D20343808B7A4A7A9B0043EA9213CA7A9D
:1039180002F0010243EA822383800B7BCA7A03F018
:103928000F03DB0143EA5203C3800A7CCB7B02F01E
:10393800070243EA022303814B7C0A7C03F03F031E
:103948005B0143EAD20343818B7C4A7C9B0043EAB8
:103958009213CA7C02F0010243EA822383810B7D21
:10396800CA7C03F00F03DB0143EA5203C3814B7D9A
:10397800DB0003828B7DDB004382CB7DDB0083820F
:103988000B7EDB00C3820B7BC3F30112012A2BD809
:1039980013F0300F14BF012300239B0203830B7B1A
:1039A8007F2B24D813F0C00F14BF012300239B02E0
:1039B80043830B7DC3F30112012A1BD813F0300F88
:1039C80014BF012300239B0283830B7D7F2B14D814
:1039D80013F0C00F14BF012300239B02C3834FF4CD
:1039E800806303844384704740F2FF73D6E740F254
:1039F800FF73DDE740F2FF73E6E740F2FF73EDE7A0
:103A080037B5214BDB8B03804A78837862F3C30395
:103A180083704A79C37862F30003C3708A79437963
:103A280062F386134371044691F902000D46FCF7D0
:103A38000FFDE37860F34703E370EA78237962F3D4
:103A4800060323712A79DBB202F0010203F07F0337
:103A580043EAC21323712A796379C2F3450223F03A
:103A68003F031343637159224FF6FF7321460DF14B
:103A78000600ADF80630FDF761FBBDF80630A4F886
:103A8800593003B030BD00BF780000202DE9F34164
:103A98009DF820601546522E88464FF05B024FF085
:103AA800000104461F4628BF52260AF0F7FB2D4B9B
:103AB800DB8B23802A78A37862F30203A3706A78E9
:103AC800D20002F00802DBB242EA081103F0070351
:103AD8001943A1706A79E37862F30003E370AA7965
:103AE800637962F38613637195F90200FCF7B0FC01
:103AF800E37860F34703E370EA78237962F3060317
:103B080023712A79DBB202F0010203F07F0343EA52
:103B1800C21323712A796379C2F3450223F03F0364
:103B280013436371A379224666F3470302F8063FFD
:103B38003E443B46B34210D14FF6FF73592221460B
:103B48000DF10600ADF80630FDF7F8FABDF80630BD
:103B5800A4F8593002B0BDE8F08113F8011B02F84F
:103B6800011FE7E77800002007B5009313460A46CF
:103B78000121FFF78BFF03B05DF804FB30B5374B2D
:103B8800027893F8261061F30302027093F8271065
:103B980061F30712027093F82810427861F3030268
:103BA800427093F8291061F30712427093F82A10B3
:103BB800827861F30302827093F83210827961F39C
:103BC8000302827193F82B10827861F307128270D6
:103BD80093F83410C27961F30302C27193F82C1080
:103BE800C27861F30302C27093F82D1061F30712D3
:103BF800C27093F82E10027961F3030202714279C0
:103C080093F8301061F30302427193F8331082790C
:103C180061F30712827103F1390100F10A0200F120
:103C2800160411F9015F02F8015FA242F9D193F875
:103C38004610C27D61F30102C27593F8471061F323
:103C48008302C27593F8481061F30512C27593F8A0
:103C5800493063F38712C27530BD00BFD40000201D
:103C68000278314BC2F3030230B583F8262002787C
:103C7800C2F3031283F827204278C2F3030283F8C1
:103C880028204278C2F3031283F829208278C2F3ED
:103C9800030283F82A208279C2F3030283F83220D0
:103CA8008278C2F3031283F82B20C279C2F303028D
:103CB80083F83420C278C2F3030283F82C20C27838
:103CC800C2F3031283F82D200279C2F3030283F8AA
:103CD8002E204279C2F3030283F830208279C2F39E
:103CE800031283F8332003F1390100F10A0200F1CD
:103CF800160412F9015F01F8015FA242F9D1C27DF1
:103D0800C2F3010283F84620C27DC2F3810283F820
:103D18004720C27DC2F3011283F84820C27DC2F356
:103D2800811283F8492030BDD400002070B5522696
:103D380098B0324604460D4603A800210AF0AEFAB0
:103D4800212342F642008DF80C30FCF7ABFDADF8AC
:103D58000E004FF42150FCF7A5FD1C49ADF81000EA
:103D680014220DF11200FCF7AEFD1948FFF721FDF2
:103D7800184B8DF8260093F851308DF827300AA893
:103D8800FFF7FCFE3223ADF84630134A134BCDE95A
:103D980012236FF08023149347F6FF73ADF8543065
:103DA8000F4BB3F86C208DF85620B3F86E20B3F89B
:103DB80070308DF857208DF85830009603AB2A469E
:103DC80002212046FFF762FE18B070BDC7E5000863
:103DD800403C0020780000206400FA00F401E80369
:103DE8009002002038B5104D044600F11B01062250
:103DF80005F58970FCF7C2FD94F82130C3F303037D
:103E080085F8193194F82130C3F3031385F81A3172
:103E180094F82230C3F3030385F81B3104F125001D
:103E2800BDE83840FFF71CBFD40000200A4A1268DA
:103E380082600A4A00238380837183810384136824
:103E480003615368064A4361136883615368C36119
:103E58004EF6602303607047944A0020D5E50008B9
:103E6800DEE5000810B5114C0220FFF7FBF92046EB
:103E7800FFF75CFC11212046FFF7E0FBA36803B9BC
:103E8800FEE70021204609F0C0FF4FF47A70FEF7E4
:103E98007BF92046012109F0CFFFA3682046197855
:103EA800FFF7AEFB2046FFF741FC10BD403C002069
:103EB80008B590F8203002468BB9FDF77BFF10B9A2
:103EC80082F8210008BD92F8213001335BB2312B12
:103ED80082F82130F6DD012382F82030F2E7FDF781
:103EE80069FF18B1322382F82130EBE792F82130CC
:103EF800013B5BB2002B82F82130D8BF82F820004A
:103F0800E0E700000A4B90F820201B6872B1826835
:103F18009B1AB3F57A6F01D901234371037923B949
:103F2800437913B101230371037370478360F5E785
:103F3800944A0020037B9A1E012A4FF0000202D8FF
:103F480090F8201011B90273184670471346FBE722
:103F58000A4A38B5138801339BB2502B04460D46E4
:103F680001D8138038BD002305491380FDF7A8FC4C
:103F780029462046FDF7A4FCF4E700BF9021002065
:103F8800E7E500082DE9F84F154604460F4677493E
:103F9800FDF796FC29462046FDF792FC744B00225B
:103FA800012F1A804FF0904610D10223B362B761F7
:103FB80046F2A810FEF7E8F8B76246F2A810FEF736
:103FC800E3F829462046FFF7C3FFF0E7BB1E0122AE
:103FD8000C2B00F2BE80DFE803F0374A5E1F07BCF7
:103FE800BCBC7171717171004FF090464FF00108BF
:103FF8000227C6F8188046F2A810B762FEF7C4F880
:10400800C6F8288046F2A810B761FEF7BDF8294621
:104018002046FFF79DFFEBE74FF090464FF0010871
:104028000227C6F8188046F2A810B761FEF7ACF868
:10403800C6F8288046F2A810B762FEF7A5F8294608
:104048002046FFF785FFEBE7B26202274FF0904664
:10405800B76146F2A810FEF797F8B76246F2A810C3
:10406800FEF792F829462046FFF772FFF0E7022391
:10407800B36101274FF09046B76146F2A810FEF7EA
:1040880083F8B76246F2A810FEF77EF82946204664
:10409800FFF75EFFF0E7B26102274FF09046B76185
:1040A80046F2A810FEF770F8B76246F2A810FEF7BD
:1040B8006BF829462046FFF74BFFF0E7A7F1090AFE
:1040C8005FFA8AFA00264FF0010956453EBF4FF0C5
:1040D800904302229A614FF004084FF0904B46F249
:1040E800A810CBF81890FEF74FF846F2A810CBF8B6
:1040F8002890FEF749F808F1FF3829462046FFF7CF
:1041080027FF18F0FF08EAD10223CBF828304FF038
:1041180004084FF0904B46F2A810CBF81890FEF721
:1041280033F846F2A810CBF82890FEF72DF808F1DE
:10413800FF3829462046FFF70BFF18F0FF08EAD1A1
:104148000136A7F10803F6B2DBB2B34238BF002646
:10415800BBE70223B261B3614CF25030FEF714F8AA
:1041680029462046FFF7F4FEF6E700BFE7E500081A
:104178009021002010B50446084694F901308B427E
:1041880001D1237823B901232370FDF758FE60700D
:1041980010BD00001FB50C4670B9084801930DF119
:1041A8000E020DF10F0109F053FF019B9DF80E104F
:1041B8000248224609F003FE04B010BD403C00202E
:1041C80038B515461C46B8B9FDF7A6FD2B460A4674
:1041D80001460B4809F0CCFD09484FF6FF7109F07C
:1041E800C1FE2201064892B2012109F0E4FEBDE8B1
:1041F80038407D20FDF7C8BF0148FFF797FA38BD62
:10420800403C00202DE9F041184C05465B270E463E
:104218003A46002120460AF041F8AB692360EB6971
:104228006360134B13491B789A1E53425341627AB9
:1042380063F3000262724222A27228220023E27211
:1042480004F10E00142223736373FCF73CFB59211D
:104258002046FCF78DFF084BA4F859003A46214642
:1042680030461B7FBDE8F041FFF7AABFCB3A0020DC
:104278009F130020C7E500087800002037B50C46DA
:1042880038B91548836833B9812281F8A02081F8AC
:10429800A23003B030BD9D7A95B101F1A2020DF1B3
:1042A800060109F0B2FEBDF90630002B0FDB4FF610
:1042B800FF73ADF80630BDF8063084F8A030E8E7A3
:1042C8000DF1060109F08DFF84F8A250EBE77F336A
:1042D800F1DA4FF68173ECE7403C00200A4608B556
:1042E80001460148FFF74EFE1C0000200023FF2274
:1042F800037043708370C27003717047C17829B925
:104308008378017101338370012070470378012B92
:104318001DD0022B05D08BB98278013282700371CF
:10432800F2E7827843785340DB0703D40132827086
:104338000023F4E7FF2903D100230371002070470D
:1043480003790133DBB299420371EFD3F6E7FF2912
:10435800F2D002790132D2B291420271EED2827861
:104368000132827000220271CEE7000008B543785E
:1043780002789A4213D0042B8ABF04230370037077
:10438800027888BF4370064B064813F92210064B83
:1043980019731976836813B11972FFF74FF908BDBD
:1043A80030EB0008403C00207800002010B50AB926
:1043B800437010BD541E0B2CFBD80332D2B231F817
:1043C800122040F27E618A4207D95AB222EAE2728A
:1043D8009A42C8BF5AB24270EBE7B2F5C17F02D227
:1043E8009A1E52B2F2E740F2D4418A4204D95AB234
:1043F800032A06DCDA1EF4E7B2F54B7F03D35A1E14
:10440800EFE70122E4E70022E2E7000030B51C4CA8
:1044180085B00E2200210546684609F03FFFB4F832
:10442800A030ADF800302046FBF7C3FF8DF802003E
:104438002046FBF7B5FFB4F8A4308DF80300114807
:10444800ADF80430FFF7B5F994F8A6308DF80730C9
:1044580094F8A9308DF80830B4F8AA30ADF80A30CD
:10446800094B8DF806009B788DF80C3069460123BE
:1044780028468DF80D3005F0E2FB05B030BD00BFD1
:10448800843B0020403C0020780000200148FEF7D3
:10449800DDBA00BF813B0020F8B5154D0E46074632
:1044A8005B232946304614462A46FFF773FED7E9B0
:1044B800041328686A689A4208BF884209D0002411
:1044C80030460C49FFF7DAFE002C0CBF0120032010
:1044D800F8BD59212846FCF74BFEB5F85930834200
:1044E800EDD114B1FFF7D2FFEAE70124E8E700BFF6
:1044F800753C0020843B002013B501210446084484
:10450800FCF736FEA178ADF806000DF10600FCF7C1
:1045180009FEE178FCF706FE2179FCF703FE6179D4
:10452800FCF700FEA179FCF7FDFD04F10801032268
:10453800FCF704FE627804F10C01FCF7FFFD94F827
:104548002311FCF7EFFDBDF80630A4F80C3102B0DA
:1045580010BD00000038024B18BF012018707047CA
:10456800280300202DE9F041002A4AD1042B00F24B
:10457800A1809EB2002B42D04D4C4FF0800EFF25FB
:104588000F8894F81EC0C35D23EA0C03C355A37FAC
:1045980001325B081FFA82FCA3773BB90B88013311
:1045A8000B8084F81EE00B88C554A37FB1F8008007
:1045B80010F8087027EA030300F80830A37F5B08A7
:1045C800A3773BB90B8801330B8084F81EE00B8876
:1045D800C554A37FB1F8008010F8087027EA0303D8
:1045E80000F80830A37F5B08A37733B90B88013341
:1045F8000B8084F81EE00B88C5546645C0D8BDE81A
:10460800F081FF2AFBD1032B00F249819FB2002BD6
:10461800F5D0274C00258026B1F800C094F81EE09C
:1046280010F80C3023EA0E0300F80C30A37F013594
:104638005B081FFA85FCA37733B90B8801330B801D
:10464800A6770B88C254A37FB1F8008010F808E061
:104658002EEA030300F80830A37F5B08A37733B979
:104668000B8801330B80A6770B88C254A37F5B08A5
:10467800A37733B90B8801330B80A6770B88C25414
:10468800A37FB1F8008010F808E02EEA030300F8D1
:104698000830A37F5B08A3772BB90B8801330B8005
:1046A800A6770B88C2546745B6D8BDE8F08100BF2D
:1046B800A02300200D889A4C425DA67F22EA0602BC
:1046C8004255A27F520803F5C063A2773AB90A8817
:1046D80001320A808022A2770A88FF2585540D8836
:1046E800A67F425D22EA06024255A27F5208A277BF
:1046F8003AB90A8801320A808022A2770A88FF25FF
:104708008554A27F5208A2773AB90A8801320A80F2
:104718008022A2770A88FF258554A27F5208A277B3
:104728003AB90A8801320A808022A2770A88FF25CE
:1047380085540D88A67F425D22EA06024255A27F73
:104748005208A2773AB90A8801320A808022A277F1
:104758000A88FF2585541E0605D40D88A67F425D6C
:1047680022EA06024255A27F5208A2773AB90A887D
:1047780001320A808022A2770A88FF2585545D06C7
:1047880005D40D88A67F425D22EA06024255A27F23
:104798005208A2773AB90A8801320A808022A277A1
:1047A8000A88FF2585549A0605D40D88A67F425DA0
:1047B80022EA06024255A27F5208A2773AB90A882D
:1047C80001320A808022A2770A88FF258554DF06F5
:1047D80005D40D88A67F425D22EA06024255A27FD3
:1047E8005208A2773AB90A8801320A808022A27751
:1047F8000A88FF2585541E0705D40D88A67F425DCB
:1048080022EA06024255A27F5208A2773AB90A88DC
:1048180001320A808022A2770A88FF2585545D0725
:1048280005D40D88A67F425D22EA06024255A27F82
:104838005208A2773AB90A8801320A808022A27700
:104848000A88FF2585549A0705D40D88A67F425DFE
:1048580022EA06024255A27F5208A2773AB90A888C
:1048680001320A808022A2770A88FF258554DB0757
:1048780005D40A88A57F835C23EA05038354A37FB4
:104888005B08A377002B7FF4BAAE0B888022013334
:104898000B80A2770B88FF22C254BDE8F0810E88F6
:1048A8001F4C855DA77F25EA07058555A57F6D08FF
:1048B80003F5E063A57735B90D8801350D808025AE
:1048C800A5770D8842550D88A67F425D22EA06022B
:1048D8004255A27F5208A2773AB90A8801320A8063
:1048E8008022A2770A88FF258554A27F5208A277E2
:1048F8003AB90A8801320A808022A2770A88FF25FD
:104908008554A27F5208A277002A7FF418AF0A883C
:1049180001320A808022A2770A88FF2585540EE793
:10492800A02300202DE9F0479C4C802500270F800C
:10493800A577FF2505709846002B00F02C8103F120
:10494800FF3912FA89F9561EBA463B460BE055451F
:1049580040F0C0800137BFB20A88424580F0B3807A
:104968004E4500F0078116F8015F002BEFD16B1E52
:10497800DBB2FD2B00F2AA803F2B40F2E18005F16B
:104988004103DBB23F2B00F2AC80A37F01355B080B
:10499800EDB2A377002B00F0E4805B08A37743B95E
:1049A8000B8801330B808023A3770B88FF22C25426
:1049B800A37FAA0608D4B1F800C010F80C2022EA98
:1049C800030300F80C30A37F5B08A37743B90B8877
:1049D80001330B808023A3770B88FF22C254A37F67
:1049E800EA0608D4B1F800C010F80C2022EA030344
:1049F80000F80C30A37F5B08A37743B90B88013319
:104A08000B808023A3770B88FF22C254A37F2A0739
:104A180008D4B1F800C010F80C2022EA030300F80B
:104A28000C30A37F5B08A37743B90B8801330B8055
:104A38008023A3770B88FF22C254A37F6A0708D478
:104A4800B1F800C010F80C2022EA030300F80C307B
:104A5800A37F5B08A37743B90B8801330B808023BE
:104A6800A3770B88FF22C254A37FAA0708D4B1F802
:104A780000C010F80C2022EA030300F80C30A37FD2
:104A88005B08A37743B90B8801330B808023A37796
:104A98000B88FF22C254A37FEA0705D40D88425D24
:104AA80022EA03034355A37F5B08A377BBB90A88AF
:104AB80001320A808022A2770A88FF2585540A8855
:104AC8004245FFF44DAF0020BDE8F0870127AA4614
:104AD8003B4641E7FBB25246FFF744FD47E7002358
:104AE8003AE70A8894F81EC0835C23EA0C038354CF
:104AF800A37F3F355B08EDB2A37743B90B88013339
:104B08000B808023A3770B88FF22C254A37F5B0806
:104B1800A37743B90B8801330B808023A3770B88D5
:104B2800FF22C254A37F6A063FF537AFB1F800C031
:104B380010F80C2022EA030300F80C30A37F2CE7BE
:104B4800A37F7F355B08EDB2A377002BEED10B88EE
:104B580001330B808023A3770B88FF22C254A37FE5
:104B6800E4E70B8801330B808023A3770B88FF22AF
:104B7800C254E3E75BB9A37F802B1EBF013292B218
:104B88000A80904594BF00200120BDE8F087FBB261
:104B98005246FFF7E7FC0A88EDE700BFA023002094
:104BA8002DE9F04F47F26F730022827003800B7873
:104BB800A3F1FE03B3FA83F35B0983708A780D4689
:104BC80012F001011CBF43F080038370D5F8202147
:104BD80022F07F4222F0FF0285B0044612B143F072
:104BE80008038370AA68C2F31702FF2A1ED9B2F518
:104BF800803F18D363F07F03A37041F002014FF0A8
:104C0800020B09234FF00A0C0822E1700B20CDF8A3
:104C180004C01E4617464FF0070E4FF006094FF026
:104C2800050A042117E043F00203A370180600F1F7
:104C3800D68008234FF0090C07220A204FF0000BFA
:104C4800CDF804C01E4617464FF0060E4FF0050972
:104C58004FF0040A032195F8018004F8018004EB61
:104C68000108297904F80A10697904F80910A97962
:104C780004F80E10A178090709D595F82111A15457
:104C880095F82211A1550346674662460646A9686B
:104C9800A154A278900707D5BA1C1F46AB68C3F386
:104CA8000F23A35596B23346BBF1000F05D05A1C0B
:104CB8001F46AB7AA35596B23346A278D10606D5DD
:104CC8005A1C1F4695F82331A35596B23346454AD8
:104CD800127803F1010914FA89FA05F10C0B42B1B3
:104CE8006B785A460DF10E015046FFF71BFE00285F
:104CF8005AD16A78504659461FFA82FA09F030FBB1
:104D08002278394B6178D243D2B2072F9A5C82EA73
:104D18000102995CA27882EA0102995CE27882EA4F
:104D28000102995C227982EA0102995C627982EA3D
:104D38000102995CA27982EA0102995CE27982EA2D
:104D48000102995C1BD0227A5140082F595C16D079
:104D5800627A5140092F595C11D0A27A51400A2F2A
:104D6800595C0CD0E27A51400B2F595C07D0227B5A
:104D780051400C2F595C1EBF627B5140595CA155B4
:104D88001AFA89F39BB2B5F80C21E2545A1CB5F80B
:104D98000C1192B2090AA154AA78981CD20780B2C1
:104DA8000BD405B0BDE8F08FA378BDF80EA043F092
:104DB8004003A37088F800A0A2E7D5F81071D5F8D1
:104DC8001811D5F81461275022180F3356609160D6
:104DD80095F81C11117398B205B0BDE8F08F4FF02B
:104DE800000B0EE72803002070EB00082DE9F04FB8
:104DF8008F4D0C4683B0014607462846164609F0F3
:104E0800AFFA8C4A002380212380138482F8221071
:104E1800002E00F0C58028784FF0400B4FEAD01CD8
:104E280082F822B09E464FF0FF0892F8229015F8BB
:104E380003A04FEA4C001AEA090F4FEA590C18BFB1
:104E480040F0010082F822C0BCF1000F00F0AB80F6
:104E5800022800F04484032800F0E083012840F091
:104E6800B2809E4240F29C8015F8039019EA0C0F1C
:104E780014BF012000205FEA5C0A40F0B8830133C8
:104E88009BB29E42138482F8221040F2898015F961
:104E980003C0BCF1000F4FEA400001DA40F0010006
:104EA80082F822B04FF0400C9E4279D915F8039051
:104EB800400019EA0C0FC0B218BF40F001005FEAC9
:104EC8005C0A40F02C8401339BB29E42138482F822
:104ED800221065D915F903C015F803904000BCF1FC
:104EE800000FC0B201DA40F00100400019F0400F95
:104EF8005FFA80FA18BF4FF0200C00F0A3854AF043
:104F0800010ABCF1000F40F09F8501339BB29E421D
:104F1800138482F8221043D915F9039015F803C0B9
:104F28004FEA4A00B9F1000FC0B201DA40F00100BF
:104F380040001CF0400FC0B218BF4FF0200C00F02A
:104F4800BC8540F0010082F822C0BCF1000F03D1FB
:104F58000133138482F822107D2821D84130238818
:104F680003F1010CA4F800C0F854138C9E4217D921
:104F780092F8220015F803C010EA0C0F4FEA50000F
:104F880014BF4FF0010C4FF0000C82F8220020B93A
:104F980001339BB2138482F822109E423FF645AF3C
:104FA80003B0BDE8F08F01339BB20228138482F866
:104FB800221000F0B481032800F03C8201284FF051
:104FC800800C3FF44EAF9E42EAD9E85C1CEA000F21
:104FD8001ED05FEA5C092FD101339BB29E42138435
:104FE80082F82210DCD9E8560028C0F2F1804FF090
:104FF80080094FEA590082F8220018B90133138456
:1050080082F822102388581C208007F80380ACE718
:105018004FEA5C0082F8220018B90133138482F841
:1050280022102388581C208007F803E09DE700BF62
:1050380074220020A023002019EA000FD9D05FEACB
:105048009C0C40F0C78001339BB29E42138482F8C7
:105058002210A5D9E8560028C0F26E824FF0800CC5
:105068005FEA5C0040F0478201339BB29E421384A2
:1050780082F8221094D915F803C04FEADC101CF00E
:10508800400F4FEA400000F0BF844FF0200C40F082
:10509800010082F822C0BCF1000F06D101339BB297
:1050A800138482F822104FF0800C9E427FF678AF6E
:1050B80015F8039040001CEA090FC0B218BF40F071
:1050C80001005FEA5C0C40F0718301339BB29E42A1
:1050D800138482F822107FF663AF15F903C04000ED
:1050E800BCF1000FC0B280F231844FF0800C5FEA4F
:1050F8005C0C40F0010040F0658301339BB29E4296
:10510800138482F822107FF64BAF15F903C04000D4
:10511800BCF1000FC0B280F225844FF0800C5FEA2A
:105128005C0C40F0010040F0598301339BB29E4271
:10513800138482F822107FF633AF15F903C04000BC
:10514800BCF1000FC0B280F226844FF0800C5FEAF9
:105158005C0C40F0010040F04D8301339BB29E424D
:10516800138482F822107FF61BAF15F903C04000A4
:10517800BCF1000FC0B2C0F211844FF0400C15F81A
:10518800039040001CEA090FC0B200F052834FEAB6
:105198005C0C40F0010082F822C0BCF1000F40F026
:1051A800048401339BB2138482F822101FFA80FC16
:1051B80000283FF4DBAE00232088013300F1010909
:1051C800A4F8009007F800E098B26045F4D3CCE664
:1051D8004FF0400CE85C1CEA000F3FF441AF5FEA77
:1051E8005C0C40F0AB8101339BB29E42138482F881
:1051F80022107FF6D5AE15F803904FEAD91019F0B2
:10520800400F4FEA400000F0F4834FF0200C40F0CC
:105218000100BCF1000F40F0EE8301339BB29E42C7
:10522800138482F822107FF6BBAE15F903C015F877
:1052380003904000BCF1000FC0B201DA40F0010059
:10524800400019F0400FC0B218BF4FF0200C00F01A
:10525800298440F00100BCF1000F40F0258401339F
:105268009BB29E42138482F822107FF699AE15F9FC
:1052780003C04000BCF1000FC0B201DA40F00100E9
:1052880082F822B04FF0400A9E427FF689AE15F8A8
:1052980003C040001AEA0C0FC0B218BF40F001006A
:1052A8005FEA5A0C40F0D48201339BB29E421384C9
:1052B80082F822107FF674AE15F903C04000BCF1E5
:1052C800000FC0B2C0F274834FF0400C15F8039081
:1052D80040001CEA090FC0B200F0D9824FEA5C0C0A
:1052E80040F0010082F822C0BCF1000F40F0678353
:1052F80001339BB2138482F822101FFA80FC002825
:105308003FF434AE00232088013300F10109A4F8EA
:10531800009007F8008098B28445F4D825E69E42AC
:105328007FF63EAEE85C4FF04009C009B2F820C0F5
:10533800430015F80C0019EA000F4FEA590A01D08A
:1053480043F00103BAF1000F40F0B0820CF1010CF8
:105358001FFA8CFC6645A2F820C082F822107FF65E
:105368001FAE15F90C905800B9F1000FC0B280F2C9
:10537800DB82402340F00100002B40F0A4820CF1B6
:10538800010C1FFA8CFC6645A2F820C082F8221096
:105398007FF606AE15F90C304FEA4009002B5FFA8C
:1053A80089F980F2CA82402049F00109002840F0BA
:1053B80099820CF1010C1FFA8CFC6645A2F820C0FA
:1053C80082F822107FF6ECAD15F90C004FEA49037C
:1053D8000028DBB280F2BD824FF0400943F00103A0
:1053E800B9F1000F40F08D820CF1010C1FFA8CFC12
:1053F8006645A2F820C082F822107FF6D1AD15F9D3
:105408000C005B000028DBB280F2C282402043F02F
:10541800010382F8220028B90CF1010CA2F820C07F
:1054280082F822102088013300F1010CA4F800C092
:105438003B549AE59E427FF6B3AD15F803A04FF0B2
:1054480040094FEADA101AEA090F4FEA40004FEA1A
:10545800590C01D040F00100BCF1000F40F033833B
:1054680001339BB29E42138482F822107FF698ADD6
:1054780015F903C015F803A04000BCF1000FC0B235
:1054880001DA40F0010040001AF0400FC0B218BF26
:105498004FF0200C00F0EE8240F00100BCF1000F4C
:1054A80040F0EA8201339BB29E42138482F82210B4
:1054B8007FF676AD15F9039015F803C04000B9F1F1
:1054C800000FC0B201DA40F0010040001CF0400FAC
:1054D800C0B218BF4FF0200C00F0D78240F0010096
:1054E80082F822C0BCF1000F03D10133138482F883
:1054F8002210413833E515F8039019EA000F14BF5C
:10550800012000205FEA9C0A40F0388201339BB2F8
:105518009E42138482F822107FF642AD15F903C02B
:10552800BCF1000F4FEA400001DA40F0010082F8B8
:1055380022B04FF0400CB8E54FF0400C15F803903E
:1055480019EA0C0F14BF012000205FEA5C0A40F042
:105558000C8201339BB29E42138482F822107FF69C
:105568001FAD15F903C015F80390BCF1000F4FEA01
:10557800400001DA40F00100400019F0400FC0B2CD
:1055880018BF4FF0200A00F0478240F00100BAF13E
:10559800000F40F0438201339BB29E42138482F88D
:1055A80022107FF6FDAC15F9039015F803C04000F2
:1055B800B9F1000FC0B201DA40F0010040001CF060
:1055C800400FC0B218BF4FF0200A00F0638240F0CD
:1055D800010082F822A0BAF1000F7FF455AE013322
:1055E8009BB2138482F822104FF0800A4CE619EA25
:1055F8000A0F4FEA9C0C4FEA400001D040F001002E
:1056080082F822C0BCF1000F7FF44EAC01339BB28C
:10561800138482F822104FF0800C45E415F803A09B
:105628001AEA0C0F14BF012000205FEA99097FF4E1
:105638000AAF01339BB29E42138482F822107FF690
:10564800AFAC15F903C015F803A0BCF1000F4FEA81
:10565800400001DA40F001001AF0400F4FEA400024
:1056680018BF4FF0200900F0B98140F00100B9F1EE
:10567800000F40F0B58101339BB29E42138482F83B
:1056880022107FF68DAC15F903C015F803A0400071
:10569800BCF1000FC0B201DA40F0010040001AF07E
:1056A800400FC0B218BF4FF0200900F0C08140F091
:1056B8000100B9F1000F40F0BC8101339BB29E425A
:1056C800138482F822107FF66BACEB564000002B57
:1056D800C0B201DA40F0010082F822B009E792F87E
:1056E800229019EA0A0F14BF012000205FEA590925
:1056F8007FF41CAE01331FFA83FC6645A2F820C074
:1057080082F822107FF64CAC15F90C90B9F1000F15
:105718004FEA400380F200814FF0400A10E6400053
:10572800C0B2009019EA0A0F4FEA9C00019003D01A
:10573800009840F0010000900198002840F0CC81CA
:1057480001339BB29E42138482F822107FF628AC64
:10575800009815F903C015F803904000BCF1000F3C
:10576800C0B201DA40F00100400019F0400FC0B2A9
:1057780018BF4FF0200A00F0718140F00100BAF123
:10578800000F40F06D8101339BB29E42138482F872
:1057980022107FF605ACEB564000002BC0B201DAB0
:1057A80040F0010082F822B0FFF7D6BB15F803904D
:1057B80040001CEA090FC0B27FF499AC5FEA5C0CA8
:1057C8003FF49BAC15F8039040001CEA090FC0B2E7
:1057D8007FF4A5AC5FEA5C0C3FF4A7AC15F8039026
:1057E80040001CEA090FC0B27FF4B1AC5FEA5C0C60
:1057F8003FF4B3AC15F8039040001CEA090FC0B29F
:1058080001D040F001005FEA5C0C7FF4B8AC0133D2
:105818009BB29E42138482F822107FF6C1AB15F921
:1058280003C04000BCF1000FC0B2C0F2BA804FF014
:10583800800C4FEA5C0C82F822C0BCF1000F3FF4E8
:10584800B0AC1FFA80FC00287FF4B5ACFFF790BB22
:1058580015F8039040001CEA090FC0B201D040F0CF
:1058680001005FEA5C0C7FF431AD01339BB29E42CC
:10587800138482F822107FF693AB15F903C0400019
:10588800BCF1000FC0B2C0F296804FF0800C4FEA16
:105898005C0C82F822C0BCF1000F3FF429AD1FFA5E
:1058A80080FC00287FF42EADFFF762BB15F80C9042
:1058B80058001AEA090FC0B24FEA5A037FF45AADEA
:1058C800002B3FF45CAD15F80CA04FEA400913EA31
:1058D8000A0F5FFA89F94FEA53007FF465AD002893
:1058E8003FF467AD15F80CA04FEA490310EA0A0F18
:1058F800DBB24FEA50097FF471ADB9F1000F3FF404
:1059080073AD15F80CA05B0019EA0A0FDBB24FEA79
:1059180059003FF47EAD7AE515F80C305B064FEA86
:1059280080004FD5202325E59B005FFA83F915F801
:105938000C30580648D5202036E58000C3B215F84B
:105948000C00400642D54FF0200947E54FF0400CC7
:1059580038E715F80C004FEA89034006DBB238D562
:10596800202054E54FF0400C38E719EA0A0F4FEAB7
:105978009C0C4FEA40003FF44CAC48E419EA0A0F8B
:105988004FEADC0C4FEA40003FF483ABFFF77FBBE4
:1059980082F822B046E54FF0400C2BE74FF0800C20
:1059A8002FE740F0010082F822B01FFA80FC02E4E1
:1059B8004FF0800C53E740F0010082F822B01FFA44
:1059C80080FC9FE420237EE720208BE74FF020090E
:1059D80097E74FF0200082F8220023E54FF02009D6
:1059E800400019EA0A0FC0B24FEA590C3FF456AD0D
:1059F80052E54FF0200C400019EA0C0FC0B24FEAF4
:105A08005C0A3FF4C4ADC0E54FF0200C82F822C018
:105A18004FF0200CFFF749BB4FF0200A400019EA6D
:105A28000A0FC0B24FEA5A0C3FF415AC11E44FF01C
:105A38002009400019EA0A0FC0B24FEA590C3FF496
:105A48004FAD4BE54FF0200C4FEA4A001CEA090F16
:105A5800C0B24FEA5C0A3FF492AE8EE64FF0200ADD
:105A6800400019EA0A0FC0B24FEA5A0C3FF46BAA79
:105A7800FFF767BA4FF0200C40001CEA0A0FC0B2CB
:105A88004FEA5C093FF415AE11E64FF0200382F8A7
:105A980022302EE54FF0200C82F822C04FF0200A69
:105AA800FFF7F2BB4FF0200C400019EA0C0FC0B210
:105AB8004FEA5C0A3FF48DAD89E54FF0200382F888
:105AC8002230FFF749BA40001CEA0A0F4FEA990949
:105AD800C0B23FF4CCADC8E5009840005FFA80FA48
:105AE800019819EA000F4FEADC0C3FF40AAAFFF705
:105AF80006BA00BF2DE9F04F5788B7F58F7F8BB0F6
:105B0800144606460BD90022227000226F2B6280B1
:105B180000F06581002333700BB0BDE8F08F127878
:105B28000E2A0D4624D80E2A00F2118101A151F83F
:105B380022F000BF135B0008635D0008575D000892
:105B4800575D0008635D0008635D0008635D000839
:105B5800635D0008635D0008635D0008B15D0008CF
:105B6800575D0008575D0008575D0008D55D0008BF
:105B7800692A40F2EA806A2A40F0E9809C4FFA8A52
:105B880002F1FF3C1FFA8CFC002A00F077820CF12E
:105B9800030CDFF864E2BC44FF22B91C11F8010BC6
:105BA800424061451EF80220F8D1934200F0CF81AF
:105BB80000222270C4F80220E280FA8A022AA9D9B7
:105BC80039796F2900F02B83032AA3D079796F29BB
:105BD80000F03583042A9DD0B9796F2900F032830B
:105BE800052A97D0F9796F2900F03B83062A91D0CE
:105BF800397A6F2900F04482072A8BD0797A6F2985
:105C080000F03283082A85D0B97A6F2900F02F83F3
:105C1800092A3FF47FAFF97A6F2900F02B830A2A0B
:105C28003FF478AF397B6F2900F027830B2A3FF4C4
:105C380071AF797B6F2900F023830C2A3FF46AAF98
:105C4800B97B6F2900F01F830D2A3FF463AFF97BFE
:105C58006F2900F01B830E2A3FF45CAF397C6F2953
:105C680000F01A830F2A3FF455AF797C6F2900F0B2
:105C78001083102A3FF44EAFB97C6F2900F00F83D0
:105C8800112A3FF447AFF97C6F2900F00B83122AE1
:105C98003FF440AF397D6F2908BF4FF012087FF4F9
:105CA80039AF02F101091FFA89F93A44A7F81690A9
:105CB8005FFA89F993704F494A4602A808F050FBE9
:105CC8006F234FF0010CBB704FF0000E6423A7F850
:105CD80000E0A7F816C0237008EB0C0399451FFADB
:105CE80089F27FF617AF901E02A9A0EB08005A1E92
:105CF8000B440A4413FA80F04FF06A084FF0070982
:105D08004FF0660A05E0002B40F0BD8190423FF459
:105D180001AFFB8A12F8011F07EB030B01338BF865
:105D28000210FB822378092BEDD9A3F1640BBBF198
:105D3800050FEBD8653B042B00F2B782DFE813F0C0
:105D48001E01160111010D011A01632A05D800234D
:105D58002370C4F80230E380DDE6254FFA8AB918CB
:105D680001328B70FA822278092A00F2A480002A74
:105D78003FF4D0AE013A082A3FF6CCAE01A151F863
:105D880022F000BF4B6000081D5B00081D5B000887
:105D9800AD5F0008AD5F00083560000801600008CD
:105DA8006F6000081F6000087A1C6280104EEB5577
:105DB800A088727F618883189942FFF6ADAE337868
:105DC8005F0600F1E1810E232370A5E67A1C62804C
:105DD800EB55E2886388934210D201239BE604497D
:105DE8000A800122CA8264228B702270002392E604
:105DF800A0230020A223002070EB0008002363806A
:105E080023700223037042802B78FD2B00F08680DC
:105E1800EB7803722B7943726B7943606A780832A6
:105E2800728000224FF4BC70DFF8B0C47281F62192
:105E38000446013499424FEA54042ED849D38B4280
:105E480040F089802B78FD2B7ED04FF0060B28463A
:105E5800DFF8888410F801AF0BEB0A0909F1FF316C
:105E680089B2FBF785F904EB440708EB8707ADF81F
:105E780008003979019102A8FBF754F905EB0902EA
:105E880015F809305278019903EB0223BDF8082070
:105E98009BB29A421FD005233DE6601E1418824229
:105EA80004F1010780F0698127F0010101EB570136
:105EB8005CF82110BDE7A2F1640105293FF62AAE7E
:105EC800653A042A00F2FA81DFE802F0807C7874EF
:105ED80092002246E2E7BB79DA0706D5FA799245BD
:105EE80082BF521912F80B20B2729B070BD56300C0
:105EF800234408EB83036A781B7A9A4282BF5B19B2
:105F080013F80B30F3726300234408EB83083173F2
:105F180098F8053073730BB0BDE8F08F6B79037296
:105F2800AB7943726B7A297AEA791B0403EB012374
:105F3800134443606A7802F10C014180A978C907CB
:105F48007FF56FAF19326BE74FF00A0B7FE70A2234
:105F580001232270DFE50323DDE5F97684F800905C
:105F6800D4E64FF06803B9762370CFE6797084F8E9
:105F780000C0CBE6397784F80080C7E6397001F0B5
:105F88000103618887F801E0033B01F1010BA4F8E4
:105F980002B06B5497F90030002BACBF63465346F0
:105FA8002370B3E66288511C6180AB5423780133B7
:105FB8002370AFE50722FB76227017E76822BB76CD
:105FC800227013E701227B7022700FE762883B7012
:105FD800002103F00103033B7970511C6180AB542D
:105FE80097F90030002BC0F230810123237091E52E
:105FF8006A223B772270F9E66288511C6180AB54B3
:106008003B787A78134313F0020340F0D580628816
:10601800511C6180AB546288511C6180AB543B7841
:10602800D8064CBF69236A23237073E56288511C24
:106038006180AB543B781D074CBF6723072323704F
:1060480068E562883A83511C6180AB543A787B7763
:1060580012F0010200F0CE8006220833A280E3800D
:106068000423237056E56288511C6180AB547B7809
:1060780013F00203CFD0092323704BE5FF2294E5E8
:106088004FF006080DE6013B082B3FF63FAE0FF236
:10609800080B5BF823F000BFD9600008155D000805
:1060A800155D0008C5600008C56000084D6100085E
:1060B8001B61000867610008FF600008638803F13E
:1060C800010BA4F802B0E9542378013323701DE6CC
:1060D80063883B8303F1010BA4F802B0E9543B78D1
:1060E800797713F001036AD008310623E180A38091
:1060F800042323700AE6638803F1010BA4F802B0B5
:10610800E9543B78DB067FF536AF4FF0690323701F
:10611800FCE5638803F1010BA4F802B0E9543B786D
:1061280079780B4313F0020343D1618801F1010B25
:10613800A4F802B06B54618801F1010BA4F802B015
:106148006B54DEE7638803F1010BA4F802B0E9544D
:106158003B7819077FF502AF67232370D6E563887C
:1061680003F1010BA4F802B0E9547B7813F00203A1
:10617800E1D04FF009032370C8E5584902EB42000B
:10618800144651F820105AE602A92844FEF72EFEBC
:10619800737FBDF808106288CB1A9BB21A446280DC
:1061A800727F1A447277E2881344E380338BE95490
:1061B80009E608232370A9E508232370AAE40C3113
:1061C800E18079784FF00A0B11F00101A4F804B0CE
:1061D80028D0618801F1010BA4F802B005F801C0CC
:1061E800618801F1010BA4F802B06B54E3880D3308
:1061F800E3807DE779780C33E38011F001014FF0FB
:106208000A03A38024D06388012158186080E954C8
:10621800638859186180EA54E3880D331FE74FF00B
:1062280002083EE5638803F1010BA4F802B0E954C3
:10623800638803F1010BA4F802B0E95458E74FF062
:1062480003082EE54FF004082BE56623237061E46C
:1062580063885A1C6280E95463885A1C6280E95436
:10626800FEE64FF005081CE54FF0070819E54FF06A
:10627800080816E54FF0090813E54FF00A0810E57D
:106288004FF00B080DE54FF00C080AE54FF00D082C
:1062980007E54FF00F0804E54FF00E0801E54FF051
:1062A8001008FEE44FF01108FBE477290ED084F8BB
:1062B80000E0C4F802E0A4F806E027E5772B09D04F
:1062C80000232370C4F80230E38023E44FF0650311
:1062D80023701BE5652323701CE400BF70EC0008E5
:1062E8002DE9F8431F46184B164693F8302004460C
:1062F8003AB393F82B301FB11BB31F1F18BF0127E8
:10630800A1F1020804F5E36901F11E0538F8020F4E
:10631800FAF713F929F8020FB8F80000FAF71AF992
:10632800A845A9F82000F1D1084B84F85A771B68D2
:10633800C4F85C3786F00106012384F8606784F8A6
:106348001937BDE8F88300BFD4000020944A002024
:10635800B0F8E834B0F8EA249B1A98B21B0444BF9A
:1063680000F5007080B2003818BF01207047D0F8DF
:10637800F836B0F8E8240133C0F8F836D0F800371A
:106388000133C0F80037B0F8EA349A421FBFC21888
:10639800B0F8EC1492F8EE24013316BF0B4000223B
:1063A800A0F8EA341046704708B50023A0F8EA348C
:1063B800A0F8E8340148FAF7EFFE08BD20000020F5
:1063C80008B50548FFF7F0FF044B05480022C3F85D
:1063D8001C26FAF7E1FE08BDD8230020802C0020F7
:1063E80020000020F0B54E78202E0D468BB00446D4
:1063F80001F10C0132D8324601A807F0B1FF01AB18
:10640800C6F121020021981907F048FF9DF82230B3
:10641800332B64D19DF82330442B60D1BDF8203054
:10642800F62B02D0B3F5FA7F59D1B4F87027A4F847
:1064380070379A421CBF002284F87427012284F81E
:106448006D276A7984F87227AA7984F87327F62B5E
:1064580013D0B3F5FA7F26D0002331E00B4601AA0A
:1064680005F12C0718685968164603C60833BB425D
:106478003246F7D11B783370C8E71A4B1B78002BCC
:10648800EAD09DED037AF0EE087AB4EE677AF1EE81
:1064980010FAE1D1DFED147A9DED047AB4EE677A53
:1064A800F1EE10FAD8D1DFED117A9DED077AB4EE4E
:1064B800677AF1EE10FACFD19DF82430012B02D182
:1064C80084F874370BE0022BC6D194F87427002A9D
:1064D800C2D084F87437064B1B68C4F878370BB001
:1064E800F0BD00BF000000200000884288AC96493B
:1064F800944A00204FF47F4303800023C0E901330E
:10650800C0E90333436103767047000038B50023C0
:10651800C0E90733C0E955334362C0F85C3104462B
:10652800FAF7B6FE254B9878022845D0431F584203
:106538005841FEF70FF840F2FF13A4F8EC34204B53
:106548001B68002503F57A73C4F8F43604F2047066
:10655800C4E9A255C4F89052A4F8EA54A4F8E8543F
:10656800C4F8F05684F8FC5684F81857C4F8F8565E
:10657800C4F80057FAF72EFD84F81957294604F293
:106588001A70402207F08AFE7D2384F85A57C4F80F
:106598005C5784F86057C4F86457C4F86857A4F87F
:1065A8006C37A4F8725784F87457C4F878572046A3
:1065B800BDE83840FFF79EBF0120BAE77800002009
:1065C800944A002030B40E4A92F82E40012C14D17F
:1065D8000C4A0178126881B1016940F6C415511A54
:1065E800A94202D930BCFFF785BF416829B9416982
:1065F800511AFA2984BF4261047630BC704700BF43
:10660800D4000020944A00204378032B06D1C068A8
:10661800B0F5834F34BF0020012070470020704739
:106628004378032B0FD1D0E902232AB1B3F5834F66
:1066380034BF00200120704744F2BF12934294BF38
:10664800002001207047002070470000F0B54E7808
:10665800082E85B005460C4601F10C0717D83246BE
:10666800394601A807F07CFE01ABC6F109020021FA
:10667800981907F013FE9DF80930032B05D16279AC
:106688002A70064A12682A616B7005B0F0BDC868A6
:1066980079683A7A01AB03C31A70ECE7944A002090
:1066A80030B5037895B004461BB34A799A4220D195
:1066B8004D784D2D01F10C011DD82A46684607F08A
:1066C8004FFEC5F14E0200210DEB050007F0E6FD77
:1066D800049B6360190EC3F3072242F2107000FB9B
:1066E8000122C3F30743642101FB0323E360059BF5
:1066F800A36015B030BD4E22684607F031FEE7E7CB
:106708008A68C2F317024C2A16D0942A0AD0AAB96A
:106718000B4A92F82E20012A10D18B79012B0DD12A
:10672800FFF794BF064A92F82E20012A06D18B79EA
:10673800012B03D1FFF7B4BFFFF754BE704700BF6A
:10674800D400002070B54C88B4F5427F4FF00003A8
:106758000AD80D780B2D73D8DFE805F0060D1A2A34
:106768002D30363952555969A2F1240462424B80C2
:1067780062410A7007E04D2A01D0582A06D10270FA
:1067880002230B70002380F8093333E00023F8E775
:1067980002F0FD033C2B01D0212AF7D10378427087
:1067A8004D2B0CBF082303230B7000238370E9E7EC
:1067B80082700422DDE782800522DAE7838803EB12
:1067C800022383800623DCE7C2800722D1E7C3883F
:1067D80003EB02239BB2002BC3800CBF0B230A23BD
:1067E8000B7000234B80012380F80933C388B3F56D
:1067F800407F01D8002002E000200870488070BD6A
:10680800C2800922B5E70A2382800B70EBE7B4F552
:10681800407F3CBF241822724B8801339BB24B80C7
:10682800C2889A429CBF0B230B700123ABE780F808
:1068380008230B704B80022380F809330120DEE720
:106848000B704B80D6E7CB88B3F5407F70B531D855
:10685800242303700B7843704B7883700B784D2B8F
:1068680014D1CB88C3708B88037105230022CD888F
:10687800D4189542A6B210FA84F415D891F80823D2
:106888002270CA880132981880B270BD8B78C370A4
:106898008B8803718B881B0A4371CB888371CB88E3
:1068A8001B0AC3710823E1E78C180132247A845546
:1068B80092B2DCE70020E8E72DE9F74F16464A8850
:1068C800B2F5427F04460D462ED80B780A2B0FD915
:1068D800A3F16402032A03D90020287068802DE000
:1068E800653B8F4F022B33D8DFE803F063A4A70082
:1068F80000210A2BF0D801A050F823F031690008D4
:106908004B690008E1680008E16800088F69000821
:106918009D690008A9690008AF690008E1680008D6
:10692800E16800081D6A0008A6F124077E424FF0BE
:1069380000007E4168802E7084F8090303B0BDE82A
:10694800F08F6F2E0CBF642300232B700020F3E719
:1069580016F0040F14BF4D2358233E7023703A7865
:10696800D1070ED412F0020F14BF21233E23637007
:10697800C2F3C003D20648BF43F00203A370042346
:10698800E3E73C23F3E7A68005232B7084F809137B
:106998000020D3E7A38803EB0623A3800623D4E7CC
:1069A800E6800723F1E7E38803EB0623E38065230A
:1069B800CBE70DF106007E70FAF716FC3978FAF786
:1069C8000BFCA7882179FAF707FC390AFAF704FCC7
:1069D800E788A179FAF700FC390AFAF7FDFB9DF878
:1069E8000630B34206D000232B706B80032384F853
:1069F8000933CDE7002F0CBF66230A232B70012330
:106A080084F8093300236B80E288B2F5407FBFD950
:106A18002B70BDE7B2F5407F3CBF121916726B8828
:106A280001339BB26B80E2889A4201D866232B70AF
:106A38000123DCE77E806723F9E7B7F8028097F83F
:106A4800009008EB06284FF6FF730DF106001FFAB9
:106A580088F84946ADF80630A7F80280FAF762FBD5
:106A68002679B4F804A03146FAF75CFB4FEA1A21FC
:106A7800FAF758FB94F806B0B4F806A05946FAF7A6
:106A880051FB4FEA1A21FAF74DFB797804F1080710
:106A9800FAF748FB52463946FAF750FBBDF806307C
:106AA80043453AD119F0040015D086EA0B01E21DDE
:106AB800002398B2824584F8081307D802230120DE
:106AC80000222A706A8084F8093337E712F8010F28
:106AD80001334140EDE7A178F9F792FD217984F877
:106AE8000803F9F78DFDA18884F80803090AF9F766
:106AF80087FDA17984F80803F9F782FDE18884F815
:106B08000803090AF9F77CFDE28884F80803394686
:106B1800F9F77CFD84F80803D0E703230020CFE7CA
:106B2800503A0020CB88B3F5407F2DE9F041044668
:106B38000D464AD84B783C2B40D0A3F12100434264
:106B480043415B002A784D2AAA7808BF43F0040322
:106B5800D10748BF43F0080392074FF02402227080
:106B680048BF43F010036F226270A370AB88E370D4
:106B7800AB881B0A2371EB886371EB88A71C1B0A7F
:106B8800A3713846FAF774FC0822E071E988A2F18B
:106B980008039BB2561C8B42B6B204EB02080FD313
:106BA800063189B23846FAF7E3FA88F80000000A95
:106BB800A055E8880A3080B2BDE8F0810123C1E71A
:106BC8002B441B7AA3543246E0E70020F4E730B4A4
:106BD800BDF80C40B4F5407F03D8039430BCFAF7F5
:106BE8005FBC002030BC704710B5044624202070DC
:106BF80058206070237100201B0AA170E270637135
:106C0800A071E0710522E11CF9F700FD207209204E
:106C180010BD00002DE9F04F0025DFF8E4A00D803D
:106C2800D71891468FB080460C462B462A464FF01F
:106C3800FF0BB94502D10FB0BDE8F08F19F8010B71
:106C48003B28114609D001323831D2B26944202A92
:106C580001F8300C08BF0022EBE738326A444FF0E5
:106C6800000102F8301C0026F2B25AF836100193DF
:106C780002A80092F9F7CCFADDE90023A0B9FF2BAE
:106C88001FBF2388591C218008F803B023880AEB0A
:106C9800C606591C218008F803203379142B01D823
:106CA800189AD554FF231BE00136372EDCD1FE2B72
:106CB80006D023885A1C22806FF0010208F80320AE
:106CC800002602A8F9F7AEFA721CF6B2B042238881
:106CD8000AD85A1C22804FF03B0208F80320FE23F2
:106CE8000135EDB20022A4E7591C218006F13801D4
:106CF8000DEB010616F8301C08F803101646E0E7FD
:106D0800A401010840F2FF3270B40023A0F8202645
:106D18007D2280F8542A0360C0F80E33A0F81E368E
:106D2800A0F81C36A0F8423AA0F8443A80F8463A4F
:106D3800C0F8483AC0F84C3AC0F8503AC0F8583A47
:106D480000F66724024600F66D250A2614F8011F8E
:106D580009B1B6FBF1F1AC4282F8701A82F8713AC7
:106D6800C2F8743A02F10802F0D170BC1522FF2172
:106D780000F52A6007F092BAF8B5134A044692F86B
:106D88003000F8B192F82B2003B1DAB18E1E04F569
:106D9800226701F11E0536F8020FF9F7CEFBAE4265
:106DA80027F8020FF7D1012384F8423A94F8453ABC
:106DB80083F0010384F8433A94F8463A83F00103D8
:106DC80084F8443AF8BD00BFD4000020B0F81C365F
:106DD800B0F81E269B1A98B21B0444BF00F58060C9
:106DE80080B2003818BF01207047000030B50A246F
:106DF80085B00125032322464FF400614FF09040EF
:106E0800CDE90045FAF7FAFD4FF4805103232246F5
:106E18004FF09040CDE90045FAF7F0FD3B4AD2F833
:106E2800883023F0407343F00073C2F888304FF085
:106E38000070FAF751F94FF4805004F0D1FB34494F
:106E480002AA06F01FFD002805DA32493248FAF78F
:106E580037FD05B030BD31492F48FAF731FD04F050
:106E68009BFB06F0A1FE01462B48FAF729FD2C49A9
:106E78002948FAF725FD4FF4805004F0B1FB06F0DD
:106E880093FE01462448FAF71BFD26492248FAF7E3
:106E980017FDBDF8080006F073FE01461E48FAF714
:106EA8000FFD21491C48FAF70BFD9DF80A0006F072
:106EB8005DFE01461848FAF703FD1C491648FAF723
:106EC800FFFC9DF80B0006F051FE01461248FAF748
:106ED800F7FC17491048FAF7F3FC9DF80C0006F088
:106EE80045FE01460C48FAF7EBFC022202A90020F5
:106EF80006F002FA041EACDA0E490748FAF7E0FC7D
:106F0800204606F047FE0146A0E700BF00100240F9
:106F180040420F00E9E500081C0000201DE60008BB
:106F280028E6000837E6000846E600084FE60008AD
:106F380058E6000861E6000810B50446FAF756FE60
:106F4800014B1B68E36010BD00ED00E0054B0649EE
:106F58001A68064801FB020020F000401860000C87
:106F6800704700BF10000020FD430300C39E2600A9
:106F78001FB5684606F0B4FB041E0CDA0B490C4832
:106F8800FAF79EFC204606F005FE01460848FAF787
:106F980097FC04B010BDFCD0FBF75EFC02460B4624
:106FA8000448694605F03EFFF3E700BF83E60008A2
:106FB8001C0000207003002008B5074805F052FDAA
:106FC80048B1064B196806F023FA20B1BDE808401D
:106FD800014805F04BBD08BD70030020944A00200D
:106FE80008B506F0C1FB02490248FAF769FC08BD7A
:106FF8008EE600081C0000202DE9F047054686B003
:10700800284805F06BFC01248DF8084098BB264BF6
:107018004FF48072CDE9002324492548DFF898A071
:10702800234FDFF89890FAF74BFC6E460025B046E0
:1070380051463846FAF744FC306806F0C7FD014669
:107048003846FAF73DFC49463846FAF739FC706885
:1070580006F0BCFD01350146EDB23846FAF730FCC2
:10706800AC4206F10C06E3D12146404606F08AFB05
:1070780006B0BDE8F0870B4805F030FC030203F4C6
:10708800FE4343F4C03343F080032A780093064B51
:107098000193002AC0D0074A0224CDE903238DF8C2
:1070A8000840B9E77003002080FFFF009BE6000856
:1070B8001C00002000B90B00A3E60008ADE600089C
:1070C80037B500250170C0E905552E4945800446AD
:1070D80005710572C5600574057780F82050456212
:1070E80080F82850C5858585A0F83458A0F832580E
:1070F80080F8505AC0F8385AC0F83C5AC0F8405A7C
:10710800C0F8445AC0F8485AC0F84C5A1E48FAF712
:10711800D7FBFFF76BFE1D4B00931D491D4B1E4807
:1071280001954FF4805205F0ABFB23781BB11A4848
:10713800442105F0CCFB184805F0D0FBB0FA80F0EC
:10714800400920772046FFF757FF002803DA134944
:107158000D48FAF7B5FB06F08FFA002803DA104954
:107168000948FAF7ADFB06F045F9002803DA0D499E
:107178000548FAF7A5FB0C490348FAF7A1FB03B049
:1071880030BD00BFB7E600081C0000202918000821
:107198009C030020AD9A000870030020C3E6000895
:1071A800E0E60008FEE6000817E700080000000017
:1071B80070B5044686B060480E46154605F08EFB4D
:1071C800002874D05D49E3680A68D31A122B6ED977
:1071D8005B4BE26093F82B3025B1002B67D01D1F65
:1071E80018BF0125574B1B786D00A4F8585A022B7D
:1071F8004FF00005A4F85A5A2AD15348FFF710FA5D
:10720800002800F08A80514A13780133DBB2022B40
:1072180094BF137015701378012B4AD14C4D284632
:10722800F9F7C7F895F8A43084F85A0A012BB4F88E
:10723800583A04BF60F07F0084F85A0A43F0040308
:10724800A4F8583AB4F8583A43F00103A4F8583A65
:107258001023B21E84F85C3A04F65C211E3640F214
:10726800592032F8023FA3F58063434348BF03F235
:10727800FF3302319B1203F2DC5396420B80F0D1AC
:1072880004F53E6504F658202946F9F7E5FC08237D
:1072980080B21C44029340F27443CDE9035000933A
:1072A8002548019422A3D3E9002305F05CFB06B02E
:1072B80070BD022B25D127480D68FCF77AFA264ABB
:1072C800136840F6C411EB1A8B42244B03D893F988
:1072D800001081420AD018701560F9F7A7F9B4F8C0
:1072E800583A84F85A0A43F01003A9E71848F9F7FE
:1072F80057F8B4F8583A803884F85A0A43F00C031F
:107308009EE71348F9F743F8F9F75AF9B4F8583AE9
:1073180084F85A0A43F0080392E70D48F9F737F85A
:10732800F9F7ACF884F85A0A8CE700BFAFF300808D
:10733800CFB4AA96E555157770030020944A00202B
:10734800D40000209F130020D8230020190000201B
:10735800843B0020403C002040030020180000200F
:1073680070B500239CB2A24205D8D0F83C3A134429
:10737800C0F83C3A70BDB0F83258B0F836686C1CAA
:107388003440B0F83468A6421EBF2D18CE5C85F88C
:10739800386803F1010318BFA0F83248E2E700009B
:1073A80010B4074C2478084624B15DF8044B114604
:1073B800FBF704B903485DF8044BFFF7D1BF00BFE2
:1073C80000000020B013002010B500F27C7400F516
:1073D800B0712046F9F70DFF214602460148FFF734
:1073E800DFFF10BD200000207FB50B46374991F81C
:1073F8002D1000F128060229044600F11C0231462E
:1074080068461BD1FEF776FB9DF80030022B5BD156
:1074180004F5B075324669462846F9F747FFD4F8AF
:10742800683123F07F436E2B43D1294B9A78052A84
:107438003DD8DFE802F0303438063038FAF788F8FB
:10744800E2E75A6CB2F5613F94BF00220122204660
:10745800FFF7DAF8C8B9C2B194F86E31012B14D825
:1074680094F87231042B10D11A49102204F27B10BF
:1074780006F038FF48B9782384F8883184F88231D7
:1074880084F87C312846FDF737F8204604B0BDE87B
:107498007040FFF799BF5A6CB2F5E13FD4E75A6CD8
:1074A800B2F5614FD0E75A6CB2F5164FCCE701221E
:1074B800CDE74C2BE9D1084B1B78002BE5D0B4F86D
:1074C8008831B3F5FA4FE0D104B070BDD400002084
:1074D8007800002023E70008B0130020F8B5234FF8
:1074E80004463846F8F753FFF8F7C8FF064697F9F9
:1074F800A600F8F7C3FF05463846F8F751FF94F899
:10750800FC3684F87231FF2384F87431332384F80D
:107518006531442384F86631D4F8683184F87061A1
:107528006D2262F31703C4F86831C0F10A00002322
:10753800C4F86C3184F8813200B24FF43943A4F8AE
:10754800823280F30700092384F8730184F87151AB
:1075580004F5B07084F8843204F5AA71FAF704F9D6
:107568002046BDE8F840FFF72FBF00BF843B00204E
:107578002DE9F04F044685B0B4F82E270092B4F8F0
:1075880030270192B4F83227B0F828670292B4F88D
:1075980038270378B0F822E7B0F824C7B0F81CA75A
:1075A800B0F81E97B0F82087B0F82677B0F82A57B9
:1075B8000392B0F82C07B4F81A27A4F87A610026C9
:1075C800B4F83617B4F834B7A4F86C21A4F874E109
:1075D800A4F876C184F87C31A4F86EA1A4F870915F
:1075E800A4F87281A4F8787184F87D61A4F87E51BA
:1075F800039AA4F88C21FF2284F865214422A4F878
:10760800800184F866210098D4F86821A4F88201E2
:10761800A4F88A11019884F8813246214FF4F8437E
:1076280061F31702A4F88401A4F882320298A4F83E
:107638008601262304F5B070A4F888B184F88E6119
:1076480084F88F6184F8906184F89161C4F86821A6
:1076580084F8843204F5AA71FAF786F8204605B052
:10766800BDE8F04FFFF7B0BEF0B591B0044600F2A8
:107678003A736D4600F25A76186859682A4603C26A
:107688000833B3421546F7D120220DEB0200002142
:1076980006F004FE94F8602794F85A370AB943F0C4
:1076A8000203A4F8703100232678D4F85C2784F804
:1076B8007331102384F87431C4F86C2184F8726132
:1076C8006B4604F2751510AF1A4603CABA42286011
:1076D8006960134605F10805F6D1332384F865314E
:1076E800442384F86631D4F8683184F881624FF411
:1076F800D27262F31703C4F868314FF4A053A4F8A8
:107708008232492304F5B07084F8843204F5AA71F2
:10771800FAF72AF8204611B0BDE8F040FFF754BE4A
:107728002DE9F04F614B1A68D0F864372DED028BC4
:10773800D31A122BA1B0044640F2B280DFF8809130
:107748005B4D99F80010C0F864278A1E51425141D8
:1077580095F9A000F8F7AAFE95F8A43095F8A520A9
:1077680095F9A280012B0CBF03230123012A95F868
:10777800AA200CBF43F0080343F00403012A95F83C
:10778800AB2008BF43F010030746012A49480CBF45
:1077980043F0200643F04006FCF71AF807EE900A7B
:1077A800B8EE670ADFED447A20EE270A06F028FDD6
:1077B800DFED427A3E4820EE278AF8F7FAFD824646
:1077C8003B48F8F704FE99F800108B1E02290CBFFD
:1077D80095F8A9904FF0000959425941834695F907
:1077E800A600F8F763FE802205460021684606F0E9
:1077F80055FD4FF67F73ADF80A30ADF80C307F2396
:107808008DF80E3018EE103ACDF80F30CDF8133051
:1078180000238DF8095084F86D31257884F86F318C
:107828006FF02F02172384F86C2184F870316946B1
:1078380084F86E51802204F27110ADF800608DF862
:1078480004A08DF805B08DF806708DF807808DF8C6
:10785800089006F085FD332384F86531442384F8C5
:107868006631D4F8683184F8815240F2811262F3AB
:107878001703C4F868314FF41343A4F88232852300
:1078880004F5B07084F8843204F5AA71F9F76CFF36
:10789800204621B0BDEC028BBDE8F04FFFF794BD48
:1078A80021B0BDEC028BBDE8F08F00BF944A0020E8
:1078B800843B0020942100200000503900247449A2
:1078C8009F1300202DE9F0434D4B0446A9B04D48C5
:1078D8001D68FBF76EFFD4F8683740F6C312EB1A41
:1078E800934204D894F96C37834200F08580464E61
:1078F800C4F86857B17884F86C07052998BF434BDA
:107908008DF811009CBF33F81190414B8DF80F1082
:1079180098BF33F811504FF006084FF07F0388BF27
:1079280000254FF000078DF810304246B6F84A306F
:10793800ADF804300DF1120088BFA946ADF8063045
:10794800ADF80C708DF80E80F8F7F4FF71784246A8
:1079580006A8F8F7CBFF2B48ADF80A50ADF8089009
:10796800FBF710FF40428DF81E002648FBF70AFF80
:1079780040428DF81F00642239460FA801AE06F078
:107988008DFC0FCE08AD0FC596E807006FF02E03EB
:1079980085E8070084F86C31257884F86D711C231C
:1079A80084F87031802208A984F86E5184F86F71C8
:1079B80004F2711006F0D4FC332384F865314423B3
:1079C80084F86631D4F8683184F8815240F2811223
:1079D80062F31703C4F868314FF41343A4F88232F2
:1079E800852304F5B07084F8843204F5AA71F9F798
:1079F800BBFE2046FFF7E8FC29B0BDE8F08300BFD6
:107A0800944A0020403C002078000020B0EA00089A
:107A1800BCEA000838B50446B0F87007A4F86C0151
:107A2800F62808BF234B94F8721708BF1B7894F800
:107A3800732794F8745784F8741103BF83F0010313
:107A48005B00DBB2002384F86E316FF06E0384F8BC
:107A580070316FF02A0384F87131122384F872317F
:107A6800002384F87331332384F86531442384F880
:107A78006631D4F8683184F881124D2060F3170319
:107A8800C4F868318F2384F883320A2304F5B07070
:107A980084F86F5184F8752184F8822284F884323E
:107AA80004F5AA71F9F760FE2046BDE83840FFF7F3
:107AB8008BBC00BF0000002010B54FF07E52C0F80C
:107AC8006C210022C0F87021C0F87421C0F8782118
:107AD800C0F87C21C0F88021C0F8842180F88C216E
:107AE8000821332280F8881180F865210221442278
:107AF800037880F8891180F866210121D0F868217F
:107B080080F88A3180F88B1180F881324C2149F64F
:107B18000103A0F8823261F3170221230446C0F85A
:107B2800682180F8843200F5AA7100F5B070F9F781
:107B38001BFE2046BDE81040FFF746BC70B5061D89
:107B480004460A4601463046FEF7B6FE08B304F678
:107B5800B52531462846FEF776FE294602460D48E9
:107B6800FFF71EFC63793C2B13D121890A4804F6E0
:107B78005A2304F66622A4EB8404A4F5F7541C3CAB
:107B880033F8025F8D4204BF056844F823509342DE
:107B9800F6D170BD20000020944A002070B511482D
:107BA80090F82D00451E012D0C460AD80E4E8D1852
:107BB800AC4200D170BD14F8011B3046FFF714FC2D
:107BC800F6E7032809D1094E8D18AC42F2D014F813
:107BD800011B3046FFF7B2FFF7E70548FFF7E0FB68
:107BE800E8E700BFD4000020D8230020802C002024
:107BF8002000002010B500F6B5240B4602223C21D7
:107C08002046FEF7F1FF214602460248FFF7C8FB6F
:107C180010BD00BF200000200E4B1A68D0F8483A6B
:107C2800D31A122B13B513D9C0F8482A00F6B52475
:107C3800202300F622200193009003223C21C82330
:107C48002046F9F7C1FB214602460348FFF7A8FB87
:107C580002B010BD944A0020200000207FB5224BBE
:107C68001A68D0F84C3AD31AC72B04463AD91F4D94
:107C7800C0F84C2A4FF480732846ADF80830F8F75E
:107C880086FB06461A48FBF77DFD01463046F8F7A5
:107C98009DFC8DF80A002846F8F779FBF8F790FC68
:107CA80095F8A9308DF80B0028468DF80C30F8F7B8
:107CB80080FB8DF80D002846F8F772FB072304F6C1
:107CC800B524019302AB8DF80E00009303223C21EA
:107CD80041F20D032046F9F777FB21460246054895
:107CE800FFF75EFB04B070BD944A0020843B00207F
:107CF800403C00202000002030B5204B044687B0CF
:107D08001F481D68FBF755FDD4F8503A40F6C312DA
:107D1800EB1A934203D894F9543A83422BD0C4F80F
:107D2800505A002384F8540A8DF80830F8F790FC6C
:107D3800144DADF809006978ADF80B0004220DF177
:107D48000D00F8F7D3FDA97806220DF11100F8F718
:107D5800F1FD0F2304F6B524019302AB009303222F
:107D68003C2141F20E032046F9F72EFB214602463C
:107D78000548FFF715FB07B030BD00BF944A002047
:107D8800403C00207800002020000020D0F8383A3D
:107D9800828D0133C0F8383AC38D9A421FBFC2188A
:107DA800018E92F83220013316BF0B400022C385A2
:107DB80010467047034B1B780BB1FAF71BBC0248FF
:107DC800FFF7E4BF00000020B013002008B5124BF5
:107DD80093F82D305A1E012A04D8BDE808400F48F0
:107DE800FEF7C5BA032B10D10D4AB2F81E36B2F809
:107DF8001C1699420DD0D118013391F82206B2F819
:107E080020160B40A2F81E3608BD0648FFF7D2FF21
:107E1800FAE70020F8E700BFD4000020D8230020AC
:107E2800802C002020000020194B30B51B684FF42F
:107E38007A72B3FBF2F3174AC0F8583A0023A0F855
:107E48005C3A80F85E3A1388A0F8603A00F53E651F
:107E580087B001332946044600F658201380F8F706
:107E6800D5FF1823029380B2043440F25513CDE9AC
:107E780003500093019404A3D3E90023064804F0B7
:107E880072FD07B030BD00BFF1C6A7C1D068080FAA
:107E9800944A0020440300207003002000000000E2
:107EA8002DE9F043344B16461B684FF47A72B3FB46
:107EB800F2F3C0F8583A40F201330025A0F8683AC6
:107EC8000446062380F86A3A87B0A0F85C5A80F81E
:107ED8005E5AA0F8605AC0F86C5AA0F8785A04F6AE
:107EE8008B3800F67A200F46FFF726F823494046DC
:107EF80006F02EFA2249404606F0D8F94FF05F09FD
:107F08004046F8F78FF9EBB298421ED804F53E6563
:107F180084F88A0B294604F65820F8F7D5FE002382
:107F28000393B37E029306F11903019380B20123F0
:107F3800CDE904500093F17E0DA3D3E90023384620
:107F480004F06EFD07B0BDE8F0832344013593F8D3
:107F58008B2B202A08BF83F88B9B93F88B2BA2F1DD
:107F6800410119299CBF203283F88B2BC8E700BF39
:107F78009E6AC421818A46EE944A002034E70008AC
:107F8800C7E50008F0B51D4B8BB01F6815460446C1
:107F98000E46FEF7DBFF4FF4C87307F51677B0FB04
:107FA800F3F202FB130317FA83F36361EB7E1BB949
:107FB8000023A3610BB0F0BD05A92846F8F74EFFD2
:107FC8000028F7D101A8FEF7B7FF9DF8165001A9C0
:107FD8002A460DF1170006F037F90028E8D10F2DD1
:107FE80005D86369A561A3F516736361E2E79DF897
:107FF8001410304604F06BFCDCE700BF944A002004
:1080080070B5214B8CB005461C68FEF79FFF4FF4F6
:10801800C873AE69B0FBF3F204F5167402FB1300E3
:10802800002E14FA80F0C6F1100414BF88238923A7
:10803800E4B2686108A88DF81830FEF77DFF062CB9
:1080480028BF062408AB991922460DF1190006F03D
:1080580087F906AB039318230293013405F1100343
:108068000193E4B201230093049405A3D3E9002308
:10807800064804F078FC0023AB610CB070BD00BF6B
:10808800401DA12026812A0B944A0020700300205D
:10809800F0B590F8283080F8593A314BB0F832589A
:1080A80093F82D30013B012B94BF0123FF2380F867
:1080B800583A4FF48073A0F85A3A2A4B5B6CC0F8D0
:1080C8005C3AB0F83438EB1A9AB21B0444BF02F594
:1080D800007292B2782A134628BF7823044680F8A3
:1080E800603A87B00020C1B2914220DB04F53E65BA
:1080F800294604F65820F8F7E4FE1023029304F109
:108108002003019380B240F6B933CDE903500093C0
:10811800154811A3D3E9002304F025FCD4F8443A08
:1081280094F8602A1344C4F8443A07B0F0BDB4F890
:1081380034389D421FBFE618B4F8367896F8386888
:108148000133214416BF3B400026A4F834380130DF
:1081580081F8616AC7E700BFE9A2A272EAE738B10D
:10816800D400002078000020700300202DE9F041A1
:1081780094B00446FAF770FB804658480F4604F05E
:10818800ADFB60B901232377554B1A6863699A429E
:108198002ED9204614B0BDE8F041FFF731BF237F48
:1081A8003BB100232046237714B0BDE8F041FEF729
:1081B80023BF4B4B1A6894F82830E3B1B4F834382D
:1081C800B4F83268F61AB5B2330444BF05F5007541
:1081D800ADB225B9636AD31AB3F5FA7F03D96262DF
:1081E8002046FFF755FF65885DB940F2E7336380A5
:1081F80014B0BDE8F0816262A4F83438A4F83238CB
:10820800F1E7013DADB26580002DF1D142463B4614
:10821800324804F035FC2046FFF706FE3149324863
:10822800F9F74EFBB4F8380A05F0AAFC01462E48C7
:10823800F9F746FB2D492C48F9F742FBB4F8400AF8
:1082480005F09EFC01462848F9F73AFB28492648DC
:10825800F9F736FBB4F83C0A05F092FC01462248CF
:10826800F9F72EFB23492048F9F72AFBB4F8440A0A
:1082780005F086FC01461C48F9F722FB1E491A48FE
:10828800C4F8385AC4F83C5AC4F8405AC4F8445A96
:10829800F9F716FBB4F8480A05F072FC01461248D3
:1082A800F9F70EFB15491048F9F70AFBB4F84C0A20
:1082B80005F066FC01460C48F9F702FB10490A482C
:1082C800F9F7FEFA01A805F0AFFABDF84C0005F081
:1082D80057FC01460448F9F7F3FA89E770030020D0
:1082E800944A00203AE700081C00002048E70008EC
:1082F8004DE700085BE7000860E7000876E700083C
:108308007BE700082DE9F843354E364F364DDFF848
:108318000081F9F71DFFFAF7BDFAF9F753FDF9F7F0
:108328003FFD01233B70FAF7B5F906F126012F4806
:1083380001F04AFCF9F712FEF9F772FD2C4B002404
:1083480080225A701C70C5E902442C61FAF766F85D
:10835800284B1C70F9F7AAFC274B28484FF4004219
:108368005A614FF04009F9F7E7FCF9F70DFF41F2C0
:108378008830C8F82890F9F707FF4CF25030C8F851
:108388001890F9F701FF2846F9F7BEFC2146284660
:1083980005F03BFD4FF47A70F9F7F6FEFBF7BEF8EF
:1083A8001748FAF7BDFA174B1748B3F84810FAF709
:1083B8009DFB96F8341015484B1E59425941FEF75B
:1083C8007FFE96F83430012B14BF012323463B70FF
:1083D80003D0BDE8F843F9F7A7B8BDE8F88300BFB4
:1083E800D400002000000020403C0020543A002027
:1083F800922100202400002000040140E0930400A2
:108408009C3A002078000020813B0020B013002017
:1084180000040048184B4FF4004273B55A611748DE
:10842800174C4FF6FF7105F0A9FD208023889B07A4
:1084380012D5144E35798DB1104808236A460021AB
:1084480005F0BDFCD6E90402DDE900139A4208BF35
:10845800884201D00023238002B070BD02236A46FF
:108468000648294605F0ABFC074BDA8BBDF800300F
:108478009A4218BF2580EFE700040140403C0020E5
:10848800C82300204803002078000020034A002366
:108498001370034A1370034A13707047D1230020E6
:1084A800743C0020A4130020024A00231370024ADF
:1084B80013707047D1230020743C002008B5437E18
:1084C800203B042B0FD8DFE803F0050E030B0F0049
:1084D800FBF788FC064A01231370064A137002E072
:1084E800054B01221A7008BDFBF70CF8F2E700BF34
:1084F800D1230020743C0020A4130020034B1B78D8
:10850800012B01D1FBF712BC704700BFD12300201B
:1085180070B5CB78284DC3F3000385F8AA304B79A2
:10852800C3F3801385F8AB300646C87840080C467C
:10853800F7F79EFF85F8A60023792048C3F30003C8
:1085480085F8A7302379C3F3450385F8A830637904
:10855800227903F03F035B0043EAD21385F8A93080
:1085680021461EB9BDE87040FBF77EB9FBF7BBF9A1
:10857800A37803F0F003202B04D12046BDE8704017
:10858800FFF79CBFFFF790FF0D4B1B78022B12D112
:10859800A2790C4804F119015208FFF7FFFAA179F2
:1085A80005F178004908F8F753FB05F15000BDE8DC
:1085B8007040F8F747BB70BD843B0020A43A002008
:1085C8009F1300202800002070B5054658B9194BA4
:1085D80019491C78194803794BB1012C28D0BDE8FA
:1085E8007040F8F7D1BE164B16491C78F2E7012CFB
:1085F800154B164E13D98A78C2F3C0025A7002225C
:108608001A70E31E58425841FFF782FF3046F7F7C9
:10861800B8FE032C05D13046F7F7B6FE01E001227B
:108628001A7086F8A4500948BDE87040F7F7A7BE4D
:1086380070BD00BFCE230020D03C0020480300209E
:10864800CF2300202B3D0020583C0020843B0020F5
:10865800244B1A7970B505460E4632B10A46BDE874
:10866800704001461846FBF717BF1F4A1F495B2396
:10867800FBF790FD45BB1D48FBF7C0F8044628B33F
:108688001B491C48F9F71CF905F130011948C9B212
:10869800F9F70AF918491748F9F712F9204605F0C9
:1086A8008DFA01461348F9F70BF912480A21F9F730
:1086B800FBF8012C06D0042C11D001240F492846C0
:1086C800FBF7DCFD204670BD0748D5E72EB10C4806
:1086D800FAF7BCF90CB10224F0E70324EEE7002E08
:1086E800F9D0F4E7480300202B3D0020D03C0020BF
:1086F80091E700081C00002059E70008843B00208F
:10870800813B0020024B1878831E5842584170471D
:108718009F13002070B500239CB2A24200D870BD00
:10872800058886886C1C34404688A6421EBF2D18D2
:10873800CE5CAE7103F1010318BF0480ECE7038837
:1087480042889B1A98B21B0444BF00F5006080B2AF
:10875800704708B52C30FFF7F2FF003818BF01202A
:1087680008BD000008B5094B1B785BB1084B188899
:10877800084B1B8880B29BB2C01A18BF012000F0BA
:10878800010008BD0448FFF7E4FFF8E700000020F7
:108798008C4600208A460020B013002008B50B4BF9
:1087A80093F82D305A1E012A04D8BDE8084008481D
:1087B800FDF7CEBD032B04D1BDE808400548FEF700
:1087C80005BB0548FFF7CEFF08BD00BFD400002059
:1087D800D8230020802C0020200000202DE9F04321
:1087E800074699B03D48FBF789FD0646002860D04A
:1087F8003B4B1C78002C5CD13A4B1B78022B54D194
:10880800DFF8F8900DF10C0825464846ECB2FFF762
:10881800C5FF40B14846FFF7D9FA0135522D08F88F
:10882800010BF2D12C4630482146F8F711FA2F48AF
:10883800F8F708FADFF8A4802D4D98F802308DF883
:1088480000304FF0010995F8A4308DF8053028461E
:1088580085F8A5708DF806708DF80190F7F797FDEB
:108868008DF802002846F7F7A4FD8DF80300284686
:10887800F7F7ADFD1F4F8DF804000EB3184B1B78AA
:10888800CBB91D48234603AA6946FBF76DF918487A
:1088980001233B70F7F7A9FD1548F7F7AFFD012352
:1088A80088F8033019B0BDE8F0831448FDF788FD57
:1088B800C0E70024BEE710486946FFF71FFEE6E759
:1088C8003B7803B9FEE70C486946FBF799F8284658
:1088D80087F80090F7F78EFD2846DEE7583C002021
:1088E800743C00209F130020E83B0020C03B002080
:1088F800843B002029030020263B0020280000207C
:108908000A4B1A7910B504462AB10146BDE8104051
:108918001846FBF777BCFFF761FF054B05491B7F3E
:1089280020465B22BDE81040FBF74ABC4803002004
:1089380078000020263B0020B0F8EA34B0F8E8249C
:10894800F0B5D21A93B2120444BF03F500739BB278
:10895800DD2B85B0044608D8294D00F5257600F5AD
:1089680022772846FFF7FEFE08B905B0F0BD284675
:10897800FFF720FAD4F8F02601320346C4F8F026AF
:1089880031463A466846F8F7E3FD9DF80030022B79
:10899800E7D104F57075324669462846F8F786FC33
:1089A800184B93F82D3004F27C76022B294630467A
:1089B8000FD1FCF7F5F800239AB290420CD80023A7
:1089C80029462046C4F8F03605B0BDE8F040FDF76A
:1089D80097BEF8F70EFCEEE7B4F8E814B4F8EC74B8
:1089E8004A1C3A40B4F8EA7497421EBF0919F75C6A
:1089F80081F8EE7403F1010318BFA4F8E824DBE75B
:108A080020000020D4000020B0F81E36B0F81C2644
:108A18002DE9F04FD21A93B2110444BF03F58063D5
:108A28009BB2E62BADF5057D04460CD8DFF84C81EA
:108A380000F21C6600F2123904F20E374046FFF7C6
:108A480091FE054618B90DF5057DBDE8F08F404645
:108A5800FFF7B0F9394602464846FDF773FE00288D
:108A6800ECD094F813333E2B63D1B4F81633B3F536
:108A7800005F35D194F8983A002B5AD104AF04F22C
:108A8800273A04F69F2E9C4619464FF0010B3B608F
:108A98001EF8012FFF2A0BD0D00802F007021AF89F
:108AA80000001041C20742BF0BFA03F21143AC4663
:108AB8000133152BECD1BCF1000F00D03960042331
:108AC800CDE9007304F6B52002223E2142F6FF7379
:108AD8000746F8F7E5FC394602463046FFF71AFE26
:108AE800B4F816A3BAF1740F23D10DF1100B04F5E5
:108AF8002A630025009304F21A32B4F81833ADF84B
:108B08000E500DF10E015846FEF784F8BDF80E30F0
:108B180084F8985A04F6B527CDE900B302223E211D
:108B280053463846FEF753F8394602463046FFF7B3
:108B3800F1FD94F81333212B09D1B4F8163341F21F
:108B48000D02934212D041F20E02934212D0002D30
:108B58003FF472AF04F6B52549462846FDF7E2FF13
:108B6800294602463046FFF7D5FD65E7012384F81C
:108B7800453A61E7012384F8463A5DE72000002082
:108B88002DE9F047354B1B78022B04460CD0002307
:108B9800A0F81E36A0F81C3690F86D3A13B10A22D8
:108BA800B2FBF3F384F8983A2D4B93F82D30032B4E
:108BB80051D12046FFF728FF94F8422A3AB1002302
:108BC80084F8423A2046BDE8F047FFF725B894F804
:108BD800433A33B184F8432A2046BDE8F047FFF70B
:108BE8003DB894F8448AB8F1000F06D084F8443AA6
:108BF8002046BDE8F047FFF77FB81A4B1F68D4F846
:108C0800583AFB1A632B26D9C4F8587A254604F635
:108C18005C2604F1300940F6AB5A95F8702AAAB1DF
:108C280095F8713A0133DBB29A420BD885F8718A0C
:108C3800D5F8743AFB1A534508D931882046FEF70F
:108C4800D9FF03E085F8713A002BF1D008354D457E
:108C580006F10206E1D1BDE8F08700BF9F130020AE
:108C6800D4000020944A002008B5054B1B781BB19E
:108C7800BDE80840F9F7AEBC0248FFF760FD08BD43
:108C880000000020DC13002038B5B0F8EA24B0F862
:108C9800E8349B1A9DB21B0448BF05F500750446CD
:108CA800054848BFADB2FFF7DFFF4319D4F8F00617
:108CB800184480B238BD00BF20000020F8B5D0F8B5
:108CC800F43690F81877CB1AB3F57A7F04460E4637
:108CD80026D2632B01D800207DE0012F0AD0022F75
:108CE80019D0002FF7D1FFF7CFFFB0F5806FF2D979
:108CF800012305E0FFF7C8FFB0F5806F03D9022311
:108D080084F818370CE02046FFF7BEFFB0F5C07FA7
:108D1800E1D20023F4E7FFF7B7FFB0F5806FE7D3A0
:108D28003448C4F8F466F7F769FB334D334A2B68C7
:108D38001168C3F1000C411A614501DB99424BDD12
:108D480010600A232B601368B3F5FA7FBCBF4FF499
:108D5800FA7313601268D4F8F83652214A43284946
:108D68006425B1F8481092FBF1F26B43B3FBF2F3C0
:108D78005F2B35D8552B35D83B2B03D94B2B34BF1C
:108D88005B25322594F81837022B2DD0012B2DD0D6
:108D980013B9002F18BF33254FF47A73D4F800277E
:108DA800314604F20470F8F71BF994F81837FBB948
:108DB800642D0BD1D4F8F436A3F29A23C4F8F43610
:108DC800D4F8F83603225B00B3FBF2F3C4F8F836A4
:108DD80084F8FC560120F8BD002BB4DD013BB1E757
:108DE8000025CFE71E25CDE70025D5E73225D3E7B7
:108DF8000023EBE7843B0020140000203C03002004
:108E08007800002070B5D0F8F43690F81827CB1AFF
:108E1800B3F57A7F04460E4614D2032A08D8DFE851
:108E280002F002092730FFF72FFFB0F5487F26D858
:108E3800002029E0FFF728FFB0F5AF6F11D9022312
:108E480084F81837304B94F81857B3F84800C4F82A
:108E5800F466D4F8F836032D4ED8DFE805F0371657
:108E6800494B2046FFF710FFA328E1D80323E7E783
:108E7800632BDDD9FFF708FFB0F5AF6FE2D201230E
:108E8800DEE7002084F8180770BD21254FF47A73B7
:108E9800D4F80027314604F20470F8F7A1F894F8E2
:108EA80018377BBB642D0BD1D4F8F436A3F548737F
:108EB800C4F8F436D4F8F83605229B00B3FBF2F375
:108EC800C4F8F83684F8FC560120DDE764210F4A1F
:108ED800B2FBF0F24B43B3FBF2F35F2BD6D8552B22
:108EE8000CD83B2B0CD94B2B34BF5B253225CDE757
:108EF8000025CBE75D25C9E76425C7E71E25C5E73B
:108F08000D46C3E70023DBE778000020504001004E
:108F18002DE9F041494BDFF830811E6898F80030A0
:108F2800474F022B1EBF0023A0F8EA34A0F8E8340C
:108F380097F82D30013B012B04467CD8FFF7FCFC49
:108F480097F82E50002D5AD098F80030022B4AD1AD
:108F5800012D3DD0022D41D000252046FDF732FBE2
:108F680094F8193743B1002384F8193797F830304B
:108F7800012B4ED0022B4FD015B12046FEF7AEFA8A
:108F880094F86D372BB1002384F86D372046FEF72F
:108F980041FD94F87437022B11D1D4F87837F61ABA
:108FA800B6F57A7F0BD9B4F87037F62B3DD0B3F508
:108FB800FA7F3CD00023A4F8703784F87437237EF6
:108FC800CBB3002323762046BDE8F041FEF774BDFD
:108FD80031462046FFF772FE0546BEE73146204679
:108FE800FFF710FFF8E7D4F8F436F31AB3F57A7FF1
:108FF80008D2002504F20470F7F7ECFFADE7C4F8D7
:10900800F466F7E73223C4F8F46684F8FC360125E1
:10901800F0E7FEF7ADFAAFE7FEF726FB2046FEF7CE
:109028007FFB2046FEF74EFCA6E7F8F7E9FD054B67
:1090380001225A71BEE7BDE8F08100BF944A0020C2
:10904800D4000020480300209F1300202DE9F04F92
:10905800DFF8408398F80030012B85B000F21981C1
:109068000BB9F8F70FFEA84DFFF74CF9696CA74844
:10907800F9F704FBA64B00221A809A704FF0904330
:1090880001229A6207244CF25030013CF8F7BCFEEA
:10909800F9F77AF814F0FF04F5D19E4805F022F8A4
:1090A800013880B24FF6FD73984203D99A490120DE
:1090B800FBF714F9994B97481C80994B01211C80A8
:1090C80004F0D6FF97499348FAF7CCFA7D20F9F7D0
:1090D8005BF89548F8F758FEFAF7A8FE95F820B01F
:1090E800BBF1200F00D9FEE795F828008F4EAB8D15
:1090F80003930528696A95F8297095F82A30B071A4
:1091080000D9FEE78A4A4FEA001E02EB001C52F81B
:109118000E2002B9FEE7B2609CF804209CF80C907F
:109128000292F271DCF80820326186F80C9086F819
:10913800D900B482A446A246A646039A42FA0CF283
:10914800D20707D5012202FA0CFA4EEA0A0A1FFAD8
:109158008AFE92460CF1010CBCF1060FEDD1DFF846
:10916800CCC1BAF1000F01D0ACF814E0BCF814E09F
:10917800BEF1000F00D1FEE7029AA2EB0902D2B2BB
:109188005A4528BF5A4605288CF8172000F0A980B0
:10919800012800F2AD8007F1FF30C0B200F09780DF
:1091A800022817D8581EC0B203280CD80C2A02D996
:1091B8000C208CF817009CF81700904201D98CF805
:1091C80017203C4609E0122A84BF12238CF8173076
:1091D8000023F0E7052B28BF002354482246F7F761
:1091E80061FC0024534B86F8D840B4754F48FF26DD
:1091F8001E705E70FAF7ECFA0146464804F028FE45
:109208004D4B4E481C704E4B1C704E4B1C804E4BA9
:109218001C704E4B1C704E4B1C704E4B1C704E4BB2
:109228001C704E4B1C70FFF731F94D4BB5F84A20B6
:109238001C704C4B95F840101C704B4B1C70B5F8CB
:109248004830F7F762F8B5F848104848F7F7A9FB2F
:109258004748FBF74BF8474B474893F8291000F06D
:10926800C0FC4648FDF752F94548FDF74BFD294833
:10927800FAF79FFA01464348FAF77CFF4248FDF7A0
:10928800AFFE424B1C80424B1C80F9F7B3FA88F8BA
:109298000060F9F7B9FA002800F0A380294A13887A
:1092A8000BB1013B1380264B194A19781388022900
:1092B80022D12BB3013B9BB213809278002A6BD04A
:1092C800002B73D1F8F794FDF8F79EFD6EE00228A5
:1092D80005D80C2A02D90C238CF817303C460023F9
:1092E8007BE77B1E022BFAD8082AF7D90823F3E775
:1092F8000E48F7F771FB74E7002BDBD1C723DBE7D8
:1093080040F2F313D8E700BF7800002020000020C7
:10931800CA230020403C002098E70008C62300200C
:10932800C82300207C00002048030020942100204E
:10933800D0EA0008C93A0020D0230020843B00204E
:109348009F130020A2130020A01300209C130020CC
:109358009D1300209E130020CF230020CE23002041
:10936800A7130020A6130020C4230020603C00207F
:10937800583C0020D4000020543A0020D823002074
:10938800802C002092210020B0130020703C002087
:10939800723C0020C83A002002294FF0904040F06B
:1093A80088800BB9F8F724FD012383629F4C23883A
:1093B800002B00F08480013B9BB29D482380FAF784
:1093C80077FD9C48FAF7F5F901469B48FAF7D2FE73
:1093D8009A48FEF7CBFE23881BB999499948F8F7B4
:1093E8006FFA994D994C297800296BD0022900F021
:1093F800968023889BB2FBB12B78032B40F09A8090
:109408002388DE0702D5002323802B7023889BB294
:1094180093B12388590448BF238823889A0748BFF3
:10942800238823888A4ADB0748BF238800231370D0
:10943800884A23802B701370874B1A7802F0FF0636
:10944800002A00F0D68100201870824B1F7807F19F
:10945800FF3CDCF1000848EB0C08002F7DD0FFF73B
:10946800B3F87E4A0023012F137205D87C4A13777C
:10947800D38313627B4A13707B4C2278012A00F253
:109488008A80012F13D9794F97F8A8303E2B6DD8D1
:10949800774997F8A770887D002F75D1834260D0EF
:1094A800CA7D8B759A429CBF00238B75B0460026F7
:1094B8007AE002228262002B7FF478AF04E740F260
:1094C800E7337AE7684B1B7843B1694A937DD07DCF
:1094D8000133DBB29842937598BF91756448FAF7E7
:1094E80077F90146534804F0B3FC52484FF6FF7130
:1094F800F8F71AFC04F036FD00224E48012104F06A
:109508006FFD7D20F8F740FE514A01232B700023A0
:109518001370504A1370574A1380238069E75648DE
:10952800FAF724FF4D4B187AFFF7EAF903232B705B
:109538000023F0E7012B7FF469AF238898077FF5B4
:1095480065AF434B1978B1FA81F1002049092080B1
:10955800FFF77EF83F4B187058E7484B01221A7006
:109568007FE74748017841F0010101704549002A29
:1095780040F092803F2B424B0A704FF0010028BF09
:10958800032220701A7008E0834289D13C48017890
:1095980041F00201E9E7012F89D93B4BB3F84C2090
:1095A8003A4B1A8002232B702378002B40F0B281AB
:1095B800B8F1000F00D02B703549334A0B78B2F858
:1095C8004E200133DBB293420B70294A0ADB937DAC
:1095D800D07D0133DBB2984298BF002393750023F6
:1095E8000B702B7092F8D830002B7CD0B2F8DC309E
:1095F800B2F8DA1001339BB29942A2F8DC3072D883
:109608000023A2F8DC30908A92F8D9300621013381
:10961800DBB2062B28BF002340FA03F7FF075ED50D
:109628001C4819014158002954D1FEE7703C00201C
:1096380048030020403C002092210020B013002065
:1096480038E700081C000020D0230020C823002091
:10965800CF230020CE230020A5130020603C00204B
:10966800D8230020802C00209F130020843B00205A
:1096780094210020C6230020C93A0020583C00202D
:109688009C130020A013002078000020A2130020C3
:109698009D130020D0EA00080B78A3480133027814
:1096A800DBB20B7072B9A14A92F850209A423FF689
:1096B80074AF9F4B1B78032B06D102232370012321
:1096C80003706AE70522F1E7531EDBB29A420B707A
:1096D800F3D962E782F8D93000232B7003E001390F
:1096E80011F0FF0193D1934B00221A702278002ABF
:1096F80000F00A811EB901221A7002232B708E48CD
:10970800FAF714F82378022B02D08C4B00221A7037
:109718008B4A138813B9854BB3F84A30013B9BB287
:10972800138013B98748F6F775FE8648F6F726FEC4
:109738002378022B0BD08348F6F7CFFD237833B973
:10974800FEF7B2FE804A01231370804A1370804EE0
:109758003046F9F7C9F873787E48012B01BF00221B
:1097680072707C4A5371FAF7CDFBFAF7E3FB0128D4
:10977800064607D002282DD0774B05221A7005B06F
:10978800BDE8F08F694F7348FAF76CFBB7F84830BB
:10979800724A734803EB830303EB83039B00138034
:1097A800F9F754F96F4AB7F8481082F8D86041F2CF
:1097B8008833B3FBF1F3A2F8DA300023A2F8DC30E7
:1097C8004FF09042022191619662674A2370967029
:1097D8002B70D1E7634B93F8D930052B08D8634A2F
:1097E800D25C634B83F81921624B01221A70C3E7DC
:1097F800FEE75949604A0B781BB1013BDBB20B709D
:1098080013B11378002B39D0594D5C4895F82810BE
:109818000024147000F010FA594B1B78022B4DD11C
:10982800444E484832780292F6F7B1FD074645485B
:10983800F6F7BFFD029A53492346CDE900704F4819
:1098480000F012FD4D48FAF7E1FD32784E494F48D5
:109858002346FCF745FD234632784B494C48FDF733
:109868008BFA49494B482246FDF7A2FC95F8263069
:1098780095F8332043494848FAF798FD3F4800F0E7
:1098880006FE4248FFF744FB4148FFF779F9FDF728
:109898006FFBFDF791FB374B1B78002B3FF46FAF45
:1098A8002548F9F743FF4FF09043012402229C61B9
:1098B8009A61F9F717FE88F8004060E71A4B1B78A1
:1098C800EBB16FF07E03009301231A462D492B4814
:1098D800019400F0C9FC294800F0C5F901231A4693
:1098E80029492A48FCF7FCFC0123274928481A463D
:1098F800FDF742FA244927480122FDF759FC264B77
:1099080095F826205A70B9E72B7813F0FD0F3FF42D
:10991800F6AEFAE6214B1B88002B7FF4E4AE204A12
:1099280023701370D9E600BF9E1300207800002032
:109938009C130020C4230020403C0020583C0020F9
:10994800723C0020843B0020D1230020743C00207E
:109958009C3A002048030020A71300207400002030
:10996800813B002094210020CA230020C8EA000877
:10997800D4000020A4130020A6130020543A00208D
:109988009F130020A43A0020783A0020D823002012
:10999800802C0020B0130020C93A0020A213002018
:1099A8009D13002008B5FFF751FBFCE7F8B5044606
:1099B8003A480D4602F092FF28B9D4F84C3A0133E0
:1099C800C4F84C3AF8BD04F658212846F7F7B5FA1A
:1099D8000028F2D1EB7E002BEFD0304894F8596A7A
:1099E80002F07CFF8642EDD194F95A3A002BE9D176
:1099F8002B4B93F82D305A1E012A2CD894F8583A3C
:109A0800FF2B01D0012BD8D194F828303BB1EA7E46
:109A18009A421EBFD4F84C3A0133C4F84C3AEB7E54
:109A280094F8605A84F82830002DCBD0A38D268E68
:109A3800E78D01333340BB4207D004F12C00FEF719
:109A48007EFEC5F5006398420BDBD4F8483A013333
:109A5800C4F8483AB6E7032BD6D194F8583AFF2B06
:109A6800D1E7ADB2002304F66120A18D4A1C324033
:109A780097421EBF091910F803C081F832C003F1DC
:109A8800010318BFA2859AB29542EED8D4F8403A9D
:109A980094F8602A1344C4F8403A93E7700300200E
:109AA800D40000200B7E012B0A4606D1CB8A012B5D
:109AB80014D101460A48FEF7F3B9022B0ED1CB8A1E
:109AC800012B04D040F6B932934204D070470146C6
:109AD8000348FEF757BA0248FFF768BF704700BF50
:109AE800B013002038B5214B214A1A60214B224A75
:109AF800224C1A605A619A62DA631A65204A5A66D9
:109B08009A67204AC3F88C20204600F051F81E4B73
:109B180023601E4B1E4C002240F2FF11C3F8E824BC
:109B2800C3F8EC141B4B2068C3F81C2640F2FF3125
:109B3800C3F820167D2183F8541A6168C3F8502AA7
:109B480003F65C2503C5A068218A2860E068A3F8AD
:109B58006C1AC3F8680A104B40F2FF71DA62C3F856
:109B680030280E4A1963C3F8342838BD403C002019
:109B7800ACE70008843B002094E50008543A002034
:109B88007CE5000888E5000834E80008D8230020B0
:109B98009CE30008802C0020B01300200000FF0187
:109BA8007047002070470020704700207047000071
:109BB80010B5044B0446012140F8043BF6F73AFB84
:109BC800204610BD6403010838B5242204460D461A
:109BD800FF23002103618182104404F05FFBE560EC
:109BE80038BD38B50D46017CA942044615D0012977
:109BF80018D0022912D011B903685B68984700236E
:109C0800012D6374257413D0022D0ED02DB923684D
:109C18005B68012120469847607438BD0368DB689B
:109C28000021EBE703689B68FAE72368DB68F0E745
:109C3800236829469B68EDE70430F6F709BB037CE7
:109C4800012B10B50ED100F1160301F10C0251F8E9
:109C5800044B43F8044B9142F9D10A881A8040F228
:109C68000113438210BD037C012B0BD148F28113F1
:109C7800C3824FF401420023C0E90632038440F254
:109C8800011343827047F0B5054689B008880C4631
:109C980016461F46F6F742FC9DF806308DF805007B
:109CA80023F00703C0F30220034360888DF80630D1
:109CB800F6F734FC9DF8063000F01F0203F00703A6
:109CC80043EAC2038DF806309DF80730C0F345100B
:109CD80023F03F030343A0888DF80730F6F71EFCF6
:109CE8009DF8073000F0030203F03F0343EA8213B4
:109CF8008DF80730C0F387038DF808309DF80930D8
:109D0800C0F3802023F001030343E0888DF8093075
:109D1800F6F704FC9DF8093000F07F0203F0010318
:109D280043EA42038DF809309DF80A30C0F3C310A6
:109D380023F00F03034320898DF80A30F6F7EEFB72
:109D48009DF80A3000F00F0203F00F0343EA0213F4
:109D58008DF80A309DF80B30C0F3061023F07F030E
:109D6800034360898DF80B30F6F7D8FB9DF80B306C
:109D780000F0010203F07F0343EAC2138DF80B30B1
:109D8800C0F347038DF80C309DF80D30C0F3412027
:109D980023F003030343A0898DF80D30F6F7BEFBCB
:109DA8009DF80D3000F03F0203F0030343EA8203FD
:109DB8008DF80D309DF80E30C0F3841023F01F038A
:109DC8000343E0898DF80E30F6F7A8FB9DF80E30B6
:109DD80000F0070203F01F03C0F3C70043EA421371
:109DE8008DF80F00208A8DF80E30F6F797FB9DF856
:109DF80011308DF8100023F00703C0F3022003434D
:109E0800608A8DF81130F6F789FB9DF8113000F063
:109E18001F0203F0070343EAC2038DF811309DF8CF
:109E28001230C0F3451023F03F030343A08A8DF896
:109E38001230F6F773FB9DF8123000F0030203F0BE
:109E48003F0343EA82138DF81230C0F387038DF87D
:109E580013309DF81430C0F3802023F0010303432E
:109E6800E08A8DF81430F6F759FB9DF8143000F0AD
:109E78007F0203F0010343EA42038DF814309DF892
:109E88001530C0F3C31023F00F030343208B8DF864
:109E98001530F6F743FB9DF8153000F00F0203F07C
:109EA8000F0343EA02138DF815309DF81630C0F3FE
:109EB800061023F07F030343608B8DF81630F6F706
:109EC8002DFB9DF8163000F0010203F07F0343EAF2
:109ED800C2138DF81630C0F347038DF817309DF87C
:109EE8001830C0F3412123F003030B43A08B8DF8F6
:109EF8001830F6F713FB9DF8183000F03F0203F016
:109F0800030343EA82038DF818309DF81930C0F333
:109F1800841023F01F030343E08B8DF81930F6F704
:109F2800FDFA9DF81930218C00F0070203F01F0399
:109F380043EA42138DF81930628C40F2A9539942D2
:109F480088BF0121C0F3C70098BF00219A428DF84D
:109F58001A0088BF41F002010EB141F004010FB1AF
:109F680041F008010F238DF8043000238DF81C30D0
:109F78002B688DF81B101B68192201A928469847E1
:109F880009B0F0BD30B5054689B008880C46F6F72B
:109F9800D2FA9DF808308DF8070023F00703C0F3C4
:109FA8000220034360888DF80830F6F7C4FA9DF85C
:109FB800083000F01F0203F0070343EAC2038DF8DC
:109FC80008309DF80930C0F3451023F03F030343E0
:109FD800A0888DF80930F6F7AEFA9DF8093000F040
:109FE800030203F03F0343EA82138DF80930C0F3FC
:109FF80087038DF80A309DF80B30C0F3802023F0DA
:10A0080001030343E0888DF80B30F6F794FA9DF8C6
:10A018000B3000F07F0203F0010343EA42038DF89E
:10A028000B309DF80C30C0F3C31023F00F0303432B
:10A0380020898DF80C30F6F77EFA9DF80C3000F088
:10A048000F0203F00F0343EA02138DF80C309DF85A
:10A058000D30C0F3061023F07F03034360898DF8A9
:10A068000D30F6F768FA9DF80D3000F0010203F0A4
:10A078007F0343EAC2138DF80D30C0F347038DF810
:10A088000E309DF80F30C0F3412023F00303034343
:10A09800A0898DF80F30F6F74EFA9DF80F3000F0D2
:10A0A8003F0203F0030343EA82038DF80F309DF863
:10A0B8001030C0F3841023F01F030343E0898DF8A8
:10A0C8001030F6F738FA9DF8103000F0070203F068
:10A0D8001F03C0F3C70043EA42138DF81100208A1A
:10A0E8008DF81030F6F727FA9DF813308DF8120026
:10A0F80023F00703C0F302200343608A8DF813306E
:10A10800F6F719FA9DF8133000F01F0203F0070361
:10A1180043EAC2038DF813309DF81430C0F345109C
:10A1280023F03F030343A08A8DF81430F6F703FAAF
:10A138009DF8143000F0030203F03F0343EA821352
:10A148009DF816208DF81430C0F387038DF815306C
:10A1580022F00102C0F380231343E08A8DF8163001
:10A16800F6F7E9F99DF8163000F07F0203F00103D5
:10A1780043EA42038DF816309DF81730C0F3C31038
:10A1880023F00F030343208B8DF81730F6F7D3F92C
:10A198009DF8173000F00F0203F00F0343EA021393
:10A1A8008DF817309DF81830C0F3061023F07F03A0
:10A1B8000343608B8DF81830F6F7BDF99DF8183019
:10A1C80000F0010203F07F0343EAC2139DF81A204E
:10A1D8008DF81830C0F347038DF8193022F00302C8
:10A1E800C0F341231343A08B8DF81A30F6F7A3F977
:10A1F8009DF81A3000F03F0203F0030343EA82039C
:10A208008DF81A309DF81B30C0F3841023F01F031B
:10A218000343E08B8DF81B30F6F78DF9019B03F0B3
:10A228007F42104B134301939DF81B3000F0070247
:10A2380003F01F03C0F3C70043EA42138DF81C0064
:10A248000DF10601172200208DF81B30F6F7DEF914
:10A258002B688DF81D001B681A2201A9284698470B
:10A2680009B030BDC81816002DE9F34700F12407DE
:10A278009DF928A09DF82C9090461E4604463B4622
:10A2880001F1240251F8040B43F8040B9142F9D16F
:10A29800201D39460190F5F7FFFFE1684B796EB153
:10A2A8000198042B78D8DFE803F07D77355D03004B
:10A2B8004FF00423C4E909330026B046E3681D794A
:10A2C8006B1E0B2B07D850460435F6F7FDF8EDB298
:10A2D80004EB45056884E3681D7B6B1E0B2B07D8D0
:10A2E80048460435F6F70BF9EDB204EB45056884EA
:10A2F800637C002B56D0237C012B46D013F0FD0F36
:10A3080050D1334642463946204602B0BDE8F047B0
:10A31800FFF7B9BC01F1130304F1220001F11F0595
:10A328004FF0780C13F9012FC2EB8222AB4292FB5B
:10A33800FCF202F5806220F8022FF3D104F13A0210
:10A34800233140F2FF7513F8010F48B102280CBF02
:10A3580028464FF48060994222F8020FF3D1ADE706
:10A368000120F8E704F1220304F146024FF480616A
:10A3780023F8021F9342FBD10221F5F7ABFF1030FF
:10A3880004EB40000023838098E73946204602B05A
:10A39800BDE8F047FFF7F6BD042B8FD813F0FD0F8B
:10A3A8008CD0E9E702B0BDE8F08730B54B7B032BD2
:10A3B80085B005460C4642D191F90000F6F700F940
:10A3C8008DF8030094F90100F6F7FAF8A3788DF8F0
:10A3D8000530E3788DF804008DF80630207B23796A
:10A3E8008DF80730F6F7E4F88DF8080094F90600C0
:10A3F800F6F7B9F88DF8090094F90700F6F7E0F8D0
:10A40800237A8DF80B30637A8DF80C3040F6C84308
:10A418008DF80A00ADF800300DF1020114230B226B
:10A4280000208DF80230F6F7F1F82B688DF80D0052
:10A438001B680E2269462846984705B030BD022B96
:10A4480003D1FF238DF80330BCE791F90000F6F73C
:10A45800B7F88DF80300FF20B8E7837C10B50446F1
:10A4680033B1F8F7F3F9E37C1BB10023A082E3745E
:10A4780010BDA28A801A80B2B0F57A6FF8D9A37499
:10A4880004F116012046BDE81040FFF78EBF427C5C
:10A4980022B1037C012B01D1FFF7DFBF704710B554
:10A4A80094B03822002106A803F0F8FE14220021F7
:10A4B80001A803F0F3FE002000F0D2FC01224FF4C3
:10A4C8008033CDE9062303240223552206A8CDE9CB
:10A4D8000D34CDE91023CDE912330F9300F022FD9E
:10A4E80008B172B6FEE70421CDE903000F230590F9
:10A4F8000DEB0100CDE9013400F05AFF08B172B646
:10A50800FEE714B010BD000007B5104A136823F425
:10A518008063136000F0B2F8FFF7C1FF0C4BDA6CF0
:10A5280042F02002DA64DA6C02F020020192019A09
:10A53800DA6C42F00102DA64DB6C03F00103009389
:10A54800009B03B05DF804EBFFF72CBA0020024033
:10A55800001002400B4B1A6E42F001021A661A6E86
:10A5680082B002F001020092009A9A6D42F0805285
:10A578009A659B6D03F080530193019B02B000F034
:10A58800C9BC00BF00100240FEE7FEE7FEE7FEE799
:10A59800FEE7704770477047F8F746B9034AD2F8A4
:10A5A800883043F47003C2F88830704700ED00E04B
:10A5B8000D488546FFF7F2FF0C480D490D4A002368
:10A5C80002E0D458C4500433C4188C42F9D30A4A60
:10A5D8000A4C002301E013600432A242FBD303F0CB
:10A5E80093FEFFF791FFFEE70080002000000020A7
:10A5F80058000020D803010858000020744F00209C
:10A60800FEE7704710B5094B4FF0FF3200249A63FC
:10A618009C631A641C649A629C62DA62DC621A6344
:10A628001C63FFF7EEFF204610BD00BF001002407C
:10A6380038B50F4B1A6805460AB9012038BD4FF4E2
:10A648007A73B3FBF2F30B4A1068B0FBF3F000F037
:10A658006FF804460028F0D10F2DEED8024629469F
:10A668004FF0FF3000F032F8034B20461D60E5E75D
:10A67800300000202C0000203400002010B50320FA
:10A6880000F012F80F20FFF7D3FF044618B9FFF7C0
:10A6980061FF204610BD0124FBE70000014B18684C
:10A6A800704700BF944A00200749CA6822F4E06254
:10A6B8000302120403F4E063120C134343F0BF6374
:10A6C80043F40033CB60704700ED00E0164B30B523
:10A6D800DC68C4F30224C4F10703251D042B28BF3A
:10A6E8000423062D4FF0FF358CBF033C002405FAE8
:10A6F80003F321EA0303A54022EA0502A340002848
:10A7080043EA0203ACBF00F16040084A4FEA031372
:10A71800B8BF00F00F00DBB2AABF00F561401354C8
:10A7280080F8003330BD00BF00ED00E014ED00E01C
:10A738000138B0F1807F0BD24FF0E023054A586111
:10A74800F02182F823100020072298611A617047CF
:10A758000120704700ED00E07047000038B504465E
:10A76800002800F0BA8090F85C3003F0FF021BB9B3
:10A7780080F85D20FFF7F0FF2268936923F010034B
:10A788009361FFF78BFF054623689A69110700F16B
:10A7980097809A6942F001029A61FFF77FFF0546A8
:10A7A80023689A69D20740F19A809A6942F00202B6
:10A7B8009A61574A934204BF6168C2F80011227C2B
:10A7C800012A9A690CBF22F0400242F040029A61C5
:10A7D800627C012A9A690CBF42F4804222F48042CA
:10A7E8009A61A27C012A9A690CBF22F4805242F431
:10A7F80080529A619A69A06822F4407202439A6171
:10A808009A6922F0A4029A611A6922F010021A6168
:10A81800E268012A6AD19A6942F004029A61A2693F
:10A82800511EE269013A120242EA4162216A013983
:10A838000A436169013942EA0142B0F5407FDA61B1
:10A848000ED1E26A511E226B013A120142EA01223C
:10A85800A16A01390A43616A013942EA0142DA60B0
:10A86800D3F8C020E16B2B480A43C3F8C020D3F8C3
:10A878008020616B206422F4F81242EA0142C3F896
:10A888008020254A6264D3F88020A16B22F0706290
:10A8980042EA0162C3F88020204BA364D833E36402
:10A8A800D8332365183363654FF45472002103F0DD
:10A8B800F5FC002001232066A06584F85C3038BDD3
:10A8C800FFF7ECFE401B0A287FF65EAF236E43F0CD
:10A8D80001032366032384F85C300120EFE7FFF7C8
:10A8E800DDFE401B0A287FF65BAFEFE7002A96D013
:10A8F800022A09D0996941F0800199611969032AEE
:10A9080041F0100119618AD19A6942F0200285E765
:10A918000064004000A4004070A40040B0A40040BF
:10A92800F0B590F85C30013B012B1BD8D1E900252C
:10A938008B684E69D1E903749B074AB943EAC76338
:10A94800016C334343EA044341F825300020F0BD4D
:10A95800426C02EBC50144EA4774334342F8354080
:10A968004B60F3E7036E43F0020303660120EEE752
:10A9780030B590F85C40012C10D105680398D5F8E3
:10A98800804040EA430343EA820242EA011124F08C
:10A998003F030B43C5F88030002030BD036E43F001
:10A9A800040303660120F8E790F85C30012B0BD113
:10A9B8000268022380F85C30936923F001039361F5
:10A9C8000023036618467047036E43F004030366CA
:10A9D800012070472DE9F04390F85C30022B914636
:10A9E80059D10668D6F8C44014F4001405D0036E93
:10A9F80043F400730366012031E0D1E90032D6F850
:10AA0800C450D1F810C08F68C5F301454ABB47EA66
:10AA18000C0E4EEA834CD1E906733B434F69D0F8DC
:10AA280054803B43CF683B430F6A43EA0763482798
:10AA38006F4307EB080E47F808C0194FCEF80430EB
:10AA48004A460EF1080ECB89FB5C9C4202F10402D7
:10AA58000ED30123AB40C6F8CC3083650020BDE897
:10AA6800F08343EA0C0C4CEA070C4CF0804CD2E71C
:10AA780012F8023C12F801CC1B0443EA0C6312F8EA
:10AA880004CC43EA0C0312F803CC43EA0C234EF837
:10AA980004300434D7E7036E43F00803AAE700BF85
:10AAA8008C03010890F85C30022B15BF036E036815
:10AAB80043F00803002016BF0366C3F8D010012036
:10AAC80070470368D3F8C40000F00700704730B53A
:10AAD80090F85C30013B012B60D8006811F0070545
:10AAE800836D01D0DC071DD511F0380F01D09C070C
:10AAF80018D511F4E07F01D05C0713D511F4F05F8D
:10AB080001D01C070ED511F4604F01D0DC0609D521
:10AB180011F4403F01D09C0604D511F47C0F05D0F8
:10AB28005C0603D4C46D44F00104C4650DB1DD07AF
:10AB38001DD411F0380F01D09C0718D411F4E07F10
:10AB480001D05D0713D411F4F05F01D01C070ED4B7
:10AB580011F4604F01D0DD0609D411F4403F01D053
:10AB68009C0604D411F47C0F05D05D0603D5C36D93
:10AB780043F00203C3650C0642BFD0F8DC30134330
:10AB8800C0F8DC30CB0542BFD0F8E0301343C0F842
:10AB9800E030436D0B434365002030BD036E43F046
:10ABA800020303660120F8E7094A536943F4802346
:10ABB80010B55361EFF3108272B60023CC58C4501D
:10ABC8000433B3F5807FF9D182F3108810BD00BF3C
:10ABD80000200240064B5A69002ABFBF054A9A6006
:10ABE80002F188329A60BABF5869C00F00207047D6
:10ABF8000020024023016745044B5A6942F0004295
:10AC08005A615869C043C00F704700BF0020024016
:10AC180070B50646FFF742FD0F4C05462369DB0376
:10AC28000BD423694CF2FA3213400DD00B494A6811
:10AC38001A434A600120236170BDFFF72FFD401BB6
:10AC4800B042EBD90320F7E7206910F00100F3D0F8
:10AC5800012222611846EFE7002002403800002058
:10AC68002DE9F0471D4E99463378012B05460F46CE
:10AC7800904631D04FF0010A4FF47A7086F800A060
:10AC8800FFF7C6FF0446B8B97060CDB9144A5369D6
:10AC980043EA0A035361C7F80080BFF36F8FC7F810
:10ACA800049054464FF47A70FFF7B2FF24B10C4A6F
:10ACB800536923EA0403536100233370BDE8F08726
:10ACC8006B1E012BEED841463846FFF76DFFAB1ED1
:10ACD8005D425D41AC04E5E70220EFE73800002063
:10ACE80000200240064B10F0010F1EBF5A6942F0C7
:10ACF80004025A615A6942F480325A61704700BFAF
:10AD080000200240084B5A69C00022F4FC7200F48B
:10AD1800FF60104358615A6942F002025A615A6949
:10AD280042F480325A617047002002401548037F80
:10AD3800DAB203F0FD03012B10D1134B196821F48B
:10AD480000711960196841F400611960196821F4EB
:10AD580000611960196841F400711960931E012B94
:10AD68000CD8094B1A6842F480521A601A6822F407
:10AD780080521A601A6842F480621A6000230377CE
:10AD8800704700BF38000020002002402DE9F8433A
:10AD9800314D2B78012B064688465AD001274FF4AF
:10ADA8007A702F70FFF734FF044610BB2B4B686096
:10ADB8001A6812F4007F1A6820D0510506D51A685F
:10ADC80022F480621A6003232B7700E02F77336820
:10ADD800012B1DD17068FFF785FF4FF47A70FFF7DC
:10ADE80017FF1E4A536923F0040304465361FFF713
:10ADF8009DFF00232B702046BDE8F883520505D53A
:10AE08001A6822F480621A600223DDE72877DEE7F9
:10AE18004FF0FF33C8F80030B768DFF84090D6E944
:10AE280002321344BB42E2D971683846FFF76AFF21
:10AE38004FF47A70FFF7ECFED9F8143023F4FD7361
:10AE4800C9F8143018B1C8F800700446CFE70137C4
:10AE5800E5E70224CFE700BF3800002000200240C9
:10AE6800294B1A6830BB02F4C062B2F5806FD3F880
:10AE7800802022F48072C3F880201AD11A6822F444
:10AE8800C06242F400721A60204A126832214A43B2
:10AE98001F49B2FBF1F201325969490500D522B9BF
:10AEA8005B69580503D400207047013AF4E7032092
:10AEB80070477047B0F5007F1FD102F4C062B2F549
:10AEC800806FD3F8802042F48072C3F88020EAD1E2
:10AED8001A6822F4C06242F400721A600B4A1268BF
:10AEE80032214A430A49B2FBF1F201325969490554
:10AEF800D6D5002AD4D0013AF8E722F4C06242F449
:10AF080080621A60CFE700BF007000402C0000206C
:10AF180040420F00024A936843F4804393607047AD
:10AF2800007000402DE9F341044640B30368DF0791
:10AF380014D423689E075BD423681E0700F1A480FD
:10AF480023685D0700F1CB8023689B0600F13281FE
:10AF5800E069002840F06081002028E0A14DAB683E
:10AF6800EA6803F00C030C2B0BD102F00303032B4C
:10AF780009D12B689D03DCD56368002BD9D101204A
:10AF880015E0082BF4E76368B3F5803F12D12B680E
:10AF980043F480332B60FFF781FB06462B68980348
:10AFA800C7D4FFF77BFB801B6428F7D9032002B0C6
:10AFB800BDE8F081B3F5A02F04D12B6843F48023BA
:10AFC8002B60E4E72A6822F480322A602A6822F497
:10AFD80080222A60002BDED1FFF760FB06462B6833
:10AFE8009903A6D5FFF75AFB801B6428F7D9DDE73C
:10AFF8007C4DAB68EA6803F00C030C2B17D102F008
:10B008000303022B15D12B685A0502D5E368002BE0
:10B01800B5D06B68226923F0FE4343EA02636B6094
:10B02800714B1868FFF704FB002885D0A7E7042BAD
:10B03800E8E7E368BBB12B6843F480732B60FFF744
:10B048002DFB06462B685B0507D56B68226923F044
:10B05800FE4343EA02636B606EE7FFF71FFB801B4A
:10B068000228EFD9A2E72B6823F480732B60FFF73F
:10B0780015FB06462B685F057FF55EAFFFF70EFBF5
:10B08800801B0228F6D991E76369564D9BB1D5F824
:10B09800943043F00103C5F89430FFF7FFFA0646F1
:10B0A800D5F8943098073FF54BAFFFF7F7FA801BB8
:10B0B8000228F5D97AE7D5F8943023F00103C5F8CA
:10B0C8009430FFF7EBFA0646D5F8943099077FF5E8
:10B0D80037AFFFF7E3FA801B0228F5D966E7414D41
:10B0E800AB6DDA0027D4AB6D43F08053AB65AB6D25
:10B0F80003F080530193019B01273C4E3368DB0525
:10B108001BD5A368012B29D1D5F8903043F0010352
:10B11800C5F89030FFF7C2FA41F288380646D5F8EC
:10B128009030990740D5002F3FF40EAFAB6D23F058
:10B138008053AB6508E70027DFE7336843F4807383
:10B148003360FFF7ABFA80463368D805D9D4FFF7E8
:10B15800A5FAA0EB08000228F6D927E7052B06D1A7
:10B16800D5F8903043F00403C5F89030CCE7D5F813
:10B17800902022F00102C5F89020D5F8902022F006
:10B188000402C5F89020002BC4D1FFF787FA41F2DA
:10B1980088380646D5F890309A07C4D5FFF77EFA66
:10B1A800801B4045F6D901E7FFF778FA801B404538
:10B1B800B5D9FBE6A3690B4DD3B1D5F8983043F068
:10B1C8000103C5F89830FFF769FA0646D5F89830B4
:10B1D8009F073FF5BDAEFFF761FA801B0228F5D93E
:10B1E800E4E600BF00100240340000200070004078
:10B1F800D5F8983023F00103C5F89830FFF74EFAD8
:10B208000646D5F8983098077FF5A2AEFFF746FABC
:10B21800801B0228F5D9C9E6484DAB6803F00C033A
:10B228000C2B57D02B68022823F080732B603AD15F
:10B23800FFF734FA06462B6899012ED4EA68404B8A
:10B248001340226A1343A26A43EA0223E26A43EAEA
:10B25800C263626A013A43EA0213226B5208013A56
:10B2680043EA4253626B5208013A43EA4263EB6095
:10B278002B6843F080732B60EB6843F08073EB60BE
:10B28800FFF70CFA04462B689A013FF565AEFFF705
:10B2980005FA001B0228F6D988E6FFF7FFF9801B9C
:10B2A8000228C8D982E6EB6823F00303EB60EB6859
:10B2B80023F0887323F48033EB60FFF7EFF904463B
:10B2C8002B689B017FF548AEFFF7E8F9001B0228C1
:10B2D800F6D96BE601283FF46AAEEB68226A03F000
:10B2E800030191427FF44BAE616A03F0F002013929
:10B2F800B2EB011F7FF443AEA16A03F4FE42B2EB46
:10B30800012F7FF43CAEE16A03F07842B2EBC16FE3
:10B318007FF435AE226B520803F4C001013AB1EB59
:10B32800425F7FF42CAE626B520803F0C063013AAF
:10B33800B3EB426F3FF410AE21E600BF00100240AD
:10B348000C809F01174B9A6802F00C02042A23D044
:10B358009A6802F00C02082A20D09A6802F00C02BF
:10B368000C2A1DD1D968DA68D868DB6801F00301B6
:10B37800C3F341630329C2F30312C0F3062003F1A8
:10B3880001030CBF084909495B000132B1FBF2F225
:10B398005043B0FBF3F070470448704702487047C9
:10B3A800002070470010024000127A000024F400C8
:10B3B8002DE9F8430E46054610B90120BDE8F8838B
:10B3C8006D4A136803F00F038B4245D3296811F0C7
:10B3D80001084CD12A68910740F1A780674B12F009
:10B3E800040F1EBF996841F4E0619960120741BFDC
:10B3F8009A6822F47C5242F4E0629A609A68A968DA
:10B4080022F0F0020A439A605B4C236803F00F03B2
:10B41800B34200F293802A68584C12F0040F40F0AF
:10B42800A380130706D5A3682A6923F4605343EA67
:10B43800C203A360FFF786FFA368514AC3F303134F
:10B44800D35C03F01F03D8404E4B18604E4B18686E
:10B45800BDE8F843FFF7ECB8136823F00F030B437C
:10B468001360136803F00F038B42A6D1AEE76F6831
:10B47800424C032F236849D19B019ED5E368E268BB
:10B4880003F00303032BE3680CBF40484048C2F3B2
:10B498000312C3F306230132B0FBF2F25343E2680E
:10B4A800C2F3416201325200B3FBF2F3394A9342CC
:10B4B8001AD84FF00008A36823F003033B43A360A6
:10B4C800FFF7ECF841F288390746A3686A6803F089
:10B4D8000C03B3EB820F3FF47DAFFFF7DFF8C01B1F
:10B4E8004845F2D9032069E7A36813F0F00F04D0A8
:10B4F8008807DED5AB68002BDBD1A36823F0F00307
:10B5080043F08003A3604FF08008D4E7022F09D1ED
:10B5180013F4003F3FF451AFFFF714FF1D4B98425F
:10B52800C7D9EAE713F4806FF4E7B8F1800F01BFD9
:10B53800124A936823F0F003936065E7236823F0C9
:10B548000F0333432360FFF7A9F841F28838074611
:10B55800236803F00F03B3423FF45DAFFFF79EF893
:10B56800C01B4045F4D9BDE7A368E96823F4E0634C
:10B578000B43A36055E700BF0020024000100240C3
:10B58800740301082C0000203400002000127A0007
:10B598000024F40000B4C404054B064A9B68C3F3B6
:10B5A8000223D35C044A106803F01F03D840704795
:10B5B80000100240840301082C000020054B064AB5
:10B5C8009B68C3F3C223D35C044A106803F01F03CB
:10B5D800D840704700100240840301082C00002066
:10B5E800B0F5002FA34B1DD1D3F89020D3F89010BD
:10B5F800890702F4407203D5B2F5807F00F0AC8170
:10B60800D3F89410880703D5B2F5007F00F0A7811E
:10B61800186810F400303ED09748B2F5407F18BF44
:10B6280000207047DA6802F00302022A1DD11A6866
:10B63800924912F4806218BF0A46D968B0F5807F33
:10B64800C1F3031101F10101B2FBF1F200F0008135
:10B6580022D8082815D8F0B1013807281AD8DFE809
:10B6680000F0617D1993191919A8DA6802F003022C
:10B67800032A04D11A68824912F40032DBE7002257
:10B68800DBE7402800F0C280802800F0D080202826
:10B6980000F0A48000207047B0F5805F00F02D8195
:10B6A80026D8B0F5806F00F0EF80B0F5006F00F09D
:10B6B8001081B0F5007FEDD1D3F8882012F4402234
:10B6C80051D0D3F89410880703D5B2F5802F00F035
:10B6D80046811968490503D5B2F5002F00F042816B
:10B6E800D3F8900010F00200D5D0B2F5402F30E02A
:10B6F800B0F5804F06D0B0F5004F00F00C81B0F5E2
:10B70800005FC7D1D3F8881001F04061B1F1006F34
:10B7180000F0C880D3F8980010F00200BBD0594858
:10B7280000297CE7D3F8882012F0030201D1FFF743
:10B7380045BF012A01D1FFF705BE1968490502D5A1
:10B74800022A00F00F81D3F8900010F00200A2D076
:10B75800032A14BF00220122D0037047D3F888209F
:10B7680012F00C0201D1FFF717BF042AE3D01968C1
:10B77800480502D5082A00F0F580D3F8900010F0AB
:10B78800020088D00C2AE4E7D3F8882012F03002AF
:10B79800E9D0102ACFD01968490502D5202A00F02F
:10B7A800E180D3F8900010F002003FF474AF302A23
:10B7B800CFE7D3F8882012F0C002D4D0402ABAD0FC
:10B7C8001968480502D5802A00F0CC80D3F890008B
:10B7D80010F002003FF45FAFC02ABAE7D3F8882020
:10B7E80012F44062BFD0B2F5806FA4D01968490541
:10B7F80003D5B2F5006F00F0B580D3F8900010F0D3
:10B8080002003FF448AFB2F5406FA2E7D3F88820B2
:10B8180012F44052A7D0B2F5805F8CD0186810F4AB
:10B8280080603FF438AFB2F5005F1448F7E6D3F80C
:10B83800882012F4404296D0B2F5804F3FF47BAF97
:10B84800186810F480603FF426AFB2F5004FECE7BB
:10B85800D3F8882012F4403285D0B2F5803F3FF407
:10B868006AAF186810F480603FF415AFB2F5003F76
:10B87800DBE700BF0010024090D003000024F40072
:10B8880000127A00006CDC02D3F8881011F4401121
:10B898003FF451AFB1F5801F10D1D86810F4801073
:10B8A8003FF4F9AED868DB68C3F34153C0F3062010
:10B8B800013350435B00B0FBF3F07047B1F5001F54
:10B8C80052D0186810F480603FF4E5AEB1F5401F1F
:10B8D800ABE7D3F8881011F440013FF42CAFB1F571
:10B8E800800FDAD0B1F5000F3ED0186810F48060F0
:10B8F8003FF4D1AEB1F5400F97E7D3F8881001F0C7
:10B908004071B1F1007F3FF42EAF79B3B1F1807F80
:10B918007FF4C0AEC1E7D3F8881001F04051B1F10F
:10B92800805F14D1D86810F480303FF4B4AED96881
:10B93800D868C00EC1F3062105D1DB6813F4003FB7
:10B9480014BF112007204A43B2FBF0F07047B1F151
:10B95800005F7FF49FAEEEE64FF4004070474FF46F
:10B96800FA407047024870470248704702487047DB
:10B978000024F4000080BB0000127A00024AD36A57
:10B988001843D062704700BF00100240B0F1904FDA
:10B9980008B509D10120FFF7F1FF254AD36A23F042
:10B9A8000103D362002008BD224B984207D1022030
:10B9B800FFF7E4FF1E4AD36A23F00203F1E71E4BA8
:10B9C800984207D10420FFF7D9FF194AD36A23F018
:10B9D8000403E6E7194B984207D10820FFF7CEFF8A
:10B9E800134AD36A23F00803DBE7154B984207D1C3
:10B9F8001020FFF7C3FF0E4AD36A23F01003D0E7E5
:10BA0800104B984207D12020FFF7B8FF084AD36AA5
:10BA180023F02003C5E70C4B984207D14020FFF7DD
:10BA2800ADFF034AD36A23F04003BAE70120BAE71F
:10BA3800001002400004004800080048000C0048BC
:10BA48000010004800140048001800482DE9F04F85
:10BA580002460D6895FAA5F44FF0010EB4FA84F485
:10BA680003274FF00F0C6FEA050835FA04F001D1EF
:10BA7800BDE8F08F0EFA04F32B4067D04868461EE5
:10BA8800012E1ED8966893FAA3F9B9FA89F94FEAF4
:10BA9800490907FA09F926EA090993FAA3FA8E6807
:10BAA800BAFA8AFA4FEA4A0A06FA0AF646EA09068A
:10BAB8009660566808EA0609CE686E4349EA0606A3
:10BAC8005660D66893FAA3F9B9FA89F94FEA490991
:10BAD80007FA09F926EA090993FAA3FA0E69BAFAE4
:10BAE8008AFA4FEA4A0A06FA0AF646EA09060228D4
:10BAF800D66018D1FF2BD1F814A029D8D2F82090FD
:10BB080093FAA3F6B6FA86F6B6000CFA06F629EA10
:10BB1800060993FAA3F6B6FA86F6B6000AFA06F606
:10BB280046EA09061662166893FAA3F9B9FA89F97A
:10BB38004FEA490907FA09F926EA090693FAA3F32D
:10BB4800B3FA83F35B0098403043106001348CE70C
:10BB5800D2F824901E0A96FAA6FBBBFA8BFB4FEA92
:10BB68008B0B0CFA0BFB29EA0B0996FAA6F6B6FA28
:10BB780086F6B6000AFA06FA4AEA09065662D2E7D3
:10BB8800024B1868C0F38020704700BF00100240C5
:10BB9800024BD3F89000C0F34000704700100240F9
:10BBA800024B1868C0F34060704700BF00100240A5
:10BBB800044B054A9B68C3F30313D35C03F01F03CC
:10BBC800D84070470010024074030108044B054A2E
:10BBD8009B68C3F30223D35C03F01F03D84070476C
:10BBE8000010024084030108124B9A6802F00C020C
:10BBF800082A1BD00C2A1BD1DA680F480F4902F01B
:10BC08000302032A08BF0146D868DA68DB68C3F371
:10BC18004163C0F30620C2F30312013348430132E3
:10BC28005B00B0FBF2F0B0FBF3F0704702487047DE
:10BC3800024870470010024000127A000024F40005
:10BC4800164A08B5136843F480731360FFF798FF2A
:10BC58000028FBD0536823F0FE4343F08043536031
:10BC680001239360936803F00C03042BFAD14FF47B
:10BC7800807313601360FFF793FF0028FBD14FF424
:10BC8800805140F23B73D16090611362D2F89430D6
:10BC980043F40003C2F8943008BD00BF001002400E
:10BCA800032810B52DD12D4C2D4AD4F8883003F037
:10BCB800030343F44033934209D0B3F1031F0CD07C
:10BCC800013A934210D1BDE81040FFF78DBFFFF74E
:10BCD80057FF002840D1002010BDFFF759FF00385A
:10BCE80018BF0120C003F7E7FFF77EFFFFF760FFEB
:10BCF800A3681C4AC3F3C223D35C03F01F03D840D4
:10BD0800EAE70C2817D1154B174AD3F8883003F007
:10BD18000C0343F440239342D9D0B3F10C1FDCD079
:10BD2800043A9342CFD0FFF75FFFFFF741FFBDE82A
:10BD38001040FFF74BBF3028CDD1084B0B4AD3F842
:10BD4800883003F0300343F440139342BFD0B3F17B
:10BD5800301FC2D0103AE4E70548BDE700100240A2
:10BD6800020003008403010808000C0020003000D2
:10BD78000024F400C02808B501D0002008BD144BE9
:10BD8800144AD3F8883003F0C00343F440039342C5
:10BD980009D0B3F1C01F0CD0403A934210D1BDE88E
:10BDA8000840FFF721BFFFF7EBFE0028E5D00A485F
:10BDB800E4E7FFF7EDFE003818BF0120C003DDE718
:10BDC800FFF712FFFFF7F4FEBDE80840FFF7FEBEDD
:10BDD800001002408000C0000024F40003685B06E5
:10BDE80070B502462DD4D1E900363343CE680568D4
:10BDF80048690C6A33430E6933438E6903433343FE
:10BE0800CE6925F47F45334325F0BF0523432B43F3
:10BE1800136053688D6823F4706323F0040345EAC4
:10BE280010401843B5F5006F50603EBF536843F4A7
:10BE380080535360B4F5005F01D18B8C13610020EF
:10BE480000E00120D36923F40063D36170BD0000D2
:10BE58002B4A036890420ED0B0F1804F0BD0A2F568
:10BE68009432904207D002F58062904203D002F5E6
:10BE78009632904215D14A6823F070031343204A42
:10BE8800904219D0B0F1804F16D0A2F5943290426A
:10BE980012D002F5806290420ED002F5963290429E
:10BEA8000AD0184A904207D002F58062904203D027
:10BEB80002F58062904203D1CA6823F440731343A9
:10BEC80003608B68C3620B8883620D4B98420FD066
:10BED80003F5006398420BD003F54063984207D0FE
:10BEE80003F58063984203D003F58063984201D13B
:10BEF8000B690363436943F0010343610020704702
:10BF0800002C014000400140B1F5805F30B500F0E1
:10BF180011810AD8102900F08680B1F5807F00F0E1
:10BF2800C68001293DD0012030BDB1F5803F00F029
:10BF38004781B1F5801FF6D1036A146823F4801392
:10BF48000362036A016D21F0807121F4E04141EA46
:10BF58000424116923F4001343EA0153516823F4BC
:10BF6800801343EA0153954988420FD001F50061D7
:10BF780088420BD001F54061884207D001F5806105
:10BF8800884203D001F58061884206D141689569ED
:10BF980021F4802141EA85214160D2680465C264A8
:10BFA8003EE0036A156823F001030362036A4168EF
:10BFB800846924F4803424F073042C43156923F035
:10BFC80002032B43556823F001032B437B4DA84202
:10BFD8000FD005F50065A8420BD005F54065A842CD
:10BFE80007D005F58065A84203D005F58065A8420D
:10BFF80012D1556923F0080343EA8503956823F0B5
:10C00800040343EA8503956921F480712943D569BE
:10C0180021F4007141EA4501D268416084614263BC
:10C028000362002080E7036A156823F010030362A7
:10C03800036A4168846924F0807424F4E64444EA7D
:10C048000524156923F0200343EA0513556823F0F6
:10C05800100343EA0513594DA8420FD005F50065B2
:10C06800A8420BD005F54065A84207D005F58065C4
:10C07800A84203D005F58065A84213D1556923F07D
:10C08800800343EA8513956823F0400343EA851348
:10C09800956921F4806141EA8501D56921F400613F
:10C0A80041EAC501D268416084618263B8E7036AE6
:10C0B800156823F480730362036A4168C46924F431
:10C0C800803424F073042C43156923F4007343EA85
:10C0D8000523556823F4807343EA0523374DA842A6
:10C0E8000FD005F50065A8420BD005F54065A842BC
:10C0F80007D005F58065A84203D005F58065A842FC
:10C1080013D1556923F4006343EA8523956823F422
:10C11800806343EA8523956921F4805141EA05113A
:10C12800D56921F4005141EA4511D2684160C461E2
:10C13800C26375E7036A156823F480530362036AD0
:10C148004168C46924F0807424F4E64444EA052470
:10C15800156923F4005343EA0533556823F48053E3
:10C1680043EA0533154DA8420FD005F50065A842EE
:10C178000BD005F54065A84207D005F58065A842B3
:10C1880003D005F58065A84213D1556923F400430F
:10C1980043EA8533956823F4804343EA85339569F8
:10C1A80021F4804141EA8511D56921F4004141EA31
:10C1B800C511D2684160C461026431E7002C0140B6
:10C1C800036A146823F480330362036A016D21F45F
:10C1D800803121F070010C43116923F4003343EAE4
:10C1E8000143516823F4803343EA01430F498842ED
:10C1F8000FD001F5006188420BD001F540618842FB
:10C2080007D001F58061884203D001F5806188423A
:10C2180006D14168956921F4803141EA05214160E0
:10C228000465D268816C8264FAE600BF002C014084
:10C238001C4B98420BD103F558431A6C42F48042C8
:10C248001A641A6C22F480421A6400207047164B54
:10C2580098420AD103F5E6339A6B42F400329A63A6
:10C268009A6B22F400329A63EFE7104B984209D197
:10C2780003F5E4339A6B42F480229A639A6B22F4B2
:10C288008022F0E70A4B984209D103F5E2339A6B12
:10C2980042F400229A639A6B22F40022E3E7012019
:10C2A800704700BF0038014000440040004800408B
:10C2B800004C004038B50368DB0704460D4659D4E6
:10C2C8002A69AB68016813436A691343EA6913432F
:10C2D800294A0A40134303604368EA6823F4405339
:10C2E800134343608368AA6923F44073134383604C
:10C2F800224B984220D10320FFF7D2FC2B6840B391
:10C308006A6832B30B2B15D81D4951F82330E969F7
:10C31800B0FBF3F0B1F5004F4FEA520325D103EB20
:10C328004003B3FBF2F34FF6F0721A40C3F3420333
:10C338001343E36000200DE0124B984201D10C201A
:10C34800DAE7114B984201D13020D5E70F4B9842DC
:10C3580007D00120E26A2B8822F00F021343E36220
:10C3680038BDC020FFF706FDC8E70344B3FBF2F36E
:10C378009BB2DEE70120F3E7F369FFEF00380140E5
:10C388009C0301080044004000480040004C004065
:10C398000E2815D8DFE800F0151515151515151513
:10C3A80015080A0C0E1012000C2070471020704758
:10C3B800142070471820704720207047302070479D
:10C3C800402070472DE9F041456A35B94162BDE822
:10C3D800F081CEF800100B60F9E74E6826F0604C4B
:10C3E800C6F38A47C6F3807817EA260738BF674638
:10C3F800AE462B465A6892EA060F22F060440CD5E6
:10C40800002A1DDAA40CBC4201D0BC420DD99D42C1
:10C41800DFD10D60DAE71346ECE7A4450BD102F053
:10C428008044C2F38072424507D11A689E46002AAA
:10C43800F1D11960CBE7F8D2E9E7002CF5D0E6E7AF
:10C44800BC42E2D1F1E72DE9F047089E01F007056B
:10C458004FEAD6082A4406F0070600EBD1014FF44C
:10C468007F49954201D1BDE8F08705F0070C06F039
:10C47800070AD445674638BF5746C7F10807501B17
:10C48800EC08874228BF07460C5D08EBD60004FA83
:10C498000CF413F800E029FA07FC24FA0AF45FFA0E
:10C4A8008CFC8EEA04044CFA0AFC04EA0C048EEABA
:10C4B800040E03F800E03D443E44D2E780EA012040
:10C4C800082341F2210201B24000002980B203F1A1
:10C4D800FF33B8BF504013F0FF03F4D1704738B5AD
:10C4E8000C468D18A54200D138BD14F8011BFFF782
:10C4F800E5FFF7E742684AB11368436043898189D9
:10C5080001339BB29942438138BF838110467047FB
:10C5180070B588B0202204460D466846002101F017
:10C52800BDFE20460495FFF7E5FF024658B16B466D
:10C53800054608AE1C4603CCB44228606960234611
:10C5480005F10805F6D1104608B070BD082817D9BE
:10C558000C280CD910280CD914280CD918280CD957
:10C5680020280CD930288CBF0F200E2070470920B6
:10C5780070470A2070470B2070470C2070470D2029
:10C5880070472DE9F843078C072F04461ED9D0E9D8
:10C59800029800254FF6FF73C5F12006A5F120008B
:10C5A80029FA05F108FA06F628FA00F031430143A2
:10C5B800C9B21846FFF782FF0835402D0346EBD174
:10C5C800E1693A46BDE8F843FFF789BF4FF6FF70C7
:10C5D800BDE8F88310B54B6823B9CA8A63F309022A
:10C5E800CA8210BD04691A681C600361C38A013BD2
:10C5F800C3824A60EFE72DE9F74F9846CB8A01924C
:10C60800C3F3090A5346052B81460E4632D05146DC
:10C6180000201FFA88F306F11A048DB2042D87B2A0
:10C628000FD8BB4201F1010106D8F28A534463F3E3
:10C638000902F28201201AE0019A155C6554013062
:10C64800EBE7BB42F1D9AAF1050B1C237468BBFBCD
:10C65800F3F103FB11BB1FFA8BF5002C45D14846BB
:10C66800FFF748FF044638B970606FF0020003B066
:10C67800BDE8F08F0027E6E70025056070601FFA27
:10C6880088F84FF0000BB8450ED9019B211D3B449B
:10C6980013F8010B4855A8B201371B28BFB22CD09C
:10C6A800B84505F10105F3D8F38A0AEB080262F3ED
:10C6B8000903F382BEE7013189B21C462368002BC7
:10C6C800F9D1A8F1050353441C20B3FBF0F301335F
:10C6D8009BB29942D3D2BBF1000FD0D14846FFF7A5
:10C6E80009FF20B9C4F800B0BFE70121E6E7C0F8A8
:10C6F80000B05D4620600446C1E7B845D4D9484635
:10C70800FFF7F8FE08B92060AFE7C0F800B00025D1
:10C7180020600446B7E72DE9F04F2DED028B1C464B
:10C7280083B05B69009207468846002B00F0A5801D
:10C73800238C2BB1E269002A00F09F80072B34D8A4
:10C7480007F10C00FFF7D6FE054638B96FF0020571
:10C75800284603B0BDEC028BBDE8F08F14220021FF
:10C7680001F09CFD228CE16905F1080001F0F8FD5B
:10C77800208C013080B2FFF7E9FEFFF709FE431E67
:10C788009BB25A1C23842A74626912782B4402F0E3
:10C798001F0262F03F021A7248F000436B6029469C
:10C7A8003846FFF70FFE0125D2E702339BB2072276
:10C7B800C18A0633B3FBF2F3828A521A9BB292B251
:10C7C8009342C3D800F10C034FF0000908EE103A69
:10C7D8004FF0800A4E464D4618EE100AFFF78AFEC3
:10C7E80083460028B2D01422002101F057FD002E04
:10C7F8003AD1009BABF8083002210BF1070C88B244
:10C808000728228C03D0964201F101012ED3013072
:10C8180080B20192FFF79AFEFFF7BAFD61690978C5
:10C82800013801F01F01964208BF4FF0400A1BFA79
:10C8380080FC41EA49114AEA01018CF808100130EC
:10C8480048F00041CBF804108BF8100059463846E0
:10C85800FFF7B8FD019A013596422DB289F001091A
:10C868004FF0000AB8D173E70021C6E7E269925D8C
:10C878000CF801200136B6B2C1E76FF0010567E791
:10C88800F8B515460E462C22002104461F4601F035
:10C8980005FD069B6360B5F5001F079BA76034BFC5
:10C8A8006A094FF6FF72A36297B2E66104F11000BD
:10C8B80000239A4206D800230360A782E3822383D9
:10C8C800E360F8BD0660013330462036F1E70378AF
:10C8D8001BB94BB2002BC8BF017070470078704776
:10C8E800F8B50C46C969074611B9238C002B37D116
:10C8F800257E1F2D34D83B782BBB228C072A2CD8B9
:10C90800268A36F003032BD14FF6FF70FFF7E7FDB9
:10C9180020F001003602400446EA0566400C46EA6B
:10C9280040254FF6FF72234629463846FFF7F3FEA7
:10C93800002807DD626913780133DBB21F2B88BF3B
:10C9480000231370F8BD228A2D0645EA02252046E9
:10C958001D43FFF716FE0246E5E76FF00300F1E717
:10C968006FF00100EEE770B58AB004461646002164
:10C97800282268461D4601F091FCBDF83830ADF814
:10C9880010300F9B05939DF840308DF81830119B9F
:10C9980007936946BDF84830ADF820302046CDE908
:10C9A8000265FFF79DFF0AB070BDD3692DE9F0411C
:10C9B80005460C4616460BB9138C5BBB377E1F2FFA
:10C9C80028D895F80080B8F1000F26D03046FFF738
:10C9D800D8FD3378210241EAC33141EA0801338A9C
:10C9E80041EA076141EA03410246334641F08001CA
:10C9F8002846FFF790FE00280ADD3378012B07D17F
:10CA0800726913780133DBB21F2B88BF00231370C0
:10CA1800BDE8F0816FF00100FAE76FF00300F7E777
:10CA280030B58BB01D469DF8443014465A1E53420B
:10CA380053418DF800309DF83830ADF810300F9B19
:10CA480005939DF840308DF81830129B07936A467D
:10CA5800BDF84C30ADF82030CDE90245FFF7A5FF11
:10CA68000BB030BD406A00B104307047436A1A68A1
:10CA7800426202691A600361C38A013BC38270473C
:10CA88002DE9F843D0F82090194F14461E46494620
:10CA98004FF0000809B9BDE8F883D1E90252651BD7
:10CAA80066EB0202AF4278EB02021DD2036A8B42A8
:10CAB8000ED1FFF78FFDD1F800900369C0F82090E0
:10CAC8000B60C38A0161013BC3824A461146E1E714
:10CAD800FFF780FD0A680369C9F800200B60C38A64
:10CAE8000161013BC382F1E70A688946EEE700BFAE
:10CAF80080841E002DE9F04F8BB00D46DDF8509074
:10CB080014469B468046002800F01681B9F1000FB4
:10CB180000F01281531E3F2B00F20E81012A03D12F
:10CB2800BBF1000F40F008810023CDE90833B8F8C5
:10CB38001430B5EBC30F4FEAC30703D300200BB083
:10CB4800BDE8F08F2B199F42D8F80C303ABF7F1BF5
:10CB5800FFB227461BB9D8F81030002B7AD0272D02
:10CB68004ED8C5F12806B7424FF000032CBFF6B2E5
:10CB78003E4600932946D8F8080008AB3246FFF72E
:10CB880062FCA7EB060A35445FFA8AFAB8F8143053
:10CB980003F10053053BDB000493D8F80C300393F2
:10CBA8002821039B13B1BAF1000F2CD1D8F810003B
:10CBB80040B1BAF1000F05D0009608AB5246691A89
:10CBC800FFF741FC38B2002FB8D067070AD00AAB8C
:10CBD80003EBD401624211F8083C02F0070213414A
:10CBE80001F8083C082C3CD9102C40F2B280202CCB
:10CBF80040F2B480BBF1000F00F09980082334E0C4
:10CC0800BA460026C2E7049BE02B28BFE023069320
:10CC18000B44AB42059314D95A1B039800969245CE
:10CC280034BF5246D2B2691A08AB04300792FFF7F4
:10CC38000AFC079A16441544AAEB0202F6B25FFAF8
:10CC480082FA049B069A05999B1A0493039B1B6816
:10CC58000393A6E70093D8F8080008AB3A4629469C
:10CC6800AEE7BBF1000F12D00123B4EBC30F69D0BC
:10CC7800082C11D89DF82030621E23FA02F2D6073C
:10CC880005D54FF0FF32A24013438DF820309DF8B0
:10CC9800203089F8003052E7102C11D8BDF8203028
:10CCA800621E23FA02F2D50705D54FF0FF32A240E3
:10CCB8001343ADF82030BDF82030A9F800303EE726
:10CCC800202C0ED8089A631E22FA03F3D90704D53C
:10CCD8004FF0FF33A34013430893089BC9F8003073
:10CCE8002DE7402C2BD0DDE90851631EC4F1210645
:10CCF800A4F1210225FA03F301FA06F6334321FAD7
:10CD080002F21343DB0712D50123A4F12002C4F178
:10CD1800200603FA02F223FA06F6A3405B4242EA2F
:10CD2800060262EB42022B430A43CDE90832DDE9F1
:10CD38000823C9E9002302E76FF00100FFE66FF05E
:10CD48000800FCE6082CA2D9102CB4D9202CEED867
:10CD5800C3E7BBF1000FAED0022386E7BBF1000F9B
:10CD6800BBD0042381E730B5012A144638BF01241B
:10CD7800402C85B028BF40240025012ACDE9025562
:10CD880018D81B788DF8083063070AD004AB03EB7A
:10CD9800D405624215F8083C02F00702934005F8F2
:10CDA800083C009103462246002102A8FFF74BFBEE
:10CDB80005B030BD082AE4D9102A03D81B88ADF87D
:10CDC8000830E1E7202A8DBFD3E900231B680293CE
:10CDD800CDE90223D8E710B5CB681BB98B600B618E
:10CDE8008B8210BD04691A681C600361C38A013B09
:10CDF800C382CA60F0E703064CBFC0F3C03002200C
:10CE0800704708B50246FFF7F6FF022806D1530619
:10CE1800C2F30F2001D100F0030008BDC2F30740A0
:10CE2800FBE700002DE9F04F95B0CDE902230A6831
:10CE380005461046FFF7DFFF022814BFC2F3062499
:10CE48000024002A0E46834680F2FC8112F0C04A74
:10CE580040F0F881097B002900F0F481022803D012
:10CE68002B78A34240F0F181C2F304630893104683
:10CE780002F07F0304933144FFF7C3FF049B91F84A
:10CE8800038005904FEA834949EA0B4949EA446916
:10CE9800002200235FEAD814CDE90A2349EA0009F1
:10CEA80069D0049B009302466F685B460AA928462E
:10CEB800B847002800F0CC812F6A4FB9494605F1E0
:10CEC8000C00FFF725FB074690B96FF0020056E00B
:10CED8003B6999450DD03F68002FF9D1494605F1C6
:10CEE8000C00FFF715FB07460028EED02B6A3B60C5
:10CEF8002F62F87D737B0693C0F3840008F01F034C
:10CF0800A0EB030C1FFA8CFEBCF1000FB8BF0EF1AA
:10CF1800200E0793A3EB000398B2B8BF0FFA8EFC5C
:10CF2800D7E90212002BB8BF20300993BCBF03B267
:10CF3800099351EA020097F81A90D7F804E075D0DF
:10CF48000298AF4B411A039860EB020200208B4213
:10CF580070EB02036AD3069B4B4518D14CB3BCF166
:10CF6800010F63DCBEF1000F60D1A64888427EEB5A
:10CF7800020215D36AE02F6A27B96FF00C0015B0CA
:10CF8800BDE8F08F3B699945B3D03F68F4E7DFF817
:10CF980074C28C4570EB0202F1D2002C00F088803C
:10CFA800099B0F2B42DD069B4B4540F08180002CEE
:10CFB8004CD1FB7DC8F34012B2EBD31F40F04B813C
:10CFC800079AC3F38403934240F04881327B4FEAC7
:10CFD8009813002C00F09F8013F0010840F0AD80FA
:10CFE800032A40F23E81029BBB60039BFB60FB8AE5
:10CFF800033A68F309035FFA82F906F10608FB822F
:10D0080042464B46394605F10C00FFF7F4FA002872
:10D0180057DA39462846FFF7DDFAFB7DC3F3840368
:10D02800013303F01F039B02FB824EE7FB7D08F0F0
:10D038001F0969F386036FF3C713FB753946284642
:10D04800FFF7C8FA069BBB76002C33D04FEA98133B
:10D05800022BAED0029BBB60039BFB601422002115
:10D068000FA801F01BF9029B0C93039B0D93331D32
:10D078000E93337B8DF848B0013BDBB2ADF84430FA
:10D08800059BADF84630079B8DF84930089B8DF815
:10D098004A30049B8DF84B300CA9AB68284698475A
:10D0A800FB7DC3F38403013303F01F039B02FB8260
:10D0B800002064E7FB7D09F1010969F38603FB752C
:10D0C8005BE7B3883B83DDE90A654FF6FF74CAF175
:10D0D8002002AAF1200326FA0AF105FA02F2114306
:10D0E80025FA03F319432046C9B2FFF7E7F90AF115
:10D0F800080ABAF1400F0446E9D1B8824A464146C7
:10D10800FFF7EDF9FB7DB882DA43C2F3C01262F390
:10D11800C713FB75CCE783B9013AD4B2043623466A
:10D128003246394605F10C00FFF765FA0028FFF68C
:10D1380070AFB88A22463146E2E7F98AD7F804E0A8
:10D14800C1F30901501E0429C0B253D80C4606F198
:10D15800030C002307F11B08984208D91CF8019F0B
:10D1680008F8049001340133052CDBB2F4D1834272
:10D178003ABF043356FA83F300231093059BADF8A6
:10D188004630079B8DF84930029C089B8DF84A3041
:10D198000C94049B039C8DF84B300D9401448DF83E
:10D1A80048B0002307F11B04ADF84410CDE90E4E3A
:10D1B800B88A7B60013A311DFFF791F93B8BB88241
:10D1C800834203D1AB680CA92846984728460CA986
:10D1D800FFF701FEFB7DBA8AC3F38403013303F032
:10D1E8001F039B02FB823B8B9A420CBF00206FF00F
:10D1F8001000C4E6BEF1000F21D17346B7E700BFA7
:10D2080080841E0040420F001C349C46DCF800302D
:10D21800002BF9D10C1BE31C06F103089C4404EB1A
:10D228000A09B9F11B0F5FFA8AF3A0D898429ED970
:10D2380018F8013F0CF8013F0AF1010AEFE7F4463C
:10D248000524E3E76FF0090099E66FF00A0096E617
:10D258006FF00B0093E66FF00D0090E66FF00E0094
:10D268008DE66FF00F008AE638B5204D2B685C6CB0
:10D2780022060BD59A6922F001029A611C4A1368AA
:10D288000721013328461360FDF70CFC04F0070260
:10D29800812323FA02F2D00704D5C4F30222D34033
:10D2A800D90711D42A68536C23F4E06323F00703E9
:10D2B80053640F4A5368013353600E4B1B781BB1FC
:10D2C8000A480721FDF7EEFB2B68620442BF5A6C3F
:10D2D80022F480425A641B6C13F47F0F05D0044A71
:10D2E800D168C3F307430B44D36038BDEC4E00202C
:10D2F8009C4A0020984A002030B5022A89B00D4681
:10D30800144661D800295FD00B88013B9BB2B3F566
:10D31800007F59D28B78002B56D0CB78013B1B0667
:10D3280052D40B79013B18064ED44C2200212A48CE
:10D3380000F0B4FFA11E294B4C424C411C70284BF5
:10D34800284C5A6D23605A6500234FF4807222825C
:10D35800A374C4E901332A88E3606261AA78E261B0
:10D36800EA7822622A79A2610122C4E90B22626268
:10D37800A26220460822C4E90E236363FDF7EEF992
:10D3880020BB4FF08043CDE90600029302230493AB
:10D398000546EBB2B3FA83F35B0902A9204605936D
:10D3A8000395FDF7BDFA034690B90135082DF0D174
:10D3B8000222009011460B48FDF7DAFA00280A48C5
:10D3C80008BF002009B030BD0848FBE70848F9E766
:10D3D8006FF4FA60F6E700BF9C4A0020984A0020E4
:10D3E80000640040EC4E00202EF8FFFF18FCFFFF01
:10D3F80030F8FFFF08B50448FDF7D6FA00280348BF
:10D4080008BF002008BD00BFEC4E00202DF8FFFF2C
:10D41800F0B50E468BB00546002849D0036813F0D6
:10D42800C04447D1002B45DA037B082B42D8244F50
:10D43800FFF71AFF3846FDF744FB60B9214B19681E
:10D44800002939D0711A0A2903D91F4A136C0133EC
:10D4580013640BB0F0BD3B68D3F8C43013F4001369
:10D468000CD0184B18680028F3D0311A0A2903D9B0
:10D47800154A536C013353642046EAE72A68099336
:10D4880022F0604201924FF08042CDE90223CDE9BB
:10D498000533CDE907332B7B2A1D1B0401A9384628
:10D4A8000493FDF797FA48B9064B01201E60D0E7B0
:10D4B8000648CEE70648CCE70846CAE70548C8E765
:10D4C800EC4E0020504F00209C4A002018FCFFFF23
:10D4D80016FCFFFF2CF8FFFF01684B0030B504D4A1
:10D4E8001F4A53690133536130BD8D0004D51C4A6E
:10D4F800936901339361F7E74268940204D5184AA7
:10D50800D3690133D361EFE7D30204D5144A136A10
:10D5180001331362E8E702F47023B3F5002F04D94E
:10D528000F4A536A01335362DEE70E4D0E4C2B88C7
:10D538002488013303F03F03A4B29C420BD00B4C68
:10D548002B801D0104EB031361515A6082689A60B5
:10D55800C268DA60C8E7024A136901331361C3E796
:10D568009C4A0020EA4E0020E84E0020E84A0020AD
:10D578002DE9F047DFF8E480D8F80040256D636DA9
:10D58800266D1D40636D1E4015F0070306F038092F
:10D5980010D0AA07236505D04FF0480AD4F8903078
:10D5A8001F0735D1AB0740D4680741BF2A4AD36A61
:10D5B8000133D362B9F1000F11D016F0180FC4F877
:10D5C800509004D04827D4F898301A0732D1F10681
:10D5D8003DD4B30641BF204A536B01335363226DD8
:10D5E800636D1A40236D616D12F4710203EA010341
:10D5F80003F4602304D0184922658A6B01328A63D8
:10D6080023B1154A2365D36B0133D363BDE8F08793
:10D61800D4F89070D8F84800C7F301270AFB070030
:10D62800FFF75AFFC4F89470B8E70B4A936A0133BE
:10D638009362B9E7D4F89850D8F84C00C5F301259F
:10D6480007FB0500FFF748FFC4F89C50BBE7024AF8
:10D65800136B01331363BCE79C4A0020EC4E002097
:10D66800034B1A68034B9A4201D1FFF781BF7047F9
:10D67800EC4E00200064004038B5114B114D1248A3
:10D6880000241C80114B4C2221461C8000F006FE11
:10D698000F4922462846FDF71AFA70B92B684FF051
:10D6A800FF321A650B4A934206D10B4BE02283F8EE
:10D6B80015234FF400121A6038BD0848FCE700BF74
:10D6C800EA4E0020EC4E00209C4A0020E84E002044
:10D6D8001B0008000064004000E100E060F0FFFF6C
:10D6E80038B50446002833D0FFF7BEFD1A4B1B4A55
:10D6F8001988138889B29BB299422BD013880133B9
:10D7080003F03F0313801901154A02EB0313525823
:10D7180022F0604242F0004222605A68C2F303429B
:10D72800082A28BF08222273E51C0021C8B28242B9
:10D7380088BF581801F101018ABF007A0020C0B2E1
:10D74800082905F8010FF1D100236373012038BDC2
:10D758000448FCE70020FAE7EA4E0020E84E0020E3
:10D76800E84A002018FCFFFF034A00231380034AFD
:10D778001380034A13617047EA4E0020E84E0020E8
:10D788009C4A00202DE9F0410E4686B00446002848
:10D7980044D0082942D81422002101A800F07EFDB7
:10D7A8004FF080430093DFF87880022302933746D6
:10D7B8000025B542EAB208D10024CDE90444184D49
:10D7C800FBB2082B20D100201BE0237A012B04D0C8
:10D7D800022B1CBF02F00102531C0393236801951E
:10D7E80023F0604304936368694623F0604340462E
:10D7F8000593FDF795F801350C340028D9D06FF45E
:10D80800FA6006B0BDE8F08169462846019703949E
:10D81800FDF786F801370028D2D0F0E70148F0E795
:10D82800EC4E002018FCFFFF1549D1E900321344E3
:10D838008A681344CA6813440A6913444A6913443A
:10D848008A691344CA6913440A6A13444A6A134426
:10D85800CA6A13448A6A13444A6B13440A6B134412
:10D868008A6B1344CA6B10B513440A6C13444A6C90
:10D87800044613444C228B6400F072FD204610BD10
:10D888009C4A00200F4B99420AD10F4B98420AD06C
:10D898000E4B984210D00E4B984210D00D4870474E
:10D8A8006FF47A7070477F212A23012010809170CD
:10D8B800D37013710020704777212823F5E73B21A7
:10D8C8001423F2E740420F0080FE210A006889090C
:10D8D80000B4C40448F4FFFF10B53024632807D807
:10D8E8000C703021092808D830301170187010BD1C
:10D8F80001346438E4B2C0B2F0E701310A38C9B281
:10D90800C0B2EFE730B5302442F20F75A84212D802
:10D918000C703021B0F57A7F14D211703022632850
:10D9280016D81A703023092817D8039A1370049B45
:10D938003030187030BDA0F51C5001341038E4B2F6
:10D9480080B2E3E70131A0F57A70C9B280B2E1E7AD
:10D9580001326438D2B280B2E1E701330A38DBB26F
:10D9680080B2E0E770B5324D324E3024A84232D84A
:10D978000C70314D314C3021A04230D811703049F3
:10D98800302288422FD21A702E4A302390422ED845
:10D99800049A13702C4A302390422FD8059A13709A
:10D9A800302342F20F7290422ED8069A1370302319
:10D9B800B0F57A7F2ED2079A1370302363282ED8B9
:10D9C800089A1370302309282DD8099A13700A9BD6
:10D9D8003030187070BD0134E4B23044C6E701310C
:10D9E800C9B22844C8E70132D2B2401AC9E70133A4
:10D9F800A0F57420DBB2A0F51070C7E70133A0F5DD
:10DA0800C330DBB2A038C7E70133A0F51C50DBB246
:10DA18001038C8E70133DBB2A0F57A70C8E70133E4
:10DA2800DBB26438CAE70133DBB20A38CBE700BFA0
:10DA3800FFC99A3B003665C4001F0AFAFFE0F505E6
:10DA4800809698003F420F009F86010010B58B1CFE
:10DA58000C464A1CFFF740FF0023E37010BD13B5C6
:10DA68000B1D0193CB1C00934A1C8B1C0C46FFF723
:10DA780049FF0023637102B010BD13B500280C469E
:10DA880014DA10F5004F14D0404280B22D222346FC
:10DA9800611C03F8032B621D0192221D0092A21C37
:10DAA800FFF730FF0023A37102B010BD80B220221F
:10DAB800EDE72D224FF40040E9E710B588B001F1F9
:10DAC8000903069301F108030593CB1D04938B1DED
:10DAD80003934B1D02930B1D0193CB1C00934A1C0F
:10DAE8008B1C0C46FFF73EFF0023A37208B010BD45
:10DAF80003099F2800F00F0094BF303337330928FB
:10DB08000B7094BF30303730002348708B707047EB
:10DB180013B50A46044601A9C0B2FFF7E9FF9DF80C
:10DB2800043093719DF80530D371C4F30720FFF7D3
:10DB3800DFFF9DF8043013719DF805305371C4F36D
:10DB48000740FFF7D5FF9DF8043093709DF8053026
:10DB5800D370200EFFF7CCFF9DF8043013709DF8AA
:10DB6800053053700023137202B010BD10B5034C7A
:10DB78002146FFF76BFF204610BD00BF544F002021
:10DB880010B5034C2146FFF76AFF204610BD00BFC1
:10DB9800544F002010B5034C2146FFF76EFF204676
:10DBA80010BD00BF544F002010B5034C2146FFF7AD
:10DBB80084FF204610BD00BF544F002008B502491D
:10DBC800FFF796FF084608BD544F002010B5034CD8
:10DBD8002146FFF79DFF204610BD00BF544F00208F
:10DBE80013B503688DF807109C680DF10701012330
:10DBF800A04702B010BD07B503688DF807101B6970
:10DC080001220DF10701984703B05DF804FB73B5D5
:10DC18001D460368019104465B69164698472368C8
:10DC280020461B6898470199221D2046FFF7D8FF18
:10DC38002DB123682A461B69314620469847236838
:10DC480020465B68984723689B690C21204602B0F0
:10DC5800BDE87040184773B51E4603680191044635
:10DC68005B6915469847236820461B689847221D1C
:10DC780001992046FFF7B4FF20460021FFF7BBFFBC
:10DC880023682046DB6832462946984723685B6844
:10DC9800204602B0BDE8704018472DE9F0411F4604
:10DCA800036804465B690D46164698472368204674
:10DCB8001B689847221D20461821FFF791FF290A63
:10DCC8002046FFF798FFE9B22046FFF794FF236844
:10DCD80031463A4620461B699847236820465B68C8
:10DCE8009847236820469B69BDE8F0410C211847F6
:10DCF80007B501238DF807200DF10702FFF7CDFFC7
:10DD080003B05DF804FB2DE9F0411F4603680446A3
:10DD18005B690D4616469847236820461B68984756
:10DD2800221D20461921FFF75BFF290A2046FFF72D
:10DD380062FFE9B22046FFF75EFF20460021FFF7A9
:10DD48005AFF23682046DB683A46314698472368DD
:10DD580020465B68BDE8F041184707B501230DF17F
:10DD68000702FFF7D0FF9DF8070003B05DF804FB3A
:10DD78002DE9F0411E46036804465B690F461546C7
:10DD88009847236820461B689847221D20461A2179
:10DD9800FFF726FF39462046FFF72DFF236829465F
:10DDA800324620461B699847236820465B68984797
:10DDB800236820469B69BDE8F0410C2118472DE9EE
:10DDC800F0411E46036804465B690F4615469847AE
:10DDD800236820461B689847221D20461B21FFF711
:10DDE800FFFE39462046FFF706FF20460021FFF7D1
:10DDF80002FF23682046DB68324629469847236895
:10DE080020465B68BDE8F041184737B504460D4623
:10DE18008DF80710012380210DF10702FFF7F7FEA7
:10DE28002368012D9B690CBF322140F2DC5120464A
:10DE380003B0BDE83040184707B501238DF8071037
:10DE48000DF107028A21FFF7E2FE03B05DF804FB3B
:10DE580007B50B0C8DF804300B0A8DF805308DF8DA
:10DE68000610032301AA8621FFF7D1FE03B05DF84F
:10DE780004FB07B502238DF804108DF805208F21C7
:10DE880001AAFFF7C4FE03B05DF804FB37B50C46E2
:10DE98008DF804108DF805208DF8063001AA0323AB
:10DEA8008B210546FFF7B3FE702C08D005D8502CFF
:10DEB80007D0602C05D0322204E0802CFBD1372219
:10DEC80000E01E22284640F62511FFF711FF012227
:10DED80040F63C112846FFF70BFF03B030BD07B5ED
:10DEE8008DF802309DF810308DF803309DF814300D
:10DEF8008DF8043000238DF800108DF801208DF87E
:10DF080005308DF806306A4607238C21FFF77FFE1F
:10DF180003B05DF804FB07B55BBAADF80430BDF893
:10DF2800103049BA52BA5BBAADF80010ADF8022009
:10DF3800ADF806306A4608238D21FFF768FE03B066
:10DF48005DF804FB07B5022301AA1521FFF783FE3C
:10DF58009DF804309DF8050000EB032080B203B063
:10DF68005DF804FB07B549BAADF80410022301AA0D
:10DF78009721FFF74CFE03B05DF804FB37B5054663
:10DF88000191FFF7DFFF019904462846FFF7EAFFF2
:10DF9800204603B030BD07B51F2928BF1F218DF8C3
:10DFA80004108DF80520022301AA8E21FFF72FFE09
:10DFB80003B05DF804FB13B5130A04468DF804108A
:10DFC8008DF805308DF80620032301AA8321FFF779
:10DFD8001EFE236864219B692046984702B010BD45
:10DFE80013B5130A04468DF804108DF805308DF822
:10DFF8000620032301AA8221FFF709FE2368642172
:10E008009B692046984702B010BD37B505230C46DA
:10E0180015461D216A46FFF71EFE9DF800309DF942
:10E028000110F02B84BF00238DF800309DF80030DC
:10E038005B085B42002923800B46B8BFCB1C9B10B2
:10E048002B700331BEBF22889B18238003B030BDDC
:10E0580037B502230D461446172101AAFFF7FBFD29
:10E068009DF804302B709DF80530237003B030BD47
:10E0780007B501238DF807100DF107029621FFF768
:10E08800C6FD03B05DF804FB07B501238DF8071042
:10E098000DF107029E21FFF7BAFD03B05DF804FBFE
:10E0A80010B5002304461A46C121FFF7B0FD2368C6
:10E0B80020469B69BDE810404621184738B50D46F3
:10E0C80040F691010446FFF748FE012D0ABF60F0B3
:10E0D8003F0200F03F02D2B240F691012046FFF71E
:10E0E80007FE38BD38B540F253110546FFF735FE37
:10E0F8004FF4AA7104462846FFF72FFE40EA042091
:10E1080080B238BD07B58DF804108DF805208DF85C
:10E11800063001AA03238B21FFF779FD03B05DF8D0
:10E1280004FB13B58DF802309DF810308DF80330DC
:10E138009DF814308DF804309DF818308DF80530AE
:10E1480008238DF800108DF801208DF806306A46F6
:10E1580007238C210446FFF75AFDBDF81C305BBA33
:10E16800ADF800306A46022340F6C8112046FFF792
:10E1780094FD02B010BD73B5C1F307230E0EC1F3B1
:10E18800074512F0FD0409BA019126D18C2E22D13F
:10E19800382D20D14AF6AC12ADF804209DF80420A1
:10E1A800632A0ED19DF805200E2A0AD123F0080310
:10E1B80042F66B2263F07F03ADF804208DF8063039
:10E1C800002404230DEB030240F6CF11FFF765FD91
:10E1D800204602B070BD0124E0E7141F18BF0124D7
:10E1E800EFE713B505230C466A461D21FFF733FDFB
:10E1F8009DF800305B085B42238002B010BD000030
:10E2080010EE100AC0F3C7527F3A162A15DC002A0E
:10E2180008DA013200F0004301D143F07E5300EEEA
:10E22800103A7047074911410842FAD04FF4800369
:10E238001341034423EA0103F1E7802AF1D130EEC8
:10E24800000A7047FFFF7F0010B501390244904271
:10E2580001D1002005E0037811F8014FA34201D055
:10E26800181B10BD0130F2E7884210B501EB02041B
:10E2780002D98442234607D8431EA14208D011F888
:10E28800012B03F8012FF8E7024401468A4200D126
:10E2980010BD13F8014D02F8014DF7E7024403469B
:10E2A800934200D1704703F8011BF9E710B5024605
:10E2B800147813460132002CFAD1013B11F8012BD6
:10E2C80003F8012F002AF9D110BDC9B2034610F88E
:10E2D800012B1AB18A42F9D118467047002918BF94
:10E2E8000023F9E710B56AB10139841810F8012B39
:10E2F80011F8013F9A4203D1A04201D0002AF5D17A
:10E30800D01A10BD1046FCE770B50D4D0D4C641BBE
:10E31800A4100026A64209D10B4D0C4C00F02EF893
:10E32800641BA4100026A64205D170BD55F8043B15
:10E3380098470136EEE755F8043B98470136F2E76F
:10E34800CC030108CC030108CC030108D40301085D
:10E35800034611F8012B03F8012B002AF9D1704765
:10E368000A44914200F1FF3300D1704710B511F80B
:10E37800014B03F8014F9142F9D110BDF8B500BF28
:10E38800F8BC08BC9E467047F8B500BFF8BC08BC8E
:04E398009E467047E6
:10E39C0000206C0002206A006D007400020501026E
:10E3AC0002016D696E2C00206D572C0020572C003B
:10E3BC00322E3447003931354D003836384D003463
:10E3CC0033334D003730636D003836364D003F0027
:10E3DC003530487A003331487A003139487A004672
:10E3EC004C52430046534B003139487A3778000180
:10E3FC001F136F011300000000D57FAAFE2B815460
:10E40C0029FC5683D702A87D52872DF8AC79D30608
:10E41C007BAE04D18550FA2FA471DB0E5A8F25F0F8
:10E42C008D58F22773A60CD9F623895C08DD77A2E8
:10E43C00DF0AA07521F45E8B9D48E23763B61CC9D8
:10E44C00B461CB1E4A9F35E0CF1AB06531E44E9BC8
:10E45C00E633994C18CD67B239EC4693C712B86DB8
:10E46C0010C56FBAEE3B91446BBE14C19540EA3FA8
:10E47C0042973DE8BC69C316EF3A904511C46EBB98
:10E48C00C613B96C38ED4792BD68C21743963CE988
:10E49C009441EB3E6ABF15C04B9E34E1B560CA1F78
:10E4AC0062B71DC89C49E33619CC66B3E732984D68
:10E4BC0030E54F9ACE1BB16472A70DD88C59F32658
:10E4CC005B8E24F1A570DA0F20F55F8ADE0BA17448
:10E4DC0009DC76A3F722885DD603A97C28FD578238
:10E4EC00FF2A805501D47EAB8451FB2E7AAF05D028
:10E4FC00AD78D20753862CF96162636465666768F0
:10E50C00696A6B6C6D6E6F707172737475767778F7
:10E51C00797A303132333435363738395F232D2E12
:10E52C0000000100010002000200020003000400D0
:10E53C000500060008000A000C0010001400190069
:10E54C002000280032003F00500064007D009E0037
:10E55C00C800FA003C019001F40176022003E803A4
:10E56C00E204DC05D0070000000000000000000001
:10E57C00190C00080000000000000000250C000829
:10E58C000000000000000000010C00086D6C7273AC
:10E59C002E300053657475705374617274537478B3
:10E5AC0034527800536574757053746172744D6194
:10E5BC00726B65720021656E6421004D6174656B30
:10E5CC00206D5232342D3330006D4C525301020306
:10E5DC0004006D4C525304030201000A000A455218
:10E5EC00524F523A20536F6C7574696F6E20666F80
:10E5FC00722043414E2074696D696E677320636F9E
:10E60C00756C64206E6F7420626520666F756E6425
:10E61C00000A202050434C4B313A20000A2020465F
:10E62C004443414E20434C4B3A20000A2020507268
:10E63C00657363616C65723A20000A202042533185
:10E64C003A20000A20204253323A20000A2020535C
:10E65C004A573A20000A4552524F523A20466169B5
:10E66C006C656420746F206F70656E2043414E2082
:10E67C00696661636520000A4552523A20726563EF
:10E68C0020000A43414E2073746172746564000A61
:10E69C0046696C746572000A202069643A20202057
:10E6AC00000A20206D61736B3A20000A0A0A43416C
:10E6BC004E20696E6974000A4552524F523A2066D8
:10E6CC00696C74657220636F6E6669672066616938
:10E6DC006C6564000A4552524F523A2063616E20B9
:10E6EC0069737220636F6E666967206661696C6519
:10E6FC0064000A4552524F523A2063616E20737483
:10E70C00617274206661696C6564000A43414E2035
:10E71C00696E697465640040504152414D2F7061BF
:10E72C0072616D2E70636B006D6C72732E000A201B
:10E73C0066632D3E7365723A2020200020683A20D3
:10E74C00000A207365722D3E66633A20202000205B
:10E75C00733A20000A2020206572722074785F665C
:10E76C0069666F2C2074743A2000202C2020000A3B
:10E77C0020202020202020206572722064632073CA
:10E78C00756D3A20006661696C2061005378206ECB
:10E79C006F74206F6B000000000000000000000090
:10E7AC006D1400085D140008D3230008FD23000835
:10E7BC001B240008111D00082B1100084F21000814
:10E7CC000000000000000000A5100008ED27000864
:10E7DC0085260008AB100008A97300086D87000897
:10E7EC00BD7D0008A1110008718C0008D51100082E
:10E7FC000000000000000000A5100008A710000891
:10E80C00A9100008AB100008AF100008B1100008E8
:10E81C00B5100008B9100008BB100008BF100008A4
:10E82C000000000000000000031F0008F520000895
:10E83C00B92000089920000800000000000000002A
:10E84C00A5100008F9110008A9100008AB10000869
:10E85C00A57B0008A5870008D57D0008C9630008C2
:10E86C00BB100008BF100008414E474C4500484FF4
:10E87C0052495A4F4E004E415620414C54484F4C31
:10E88C00440048454144494E4720484F4C440048B9
:10E89C0045414446524545004845414441444A009F
:10E8AC0043414D53544142004E415620525448006E
:10E8BC004E415620504F53484F4C44004D414E55FD
:10E8CC00414C00424545504552004C454453204F65
:10E8DC004646004C4947485453004F5344204F463A
:10E8EC00460054454C454D45545259004155544FE2
:10E8FC002054554E4500424C41434B424F58004624
:10E90C0041494C53414645004E4156205750004119
:10E91C004952204D4F444500484F4D4520524553D8
:10E92C00455400474353204E415600465056204113
:10E93C004E474C45204D495800535552464143458E
:10E94C0000464C415045524F4E005455524E2041BA
:10E95C005353495354004E4156204C41554E434855
:10E96C0000534552564F204155544F5452494D0077
:10E97C0043414D45524120434F4E54524F4C203150
:10E98C000043414D45524120434F4E54524F4C2071
:10E99C00320043414D45524120434F4E54524F4C4F
:10E9AC002033004F534420414C542031004F5344EA
:10E9BC0020414C542032004F534420414C542033BE
:10E9CC00004E415620434F5552534520484F4C441E
:10E9DC00004D43204252414B494E4700555345523E
:10E9EC00310055534552320055534552330055535F
:10E9FC00455234004C4F49544552204348414E47F0
:10EA0C0045004D5350205243204F564552524944D5
:10EA1C00450050524541524D00545552544C4500FE
:10EA2C004E415620435255495345004155544F20B1
:10EA3C004C4556454C205452494D00575020504C93
:10EA4C00414E4E455200534F4152494E47004D499D
:10EA5C005353494F4E204348414E4745004245458C
:10EA6C00504552204D555445004D554C5449204667
:10EA7C00554E4354494F4E004D4958455220505223
:10EA8C004F46494C452032004D495845522054526E
:10EA9C00414E534954494F4E00414E474C45204836
:10EAAC004F4C4400800CD007B704C71B800CB70434
:10EABC000410020A0B06972304100B060001020532
:10EACC00030400001CFE000850000000A001010817
:10EADC000300000000000000000000000000000027
:10EAEC00000000000000000000000000000000001A
:10EAFC00000000000000000000000000000000000A
:10EB0C0000000000000000000000000000000000F9
:10EB1C0000000000000000000000000000000000E9
:10EB2C000000000011003200140064001800FA000C
:10EB3C001B00F4011E00E80361626364656667688C
:10EB4C00696A6B6C6D6E6F707172737475767778B1
:10EB5C00797A303132333435363738395F232D2ECC
:10EB6C000000000000070E091C1B1215383F36313F
:10EB7C0024232A2D70777E796C6B6265484F464151
:10EB8C0054535A5DE0E7EEE9FCFBF2F5D8DFD6D141
:10EB9C00C4C3CACD90979E998C8B8285A8AFA6A131
:10EBAC00B4B3BABDC7C0C9CEDBDCD5D2FFF8F1F621
:10EBBC00E3E4EDEAB7B0B9BEABACA5A28F88818611
:10EBCC0093949D9A2720292E3B3C35321F18111601
:10EBDC0003040D0A5750595E4B4C45426F686166F1
:10EBEC0073747D7A898E878095929B9CB1B6BFB8E1
:10EBFC00ADAAA3A4F9FEF7F0E5E2EBECC1C6CFC8D1
:10EC0C00DDDAD3D4696E676075727B7C51565F58C0
:10EC1C004D4A4344191E171005020B0C21262F28B0
:10EC2C003D3A33344E49404752555C5B7671787FA0
:10EC3C006A6D64633E39303722252C2B0601080F90
:10EC4C001A1D1413AEA9A0A7B2B5BCBB9691989F80
:10EC5C008A8D8483DED9D0D7C2C5CCCBE6E1E8EF70
:10EC6C00FAFDF4F30000000032090000000000007F
:10EC7C00010000007C2B00000000000002000000DE
:10EC8C00890C00000000000004000000ED0E030CD5
:10EC9C000D00000005000000D91C01000000000060
:10ECAC0006000000680300000000000007000000E0
:10ECBC007720000000000000080000007524000010
:10ECCC00000000000B0000005906010400000000C9
:10ECDC001300000089180304050000001400000054
:10ECEC00D614030203000000150000009F0203006D
:10ECFC000100000016000000DC19000000000000FC
:10ED0C0017000000A81703040500000018000000FD
:10ED1C001834000000000000190000001765000006
:10ED2C00000000001A000000AA18000000000000FB
:10ED3C001B000000901D0000000000001C000000E3
:10ED4C0043100000000000001D00000073100000C4
:10ED5C00000000001E000000271C00000000000046
:10ED6C001F000000F6300000000000002000000032
:10ED7C00B91C00000000000021000000681C00000D
:10ED8C000000000022000000ED1600000000000052
:10ED9C0023000000F4160000000000002400000016
:10EDAC00DE2500000000000025000000D40703044D
:10EDBC000500000026000000090703040500000000
:10EDCC0027000000FE260320210000002800000080
:10EDDC00E605030203000000290000001C040302E6
:10EDEC00030000002A0000001C12000000000000BC
:10EDFC002B00000084030300010000002C00000025
:10EE0C00DD090302030000002D000000E8030300ED
:10EE1C00010000002E0000000B02000000000000AA
:10EE2C002F000000990803000100000030000000D2
:10EE3C002915010C0000000031000000271400000F
:10EE4C0000000000320000004E25031213000000E9
:10EE5C0033000000C405030203000000350000006D
:10EE6C000305000000000000360000000F1B031813
:10EE7C00190000003700000003190000000000001A
:10EE8C003D000000A7480000000000003E0000000C
:10EE9C00B71A0000000000003F00000077B500002A
:10EEAC000000000040000000BFE100000000000076
:10EEBC0041000000762A0000000000004200000023
:10EECC009406030203000000430000001504000038
:10EEDC000000000045000000F31E010A00000000C5
:10EEEC00460000007C2603101100000049000000C1
:10EEFC0026260320210000004A0000001414000004
:10EF0C00000000004B0000009E23031E1F000000A9
:10EF1C004C0000009821031E1F0000004D00000053
:10EF2C008F0A030809000000500000000E040302C1
:10EF3C0003000000510000006A16000000000000F1
:10EF4C005200000031330324250000005300000060
:10EF5C001625000000000000540000008F3503321D
:10EF6C0033000000550000008C330000000000004E
:10EF7C005600000005350332330000005700000036
:10EF8C00963300000000000059000000E71C000050
:10EF9C00000000005A000000B7380000000000001C
:10EFAC005B0000003F2A0000000000005C00000035
:10EFBC0036210000000000005D0000002F51000011
:10EFCC000000000064000000AF2200000000000000
:10EFDC00650000006675000000000000660000007F
:10EFEC009E7500000000000067000000D039000092
:10EFFC0000000000680000003874000000000000F1
:10F00C00690000005D3F0000000000006A00000085
:10F01C008A2C0000000000006B0000006C41000016
:10F02C00000000006C000000205C000000000000EC
:10F03C006D000000B9090000000000006E00000027
:10F04C0054FE0301020000006F00000022120310A6
:10F05C001100000070000000AE0C00000000000069
:10F06C00710000007C27000000000000720000000E
:10F07C00ED2C0000000000007300000004400000B4
:10F08C0000000000740000004C180000000000009C
:10F09C0075000000800603040500000076000000E7
:10F0AC00380E00000000000077000000740C030A0A
:10F0BC000B000000780000008661000000000000DA
:10F0CC0079000000ED020300010000007A0000004E
:10F0DC00CB020300010000007B000000FA7103006A
:10F0EC00010000007C000000573900000000000007
:10F0FC007D000000CB060000000000007E00000038
:10F10C00DC51034F500000007F0000001923000069
:10F11C000000000080000000E2230000000000005E
:10F12C00810000002E18000000000000820000008A
:10F13C001D0D00000000000083000000DFFF000038
:10F14C0000000000840000005527000000000000B3
:10F15C008500000006120000000000008600000080
:10F16C00E52B00000000000087000000CB08000029
:10F17C0000000000880000000116000000000000E4
:10F18C0089000000C3100000000000008A0000008D
:10F19C006D780000000000008B000000A82B0329F4
:10F1AC002A0000008C000000B529000000000000BF
:10F1BC008D0000002F200000000000008E000000D9
:10F1CC0048F30000000000008F00000083100000D6
:10F1DC0000000000900000007F5D000000000000B7
:10F1EC009200000067640000000000009300000023
:10F1FC009A3600000000000094000000B24E00009F
:10F20C000000000095000000C83C00000000000059
:10F21C0096000000862A0000000000009700000005
:10F22C00DB0803060700000098000000D00800006F
:10F23C000000000099000000BC0C00000000000061
:10F24C009A000000540F0306070000009B0000000A
:10F25C00160D0304050000009C00000013060300BB
:10F26C00010000009D000000150F030C0D000000B4
:10F27C009E000000860F030C0D000000A000000093
:10F28C004E0C030809000000A10000004403030019
:10F29C0001000000A2000000BD09000000000000F9
:10F2AC00A30000007F1C000000000000A400000070
:10F2BC009A2C000000000000A500000015030000BF
:10F2CC0000000000A600000015090000000000006E
:10F2DC00A70000009016000000000000A80000002D
:10F2EC00010C000000000000A9000000EA12000060
:10F2FC0000000000AA0000004922000000000000ED
:10F30C00AB000000B542000000000000AC000000A3
:10F31C001662000000000000AD0000005308000061
:10F32C0000000000AE000000A7300000000000004C
:10F33C00AF0000008A13030E0F000000B0000000A5
:10F34C00EA03030001000000B1000000F01400000B
:10F35C0000000000B20000002F18000000000000A8
:10F36C00B3000000BD1D011A00000000B400000035
:10F37C00342F012A00000000B5000000AE0400008C
:10F38C0000000000B6000000E528000000000000AE
:10F39C00B70000005502030001000000B800000097
:10F3AC009FCE030405000000B9000000BA07030457
:10F3BC0005000000BA000000481D03000100000019
:10F3CC00BF0000005C1B000000000000C00000003B
:10F3DC002436000000000000C1000000471A0000A5
:10F3EC0000000000C20000006221000000000000CC
:10F3FC00C30000007825000000000000C8000000D9
:10F40C00862A032829000000C9000000CD0E030C39
:10F41C000D000000D60000004508030607000000A0
:10F42C00D70000006503000000000000D8000000B9
:10F43C003203030001000000D9000000CA060000DE
:10F44C0000000000DA0000001107030001000000BA
:10F45C00DB000000A202000000000000DC00000045
:10F46C002220000000000000DD000000472A000000
:10F47C0000000000DE0000000F0300000000000090
:10F48C00DF000000772F032A2B000000E0000000B3
:10F49C00662D032A2B000000E1000000D04900007B
:10F4AC0000000000E2000000CF0800000000000097
:10F4BC00E6000000A32A000000000000E7000000A6
:10F4CC006928000000000000E800000097410000DF
:10F4DC0000000000E900000023B60000000000005E
:10F4EC00EA0000009628000000000000EB0000007D
:10F4FC00B32A000000000000F10000005A200000B8
:10F50C0000000000F2000000683C00000000000059
:10F51C00F3000000553D013400000000F400000031
:10F52C005F06000000000000F500000082020000F1
:10F53C0000000000F6000000B826000000000000EB
:10F54C00F70000005113000000000000F80000005C
:10F55C0008FE030304000000F9000000CC240000A6
:10F56C0000000000FA000000311E00000000000046
:10F57C00FB000000AA12000000000000FC000000CC
:10F58C002C12000000000000FD00000053360000AB
:10F59C0000000000FE0000002E090000000000002A
:10F5AC0000010000472A03080900000001010000C7
:10F5BC00830900000000000002010000BBE803000A
:10F5CC0001000000030100005CED000000000000E1
:10F5DC0004010000920E0000000000000501000074
:10F5EC00B33D000000000000060100000C170000F5
:10F5FC00000000000701000085FF00000000000073
:10F60C00080100003120000000000000090100008A
:10F61C001A140000000000000A010000C1FF0302E0
:10F62C00030000000B01000023FF03020300000095
:10F63C000C0100000E040302030000000D01000089
:10F64C006DD70000000000000E0100003B1400000C
:10F65C00000000000F010000163500000000000043
:10F66C00130100007E2000000000000014010000C7
:10F67C001232000000000000150100003E1E0000C8
:10F68C0000000000180100004621000000000000EE
:10F69C0019010000300D0000000000001A010000EC
:10F6AC007B230320210000001B0100004A91000075
:10F6BC00000000001C0100006320031E1F0000005E
:10F6CC001D01000089310326270000001E010000E7
:10F6DC00D2390332330000001F010000011703145C
:10F6EC001500000020010000141703141500000081
:10F6FC0022010000FB2E000000000000230100008E
:10F70C000A3900000000000027010000EA0C00008C
:10F71C00000000002A010000ED25000000000000A0
:10F72C002B01000013620000000000002C010000FF
:10F73C00D9160000000000002D010000F33A000073
:10F74C0000000000360100001C1100000000000049
:10F75C00370100005F740000000000004001000051
:10F76C00F3140302030000004101000058020300DF
:10F77C000100000042010000F395000000000000B1
:10F78C00430100004E9303000100000044010000FF
:10F79C0084920000000000004A01000017A700003E
:10F7AC00000000004B0100005BE9000000000000BD
:10F7BC004C010000ECEF0000000000004D010000C7
:10F7CC00E76D0000000000004E010000480A000038
:10F7DC00000000004F010000E118000000000000D4
:10F7EC0050010000F554000000000000530100001F
:10F7FC00C705000000000000540100006346000033
:10F80C00000000005E010000E8FC000000000000A9
:10F81C0062010000D20E030C0D0000006301000019
:10F82C00060C000000000000680100000B1900002D
:10F83C0000000000690100005D21000000000000D4
:10F84C007101000097180000000000007201000018
:10F85C001A8C000000000000730100000A1A00005E
:10F86C000000000075010000752A00000000000077
:10F87C0077010000FB8C0000000000007801000004
:10F88C00C7080000000000007C010000E814000024
:10F89C0000000000810100009385030203000000BA
:10F8AC0082010000841003040500000083010000A5
:10F8BC00044803040500000084010000082503200F
:10F8CC0021000000860100009CEE000000000000FA
:10F8DC008B01000000D40000000000008C0100002F
:10F8EC0032A00000000000008D010000B66C00008A
:10F8FC0000000000900100006EFE030405000000F3
:10F90C0091010000B7060304050000009A010000F5
:10F91C00A0350000000000009B0100006A030000FD
:10F92C00000000009C0100002106030405000000FB
:10F93C009D0100004D070304050000009E0100001E
:10F94C006D100000000000009F010000A1100000DD
:10F95C0000000000A4010000144903060700000089
:10F96C00B3010000862E000000000000B40100006E
:10F97C00C109000000000000B50100001E010000DC
:10F98C0000000000B801000042230000000000004D
:10F99C00B9010000A911000000000000FE010000E8
:10F9AC00F56A000000000000FF0100001C47000089
:10F9BC0000000000421F0000DA10000000000000F0
:10F9CC00431F0000E729000000000000441F000056
:10F9DC00AC62000000000000451F0000FB26000088
:10F9EC0000000000461F0000610E00000000000037
:10F9FC00471F00004020000000000000481F0000CE
:10FA0C00EA21000000000000491F000090100000D7
:10FA1C00000000004A1F00009B29000000000000AD
:10FA2C004B1F000014660000000000004C1F00007B
:10FA3C0036100000000000004D1F0000DE2E0000FC
:10FA4C00000000004E1F0000C80E00000000000067
:10FA5C004F1F00001718000000000000501F00008E
:10FA6C00951200000000000028230000718900009E
:10FA7C00000000002D230000752200000000000093
:10FA8C0011270000D1140000000000001227000014
:10FA9C00BA29000000000000132700000401000038
:10FAAC0000000000A7270000C35500000000000064
:10FABC00F82A00008634030405000000F92A00002F
:10FACC000F88000000000000FA2A0000EAB40304CA
:10FADC0005000000FB2A00004005000000000000AB
:10FAEC00FC2A00000BE8030809000000FD2A0000B6
:10FAFC005DE6000000000000022B00002E3100002B
:10FB0C0000000000032B00006A2C00000000000025
:10FB1C000C2B0000CD10000000000000162B000084
:10FB2C00902C000000000000172B0000852C00001A
:10FB3C0000000000182B0000552C000000000000F5
:10FB4C00192B0000C3250310110000001A2B000014
:10FB5C004F050000000000001B2B00008008030470
:10FB6C00050000001C2B0000B1220000000000006A
:10FB7C001D2B0000821C0000000000001E2B00004A
:10FB8C002F260000000000001F2B00008E09000033
:10FB9C0000000000202B0000842C0000000000005E
:10FBAC00212B0000D02C000000000000222B0000B4
:10FBBC00C92C000000000000232B0000C12C000009
:10FBCC0000000000242B0000BD2C000000000000F1
:10FBDC0064320000722C030001000000653200004A
:10FBEC00FE3B031E1F000000663200008C35030430
:10FBFC000500000067320000F92E03000100000030
:10FC0C00683200004D36031C1D00000069320000F4
:10FC1C00312B030001000000733200005EF9030079
:10FC2C0001000000763200008B3300000000000061
:10FC3C007732000007120310110000007832000028
:10FC4C0014050000000000006842000067B30000CB
:10FC5C0000000000FE4200001A210000000000001D
:10FC6C00FF420000481000000000000001430000AB
:10FC7C0013110000000000000243000059110000A5
:10FC8C0000000000034300001B0A000000000000FD
:10FC9C00044300000E5B0000000000000543000060
:10FCAC00BB54000000000000064300006A1800006E
:10FCBC000000000010A40000E301000000000000A0
:10FCCC0011A40000EF2E00000000000051C3000042
:10FCDC00F62000000000000052C30000B5F6000042
:10FCEC000000000053C300003E13000000000000A1
:10FCFC0054C30000F00A03080900000055C30000BB
:10FD0C00980603040500000020CB00000D640000E1
:10FD1C000000000021CB0000EF01000000000000FB
:10FD2C0022CB0000180100000000000023CB0000D3
:10FD3C00A61A00000000000024CB000027010000E0
:10FD4C000000000025CB0000910100000000000025
:10FD5C0060EA000004160314150000006AEA0000B3
:10FD6C00D0210000000000006BEA0000B707000083
:10FD7C00000000006CEA0000632403202100000056
:10FD8C006DEA000081180314150000006EEA0000F3
:10FD9C00860803040500000074EA0000CA04000091
:10FDAC000000000088EA00009CF500000000000044
:10FDBC0089EA0000BFFF0000000000008DEA00008F
:10FDCC000E170302030000008EEA0000AB1C0308B0
:10FDDC00090000008FEA0000370700000000000057
:10FDEC0092EA0000DC0E00000000000093EA000024
:10FDFC00F51800000000000094EA0000652C0000DB
:10FE0C000000000095EA00002D0600000000000034
:10FE1C003BB1B800ECC4B8009DD8B8004EECB800AB
:10FE2C000000B900B113B9006227B900133BB90047
:10FE3C00C44EB9007662B9002776B900D889B900EA
:10FE4C00899DB9003BB1B900ECC4B9009DD8B9008B
:10FE5C004EECB9000000BA00B113BA006227BA0028
:10FE6C00133BBA00C44EBA007662BA002776BA00C9
:10FE7C00D889BA00899DBA003BB1BA00ECC4BA006B
:10FE8C009DD8BA004EECBA000000BB00B113BB0009
:10FE9C006227BB00133BBB00C44EBB007662BB00A9
:10FEAC002776BB00D889BB00899DBB003BB1BB004A
:10FEBC00ECC4BB009DD8BB004EECBB000000BC00EA
:10FECC00B113BC006227BC00133BBC00C44EBC0089
:10FEDC007662BC002776BC00D889BC00899DBC002A
:10FEEC003BB1BC00ECC4BC009DD8BC004EECBC00CB
:10FEFC000000BD00B113BD006227BD00133BBD0067
:10FF0C00C44EBD007662BD002776BD00D889BD0009
:10FF1C00899DBD003BB1BD00ECC4BD009DD8BD00AA
:10FF2C004EECBD000000BE00B113BE006227BE0047
:10FF3C00133BBE00C44EBE007662BE002776BE00E8
:10FF4C00D889BE00899DBE003BB1BE00ECC4BE008A
:10FF5C000000891112239B322446AD573665BF74BD
:10FF6C00488CC19D5AAFD3BE6CCAE5DB7EE9F7F86D
:10FF7C008110080193331A22A5562C47B7753E649D
:10FF8C00C99C408DDBBF52AEEDDA64CBFFF976E84D
:10FF9C0002218B30100299132667AF763444BD557D
:10FFAC004AADC3BC588ED19F6EEBE7FA7CC8F5D92D
:10FFBC0083310A2091121803A7772E66B5543C455D
:10FFCC00CBBD42ACD99E508FEFFB66EAFDD874C90D
:10FFDC0004428D5316619F702004A9153227BB363D
:10FFEC004CCEC5DF5EEDD7FC6888E1997AABF3BAED
:04FFFC0085520C43DB
:020000040801F1
:1000000097711E60A1142805B3373A26CDDE44CF80
:10001000DFFD56ECE9986089FBBB72AA06638F721C
:1000200014409D512225AB343006B9174EEFC7FE60
:100030005CCCD5DD6AA9E3B8788AF19B87730E6240
:1000400095501C41A3352A24B1163807CFFF46EE40
:10005000DDDC54CDEBB962A8F99A708B08848195E8
:100060001AA793B62CC2A5D33EE1B7F04008C91930
:10007000522BDB3A644EED5F766DFF7C89940085F0
:100080009BB712A6ADD224C3BFF136E0C118480910
:10009000D33B5A2AE55E6C4FF77D7E6C0AA583B48C
:1000A000188691972EE3A7F23CC0B5D14229CB38F0
:1000B000500AD91B666FEF7E744CFD5D8BB502A4B0
:1000C00099961087AFF326E2BDD034C1C3394A28D0
:1000D000D11A580BE77F6E6EF55C7C4D0CC685D748
:1000E0001EE597F42880A1913AA3B3B2444ACD5BB0
:1000F0005669DF78600CE91D722FFB3E8DD604C770
:100100009FF516E4A9902081BBB332A2C55A4C4B8F
:10011000D7795E68E11C680DF33F7A2E0EE787F60B
:100120001CC495D52AA1A3B03882B193466BCF7A6F
:100130005448DD59622DEB3C700EF91F8FF706E62F
:100140009DD414C5ABB122A0B9923083C77B4E6A4F
:10015000D5585C49E33D6A2CF11E780F860010707B
:100160000410005B0000E86A4F09000098FF0000DF
:100170005018050C805B0040D41E000097FF000063
:100180006018050C805B00406A34000094FF00009A
:100190007018050C805B0040E75B000090FF0000DA
:1001A0002E0E440021EA00080000000074E8000858
:1001B000020000007AE800080300000082E800085E
:1001C000040000008EE80008050000009BE800081D
:1001D00006000000A4E80008FF000000ACE80008EA
:1001E000FF000000B4E8000807000000BCE80008B9
:1001F00008000000C8E8000809000000CFE8000877
:10020000FF000000D6E80008FF000000DFE800085B
:10021000FF000000E6E80008FF000000EEE800082C
:10022000FF000000F8E800080A00000002E90008EA
:10023000FF0000000BE900080100000014E90008BD
:100240000B0000001BE900080C00000024E9000876
:10025000FF0000002FE90008FF00000037E9000858
:10026000FF00000045E90008FF0000004DE900081C
:100270000D00000056E900080E00000062E90008C9
:100280000F0000006DE90008FF0000007CE9000895
:10029000FF0000008DE90008FF0000009EE9000853
:1002A000FF000000AFE90008FF000000B9E9000806
:1002B000FF000000C3E90008FF000000CDE90008CE
:1002C00010000000DDE90008FF000000E8E9000878
:1002D000FF000000EEE90008FF000000F4E900085C
:1002E000FF000000FAE90008FF00000000EA000833
:1002F000FF0000000EEA0008FF0000001EEA0008F0
:10030000FF00000025EA0008110000002CEA0008A8
:100310001200000037EA0008FF00000047EA00086A
:10032000FF00000052EA0008130000005AEA00082B
:10033000FF00000069EA0008FF00000075EA0008FD
:10034000FF00000084EA0008FF00000094EA0008B3
:10035000FF000000A5EA00081400000000000000F3
:1003600000000000A99B0008AB9B0008AF9B0008A1
:10037000B39B00080000000000000000010203041D
:10038000060708090000000001020304000102033F
:1003900004050607080C1014182030400100000066
:1003A0000200000004000000060000000800000039
:1003B0000A0000000C0000001000000020000000F7
:0C03C00040000000800000000001000070
:0803CC00FD010008ED9A000894
:0403D400D901000843
:1003D800010000000000000090BADCFE78563412DC
:1003E800D20400000A0000007DFF000004E80008B5
:1003F800D4E70008FF0000004CE800080024F400DF
:1004080001000000100000000000000000000000D3
:1004180000000000000000000100000000000000D3
:080428000000000000000000CC
:040000050800A5B991
:00000001FF
